:020000041000EA
:10000000002008205D0100101301001015010010F0
:100010001101001011010010110100101101001058
:100020001101001011010010110100101701001042
:100030001101001011010010190100101B01001026
:100040001D0100101D0100101D0100101D010010F8
:100050001D0100101D0100101D0100101D010010E8
:100060001D0100101D0100101D0100101D010010D8
:100070001D0100101D0100101D0100101D010010C8
:100080001D0100101D0100101D0100101D010010B8
:100090001D0100101D0100101D0100101D010010A8
:1000A0001D0100101D0100101D0100101D01001098
:1000B0001D0100101D0100101D0100101D01001088
:1000C0001D0100101D0100101D0100101D01001078
:1000D0001D0100101D0100101D0100101D01001068
:1000E0001D0100101D0100101D0100101D01001058
:1000F0001D0100101D0100101D0100101D01001048
:100100001D0100101D0100101D0100101D01001037
:1001100000BE00BE00BE00BE00BE00BEEFF3058004
:10012000103800BEF2EB887104410110304101101B
:10013000A801001090A31AE7D3DEFFFF42012110AF
:10014000FF010000AC4F0100793512AB4FF0000009
:100150002049086006C881F3088810474FF05040D6
:10016000006810B14FF00000F2E70FA40ECC002998
:1001700002D000F015F8F9E71749184A002000E00E
:1001800001C19142FCD1002080F30A8814498847BC
:10019000144988471449884700BEFDE701C901C2D8
:1001A0009A42FBD3704700BF30410110100100207C
:1001B000C4100020E45001100000082000000820B6
:1001C000E45001100010082000100820000000007A
:1001D0007047000008ED00E0C4100020989B02204A
:1001E0003D5B0010E1120010015B0010F8B500BF8C
:1001F000064B0749C91A891048BF0131491003D07D
:10020000044B0BB101481847704700BFC4100020D1
:10021000C41000200000000008B5054B1BB10549C3
:100220000548AFF30080BDE80840FFF7E1BF00BF1D
:1002300000000000F83C002040C0001038B57B4DA5
:100240002C68002C00F0A68044F001042047784B75
:10025000784A9B692A609A0600F182804FF05043E9
:100260001B68012B00F0BD800122734B1A60734B99
:10027000B3F900307F2B00F0AD806D4A936913F025
:100280002003FBD17F206E4910600A68013A00F11B
:100290009F800A60632A40F38F80002302202B6036
:1002A00038BD634B674A9B692A609B0658D44FF060
:1002B00050431B68012B00F09E8001225E4B1A60A8
:1002C000614A5E4B1178B3F900308B4200F08C80AC
:1002D000574A936913F02003FBD10D29116000F0F8
:1002E0008D807F2971D0564803685A1C0260574898
:1002F000C154CFE74E4B564A9B692A6098062FD4CB
:100300004FF050431B68012B5CD001224A4B1A600E
:100310004A4BB3F900300A2B00F08180444A9369BC
:100320009B06FCD40A231360B7E7414B494A9B69FB
:100330002A609C0614D44FF050431B68012B6BD0ED
:1003400001223D4B1A603D4BB3F90030202B5CD0AD
:10035000374A93699906FCD42021364B11602B60F3
:10036000012038BD324B3C4A9B692A60D806F7D43D
:100370004FF050431B68012B21D001222E4B1A60F5
:100380002B4A9369D906FCD411682E4B2E4A2B6058
:100390001170E5E7642221462C4806F0B1FE284B97
:1003A000234A1C609369D90606D49369DB06FCD402
:1003B00013689369DC06F8D5274B2B60D0E7274AF2
:1003C0001360DDE7254A1360A2E7224B2B60C7E7E5
:1003D0000B60F1E7164A93699B06FCD40D2313606A
:1003E0004BE71E4A136042E7114A93699C06FCD40E
:1003F0000D2313606CE7194A136061E7104A134834
:100400001168134A43542A60AAE7094A9369980677
:10041000FCD40D2313609BE7104A136093E7044A52
:1004200093699906FCD40D23136077E7183E0020EA
:10043000000007404E0200103C3D0020803F00209D
:10044000383D0020A2020010929B0220503D002067
:10045000F40200102A03001064030010403D002045
:100460002DE9F84F3F4B1F68002F78D13E4BD3F852
:100470000080B8F1000F1CD13C4E47463C4CDFF8E1
:10048000F490336811E000233A4D03EB430309EB8A
:10049000830328469B689847236832680133934258
:1004A000236005F10C05F0DB1346002B2760EADC26
:1004B000FEE7B8F1010F01D0BDE8F88F2C4C2B4EB0
:1004C000DFF8B090DFF8BC802B4DDFF8BCA0D8F887
:1004D000003032680133002AC8F80030276000DCA1
:1004E000FEE7DFF890B02F6002F0DCFD2368CAE978
:1004F000000103EB430309EB83039B6858469847CD
:100500002B68012B08D023683268013393422360A3
:100510000BF10C0BDBDAE6E72268184951F82230C0
:10052000013341F8223002F0BDFD8E46D4F800B010
:10053000134BDAF8041053F83B2003EBCB0CDAF83A
:100540000030D31ADCF8042062EB01021B180C48BF
:1005500042EB0E0240F83B30CCF80420B7E747F0FE
:1005600001073847443D00204C3D0020203E00203C
:10057000E8300020283E00203C3D0020283F00209D
:1005800048120020203F0020E81200202DE9F84FFB
:100590003F4B1F68002F78D13E4BD3F80080B8F155
:1005A000000F1CD13C4E47463C4CDFF8F4903368BA
:1005B00011E000233A4D03EB430309EB8303284684
:1005C0009B6898472368326801339342236005F1A2
:1005D0000C05F0DB1346002B2760EADCFEE7B8F1E0
:1005E000010F01D0BDE8F88F2C4C2B4EDFF8B090F6
:1005F000DFF8BC802B4DDFF8BCA0D8F800303268A3
:100600000133002AC8F80030276000DCFEE7DFF87D
:1006100090B02F6002F046FD2368CAE9000103EBA9
:10062000430309EB83039B68584698472B68012BCB
:1006300008D0236832680133934223600BF10C0B1E
:10064000DBDAE6E72268184951F82230013341F835
:10065000223002F027FD8E46D4F800B0134BDAF8B2
:10066000041053F83B2003EBCB0CDAF80030D31A1C
:10067000DCF8042062EB01021B180C4842EB0E026E
:1006800040F83B30CCF80420B7E747F00107384783
:10069000483D00204C3D0020243E0020EC3000204E
:1006A000A03E0020403D0020503F00209812002036
:1006B000243F0020F01200204FF050431B6830B45C
:1006C000012B24D024490B68092B05DD30BC002206
:1006D000224B1A60FFF7C4BE0024214A03EB4300FB
:1006E000850054511F4D02EB800043608560581C0B
:1006F0000A280860EAD002330B6000EB400399003F
:10070000545002EB8302184BC2E90103DEE717499C
:100710000B68092B05DD30BC0022154B1A60FFF772
:1007200035BF0024134A03EB4300850054510D4D9F
:1007300002EB800043608560581C0A280860EAD0FC
:1007400002330B6000EB40039900545002EB83022C
:10075000054BC2E90103DEE7203E0020443D0020B6
:10076000283E0020A10A0010A9110010243E0020FC
:10077000483D0020A03E0020F0B505680126044653
:1007800083B005B37E4D256016B9012003B0F0BDDE
:1007900002F088FC7B4FD7E9002390429941F4D3C3
:1007A0004FF050431B68012B00F0E7800122764B8D
:1007B0001A6002F077FC754B0026C01841F1000169
:1007C00038607960DFE7062700970B2732234FF464
:1007D000C8723146142000F0CDFF1421642001F0CE
:1007E00067F90F2001F076F9694801F0EBF932233F
:1007F000C822314640F2B310009700F0BBFF2846F4
:1008000001F068F902214FF4DE7001F051F9304631
:1008100001F058F95F4801F023FD0C2140F2BD10B2
:1008200001F046F95C4801F069F9162140F2BD106B
:1008300001F03EF9594801F061F9202140F2BD1064
:1008400001F036F9564801F059F92A2140F2BD105D
:1008500001F02EF9534801F051F97A21502001F0AE
:1008600027F9304601F02EF93946284601F03CF9C7
:100870007A214FF4AF7001F01BF90F230A222846AA
:1008800040F2DF1100F038FF40F2D511304601F0A0
:100890000FF9304601F016F929460F2001F024F92E
:1008A000414801F02BF90F230A22284640F2B711E4
:1008B00000F022FF40F2AD11304601F0F9F83B485C
:1008C00001F01CF90F230A22284640F28F1100F094
:1008D00013FF40F28511304601F0EAF8344801F088
:1008E0000DF90F230A22284640F2671100F004FF99
:1008F00040F25D11304601F0DBF82E4801F0FEF8C1
:100900000F230A22284640F23F1100F0F5FE40F284
:100910003511304601F0CCF8274801F0EFF840F2ED
:100920002B11C82001F0C4F829460F2001F0DCF893
:100930007721C82001F0BCF829460F2001F0D4F837
:1009400005F040FD1F211C2001F0D8FC2A46294655
:100950001C2001F0F1FC29461C2001F001FD0821BA
:10096000164B17481B68174A83F4005303F470436F
:100970000360044F024D11601BE7134A136018E730
:1009800086070010F81200203C3D002040420F0076
:1009900040C000104CC0001068C0001088C000109B
:1009A000A8C00010C4C0001078C20010D4C000104D
:1009B000D8C00010DCC00010E0C0001000000A40E9
:1009C00000100A4000200A40403D00200F22012371
:1009D00010B443EC40202649264A2748CB63916A4D
:1009E000036840F2FF100B44244C254913616268F0
:1009F0000B68244CA2F5FA62834224F813201DD020
:100A000001330B602049214B0A68214833F812302A
:100A1000FE2ADCBF01320A60C3F30B031D4943F415
:100A2000405303800E228B604FF0000343EC4020C4
:100A30000F2243EC40205DF8044B70474FF4807266
:100A400015480A600368D3E8CF1F01220029FAD1B4
:100A5000C3E8412F0029F6D1BFF35F8F0F4A002171
:100A60001368006801331360C0E88F1FCAE700BF36
:100A700000300B4000000B406809002000000A40D5
:100A8000640900209C180020103D0020F032002056
:100A9000889B022000000840783F0020D0200020E2
:100AA0002DE9F04F0368814687B0002B00F0868265
:100AB00043F001031847C74AC74913680160002B78
:100AC00000F0EB824FF050410968012900F071827B
:100AD0000120C2490860C249013B13600968002334
:100AE000C1E88F3F4FF48062BE49BF4806F0B2FCB8
:100AF000BE49DFF848834FF40072A1F5007006F09C
:100B0000A9FC282402F0CEFA4646B94D05F58067C7
:100B10000FFA84FA35F9021F0022504600F0C6FD94
:100B200036F9021F03220911C1F1780150462980CC
:100B300000F0BCFD0134AF42A4B2E9D1AD4CAE48E7
:100B40002146AE4D38F8022F30F8023F520013FB19
:100B500002F345454FEAA33321F8023FF2D14FF4A7
:100B600080620021A64806F0CBFA01200022A54EA3
:100B7000A54DA6F1020EAF1E4FF400735B1099183D
:100B8000B1F5007FFADA591E0A401A4482420DDD9F
:100B9000B6F900303EF91210318037F912102EF8F4
:100BA0001230B5F90030298027F812300130B0F545
:100BB000007F06F1020605F10205DDD108204FF0A5
:100BC000010A0146DFF838B20494CDF81490564675
:100BD000002E4FEA4A0A48DD0025CDE902160EEB49
:100BE00046090BEB4608029B884905FA03F303F11B
:100BF000800231F912C02A4631F8137001957F4204
:100C00003FB239F9120038F9123000FB07F103FB4B
:100C100007F503FB0CF300FB0CF0891301EBA33386
:100C20003EF912103BF91240C0F38F30C5F38F35F7
:100C3000C1F34F016E1801449BB2C4F34F04491B2A
:100C4000361A29F812602EF81210E11A234428F8F7
:100C500012102BF812305244B2F5007FD1DB019D07
:100C6000039B01359D42BED102990139AFD2DDE926
:100C700004494FF480626649664806F0EBFB4FF486
:100C800080625F49644806F0E5FB01200022634E64
:100C9000634DA6F1020CAF1E4FF400735B10991860
:100CA000B1F5007FFADA591E0A401A4482420DDD7E
:100CB000B6F900303CF91210318037F912102CF8D7
:100CC0001230B5F90030298027F812300130B0F524
:100CD000007F06F1020605F10205DDD108204FF084
:100CE000010ACDE904494B4FDFF82CB15646002EDE
:100CF0004FEA4A0A47DD0025CDE9020607EB46091F
:100D00000BEB4608029B414905FA03F303F180020D
:100D100031F912E02A4631F813C00195CCF1000CEC
:100D20000FFA8CFC39F9121038F9123001FB0CF073
:100D300003FB0CF503FB0EF301FB0EF180133BF9F3
:100D4000124000EBA33337F81200C1F38F31C5F323
:100D50008F359BB2A4B22E180844761A401BE11AB4
:100D6000234429F8126028F8121027F812002BF8F3
:100D700012305244B2F5007FD4DB019D039B013554
:100D80009D42BFD102980138B0D2DDE90449254D1A
:100D9000254A2946254802F5007732F8023F31F806
:100DA000026F974233449BB203F5FA66138020F832
:100DB000026FF2D100261E4B4FF400721D491E48EF
:100DC0001E6006F047FB2826DFF8748008F5806770
:100DD00038E000BFD0200020B60A00103C3D0020C3
:100DE000783F00209C1800209C1C00209C1A0020AA
:100DF000D2200020E22C0020869702209A2000209A
:100E0000DC280020E62C0020DE2800200013002033
:100E1000E42C0020F0380020F0340020F2380020CC
:100E2000F2340020EE380020EE300020EE320020B8
:100E3000103D0020F03A0020F03000209A1C0020E5
:100E4000DA2400200FFA86FA38F9021F00225046F1
:100E500000F02CFC032235F9021F50461141C1F16C
:100E6000C801A8F8001000F021FC0136B845B6B260
:100E7000E8D141F61A7743F67C1500208E4A8F4957
:100E800002F5806632F9023F31F902CF002BB8BF7C
:100E90005B42BCF1000FB8BFCCF1000C9BB21FFA53
:100EA0008CFC63459E4638BFE646634528BF6346D3
:100EB0000FFA8EFE1EFB05FC13FB07F34FEAAC3C5A
:100EC0000CEBA3337345B8BF7346964210800B807A
:100ED000D8D17B4E34F9020F01286DDD0246002384
:100EE00001215210012A1D464FEA410103F101037D
:100EF000F7D1421A033D2A4102EB03131BB223EA46
:100F0000E373A6422380E5D16E4EDFF8008230887D
:100F10004FF4EE74013000B2B0F51F7F0ABF0C230E
:100F200003461846684F338008F5A17501E0B6F90D
:100F3000000038F9023F402BB8BF4023403B1BB2B2
:100F40001A11911E062996BF02F1FF32002217F8EE
:100F5000122021B2A8F8003000F0A8FB013CA845FF
:100F6000A4B2E4D1594BC9F800301EE04FF0504311
:100F70001B68564A012B026000F091800122544BFD
:100F80001A60544B1A68D2E8CF0F01210028FAD119
:100F9000C2E8401F0028F6D1BFF35F8F4E4AC9F860
:100FA000002000221B68C3E88F2F012007B0BDE896
:100FB000F08F4A4801608EE50023A2E7484A0124E9
:100FC00092468346474D13802B8007EE904AF8EEF9
:100FD000E77A17EE900A0AF0FBFF33A3D3E9002368
:100FE00002F09EFB0022404B06460F4602F098FBA3
:100FF00002F02AFE2EA3D3E900238046894630461C
:10100000394602F0B3FB02F024FE002206460F46EA
:10101000364B4046494602F083FB0022344B02F037
:101020007FFB02F023FC32463B462AF8020F31498F
:10103000002002F061FB00222D4B02F071FB02F058
:1010400015FC0134B4F5007F25F8020FBDD102274D
:10105000294C2A49204605F0CDF9294B62685F608A
:101060002368284E284D83F00F033A4003F0CF0346
:10107000336001216A60062001F040F90121072058
:1010800001F03CF90121052001F038F901200F4B56
:10109000CBF8003007B0BDE8F08F0E4B81E70F4A68
:1010A00013606EE7AFF300806F1283C0CA2119404E
:1010B0000000000000F07F40DA280020E22C002031
:1010C000E22E00206009002098C400106C0F001070
:1010D0003C3D0020783F0020B60A0010403D002033
:1010E00000130020889702200000603F0000E03FCE
:1010F0000000D0400000F03F00000840002D31010A
:10110000003008400010084000200840EA2C002071
:101110000368014670B4002B2AD001221B4B0B60E0
:101120001AB31B4B9B699A061FD44FF050431B68A0
:10113000012B20D00122174B1A60174C174D226843
:10114000174BAE5CB3F90030B34217D01048836937
:101150009B06FCD40660531CED5C00222360002D2E
:10116000DCD102200D6070BC7047012070BC70475C
:10117000094C0A4DF0E70B4A1360DEE70448836927
:101180009B06FCD40D230360E0E700BF1C11001098
:10119000000007403C3D0020F43C0020B43D00200E
:1011A000803F0020403D0020036870B5064643B1F3
:1011B00043F001031847114B114A1249124805F038
:1011C000F1FE0022114B124C124D1A600FCD0FC4CC
:1011D00095E8030084E803000F4B0C483360FFF7E9
:1011E00097FF012808DD00220C4B1A600C4B33607E
:1011F000FFF724F80128DED8002070BD143D002040
:10120000183F0020FCC00010503D00201C3E002074
:10121000B43D0020E4C00010D8110010183E00209A
:10122000EC11001070B5C0B047222249064668464E
:1012300006F010F90021B9220DF1470005F060FF1A
:101240002F21684605F0AEFF002831D0441C1A4813
:1012500004F06AFE204604F0E5FD6846174905F0F3
:10126000B7FF174C154D03E02946002005F0B0FFED
:10127000214606F011F80028F6D1104905F0A8FF24
:101280000446104804F050FE204604F0CBFD0E4802
:1012900004F04AFE0D4A0E490E4804F045FE0E4881
:1012A00004F0C0FD31460D4804F03EFE40B070BD74
:1012B0006C46CCE7B4C1001004C100101CC1001082
:1012C00020C1001028C100103CC1001050C1001006
:1012D0005CC1001068C1001070C10010A0C10010F6
:1012E00070B584B06C460A2001F054FE04F052FD43
:1012F0004E4B4F4E0FCB07C468462380FFF792FF3B
:1013000000F0B6F8192001F02DF93060D0E8CF2FA9
:101310000123002AFAD1C0E8423F002AF6D1BFF3E8
:101320005F8F0124434A002533681460C3E88F5F50
:10133000192001F017F93060D0E8CF2F0123002ADF
:10134000FAD1C0E8423F002AF6D1BFF35F8F3A4A94
:1013500033681460C3E88F5F192001F003F930602F
:10136000D0E8CF2F0123002AFAD1C0E8423F002A5B
:10137000F6D1BFF35F8F314A33681560C3E88F5FE2
:101380002F4A304B166828461C642F4901F038F963
:101390002146284601F00EF92C4B0F209A6A16447C
:1013A0001E6100F0EDFF0F2344EC44300E2000F0EE
:1013B000E7FF0E2344EC443005F0A0F8244805F084
:1013C0000FF90A2001F0E6FD4FF050431B68A342DD
:1013D00017D0204A1368092B07DD00221E4B1A6024
:1013E000FFF73EF8002004B070BD0C205E1C1660B4
:1013F00000FB03F219491A4C8D500A44C2E901342A
:10140000EBE7184A1368092B0ADC0C205E1C1660F7
:1014100000FB03F21449124C8D500A44C2E9013416
:101420000022124B1A60FFF7B1F8DBE7FCC1001095
:10143000783F00201C3F0020E02C0020D02000201E
:101440006809002000200B40CD09001000000B406F
:10145000B9060010203E0020443D0020283E002018
:1014600079070010243E0020A03E0020483D0020C7
:101470002DE9F04F2DED028B7F498BB07F4804F0B2
:101480007BFE7F4981467D4804F076FE9FED788B98
:1014900080464FF0000A4FF4402B7A49774804F019
:1014A0006BFE8DED028B09F1080602AC06ADCDF89E
:1014B00014A0CDF810B009F101033603074646EA3F
:1014C000C31694E80F0085E80F00079695E80F0013
:1014D000012684E80F004FF4A023DFF8C4C10621E1
:1014E0001020CDF814C0029300F008FF10223346FC
:1014F00051466248009604F0BBFE23464A465146D8
:101500005E4804F0FBFE4FF4A023069308F10D03A0
:1015100008EB06021B0343EAC21323F0C04343F067
:1015200080430793584B062111200993CDF820B032
:1015300000F0E4FE1122334631465048009604F094
:1015400097FE2B46424631464C4804F0D7FE8DEDBF
:10155000028BCDE904BA07F1080CBB1C4FEA0C3C26
:101560004CEAC31C94E80F0085E80F00DFF834E173
:10157000CDF81CC095E80F0084E80F00062112206A
:10158000CDF814E000F0BAFE0621132000F0B6FEFC
:101590000621142000F0B2FE0621152000F0AEFE58
:1015A0000423122202213548009604F061FE2346EE
:1015B0003A460221314804F0A1FE304604F0F2FE22
:1015C0000446304604F0EEFE03464FF4163E2F4D1F
:1015D0002F493048DFF8D0804FEA841C0CF1A04C32
:1015E00001EA433105EA4435CCF8008041EA443150
:1015F000CCF8040045EA4330274F40F4802041F402
:10160000FC019B0103F1A04340F0110041F00901EE
:101610001A4ACCF808E0CCF810001F60C3F804C0E8
:101620009E6019615368D903FCD440F28F2313499B
:1016300013614B689A03FCD440F2DF130F4A4B61ED
:1016400053685B03FCD440F23F150123956140F2DF
:1016500007704FF0A0421149A3400860C2F850340F
:101660000BB0BDEC028BBDE8F08F00BFAFF3008084
:101670000000010000F00100E4D100100000205043
:10168000C0D10010A4D1001020460044FD1F00FC72
:10169000FD1F7EFC180020506C0900200020205007
:1016A0000002000452024010883F002010B540F2B2
:1016B000DF1E40F27F2C20EAE0707145A8BF714622
:1016C00060454FF42073A8BF604621EAE17111FB29
:1016D0000300084C4110C007635C06D503F00F03FC
:1016E00043EA0213DAB2625410BD23F00F031A4327
:1016F000625410BD883F00202DE9F0411618B04219
:101700002CDA40F2DF129142A8BF114640F27F2846
:1017100021EAE1721F0102EB8202154CFFB2D201F5
:1017200020EAE0714145D4BF02EB010C02EB080C4A
:101730004FEA6C0E14F80E101CF0010F01F00F0CA4
:1017400021F00F0100F1010547EA0C0C41EA030109
:1017500006D028B2B04204F80EC0E1DBBDE8F0814B
:1017600028B2B04204F80E10DADBBDE8F08100BF09
:10177000883F00202DE9F04F02EB000B58459DF803
:10178000246036DA5C183501A1428A46EDB230DABF
:10179000814640F2DF184FF420771B4940F27F2347
:1017A0000FFA89F020EAE0709842A8BF1846524626
:1017B00013B24345A8BF434623EAE37313FB070371
:1017C0004FEA630E11F80EC013F0010F2CF00F0357
:1017D0000CF00F0C02F1010243EA060345EA0C0C7F
:1017E00009D1944201F80E30E2D109F10109D9453D
:1017F000D4D1BDE8F08FA24201F80EC0D8D109F1D2
:101800000109D945CAD1F4E7883F00202DE9F04FFE
:10181000B0F5207F91B09DF868509DF86CC080F2C3
:10182000B080B1F5F07F80F2AC801F46062313FB39
:101830000C03002B40F3A58001EBCC03002B40F3FD
:10184000A0804FF000091FFA80FE974802EB820249
:1018500013182A01D6B28CB22846CDF804C040F243
:10186000DF1ACC467546B14626463A015FFA82FB3E
:10187000CDE90EE304F1080292B2DFF8308204925F
:1018800040F27F22BCF1050F16BF0F9B002413F816
:101890000C400E9BCDE90BC563441BB223EAE373F6
:1018A0009342A8BF1346019A06932BB20593B646FE
:1018B000134431463246254603930D96EE076CD508
:1018C000019C012C00F0BA80059B0CB21E460293CD
:1018D000039B9E423FDA019E2644B4423BDACDE9A7
:1018E00007154FF4207C0546DDF808E0CDE90242FB
:1018F000CDF8249040F27F220FFA8EF929EAE97997
:101900009145A8BF9146029802B25245A8BF5246DF
:1019100022EAE27212FB0C92541018F8041012F032
:10192000010F21F00F0201F00F0100F1010042EA66
:1019300007024BEA010127D1864208F80420E3D1CF
:101940000EF1010E7345D5D128460799DDF8249094
:10195000089D039A0393019C01322144049C92B296
:10196000A2424FEA550589B2A8D1DDE90BC5019B1A
:101970000CF1010CEB18BCF1060F0D9E9DB27FF42B
:101980007FAF11B0BDE8F08F864208F80410BBD1DC
:101990000EF1010E7345ADD1D6E7B842DBD0019C04
:1019A000012C66D0059E039B0CB29E42D3DA019BAC
:1019B0001E19B442CFDA4FF4207CCDE90721CDE9DE
:1019C000095BDDF814E0039B029440F27F220FFADA
:1019D0008EFB2BEAEB7B9345A8BF9346029D2AB270
:1019E0005245A8BF524622EAE27212FB0CB25410D2
:1019F00018F8041012F0010F21F00F0201F00F018E
:101A000005F1010542EA000249EA01010DD1B542A2
:101A100008F80420E3D10EF1010E7345D5D1DDE9BC
:101A20000721DDE9095B039395E7B54208F8041047
:101A3000D5D10EF1010E7345C7D1F0E714B254456C
:101A4000A8BF54464FF42076069B24EAE47414FBA6
:101A500006344FEA640C18F80C60E4074BBF06F03C
:101A60000F0426F00F044BEA04043C4308F80C4032
:101A700071E714B25445A8BF54464FF42076069B34
:101A800024EAE47414FB06344FEA640C18F80C6082
:101A9000E3074BBF06F00F0426F00F0449EA0404E5
:101AA000044308F80C4056E7A8CC0010883F0020FB
:101AB000024A034B10801980704700BF8C9B0220A4
:101AC0008E9B0220012838BF0120014B18807047EF
:101AD000909B0220024A034B10701870704700BFA1
:101AE000949B0220959B0220024A034B10701970B0
:101AF000704700BF959B0220949B02200278002A29
:101B000052D02DE9F0410446284D294F294E82B08C
:101B100011E00D2A0CD02B88092ADFF8A080264975
:101B200018B219D1B3F51F7F03F1040300D22B8043
:101B300014F8012F6AB10A2AEBD100221F49338819
:101B400009882A8003EBC103338014F8012F002A8F
:101B5000F1D102B0BDE8F08198F800E091F800C042
:101B60003B78CDF804E0B6F90010CDF800C0FFF7DF
:101B70004DFE134BB8F8001018782B8801EB410C80
:101B8000A1EB810203EB4C0352009BB202F52072E1
:101B90002B800028CCD09342CADD002233882A80D3
:101BA00003EBC1033380C3E7704700BF8C9B022067
:101BB000959B02208E9B0220949B0220909B0220EA
:101BC000969B02202DE9F04F0646007891B0002840
:101BD00000F04C81A74BA84A93F800E0A74B92F87D
:101BE00000801B88C6450C934FEA0E13D9B2A44B54
:101BF0000191B3F800B040F04981B14640F27F2531
:101C000040F2DF1A8C4606460BF1070292B20092B0
:101C10000BF1060292B29B4B01920BF1050292B2BC
:101C20000292994C03F10F020B9206930BF1010300
:101C30001BB223EAE373AB42A8BF2B460493069B77
:101C4000CDF8149003EB061110231A460B9B12FBE0
:101C500006360C9B5F1A0FFA8BF3BFB223EAE373CD
:101C6000013F039311E0900637D4D00653D41007F8
:101C70006FD4500700F18C80900700F1A780D20745
:101C800000F1C2808E4200F0D78011F8012B7B1842
:101C90001BB25345A8BF534623EAE37303EB830308
:101CA00010064FEAC31300F125825006DBD50498D5
:101CB00000EB03094FEA690814F8080019F0010F56
:101CC00015BF00F00F0020F00F004CEA00004EEAB4
:101CD000000004F808009006C7D50BF1020000B21E
:101CE00020EAE070A842D4BF03EB000903EB05092A
:101CF0004FEA690814F8080019F0010F15BF00F049
:101D00000F0020F00F004CEA00004EEA000004F83B
:101D10000800D006ABD50BF1030000B220EAE0705A
:101D2000A842D4BF03EB000903EB05094FEA690899
:101D300014F8080019F0010F15BF00F00F0020F093
:101D40000F004CEA00004EEA000004F808001007FB
:101D50008FD50BF1040000B220EAE070A842D4BF96
:101D600003EB000903EB05094FEA690814F80800C2
:101D700019F0010F15BF00F00F0020F00F004CEA22
:101D800000004EEA000004F8080050077FF574AF29
:101D9000BDF9080020EAE070A842D4BF03EB0009B7
:101DA00003EB05094FEA690814F8080019F0010F60
:101DB00015BF00F00F0020F00F004CEA00004EEAC3
:101DC000000004F8080090077FF559AFBDF9040042
:101DD00020EAE070A842D4BF03EB000903EB050939
:101DE0004FEA690814F8080019F0010F15BF00F058
:101DF0000F0020F00F004CEA00004EEA0000D2076E
:101E000004F808007FF53EAFBDF9002022EAE27237
:101E1000AA42D4BF9B185B195810225CDB0755BF40
:101E200022F00F0302F00F034EEA03034CEA030310
:101E30008E4223547FF429AF114B0BF1080B1FFA8C
:101E40008BFB0099019AA3F800B0DDF81490029B77
:101E500008310832083319F8016F89B292B29BB287
:101E6000009101920293002E7FF4E0AE11B0BDE824
:101E7000F08F00BF959B0220949B02208E9B022036
:101E80008C9B0220A8C40010883F0020B446B04BB1
:101E90004FEA081203F10F01CDE90AB1D7B240F2BF
:101EA0007F250BF1070240F2DF190446E346A94EF5
:101EB00092B20F930A990D920B4601331BB223EA9B
:101EC000E373AB42A8BF2B4609930BB223EAE3733B
:101ED000AB421846A8BF28468A46102308900F98A0
:101EE000CDF838B000EB04110B9813FB04045346F3
:101EF0000C980094A0EB010C981D0790581D0690BB
:101F0000981C0390D81C04331FFA8CFC059313B261
:101F10000CF1FF3C04900293B5E01AF0010F0BBFE7
:101F200020F00F0000F00F0048EA0000384306F8E8
:101F30000B00BDF90C0020EAE070A842D4BF03EB0F
:101F4000000A03EB050A94064FEA6A0B16F80B0029
:101F500000F143811AF0010F0BBF20F00F0000F0D9
:101F60000F0048EA0000384306F80B00BDF91000E6
:101F700020EAE070A842D4BF03EB000A03EB050A95
:101F8000D4064FEA6A0B16F80B0000F108811AF02C
:101F9000010F0BBF20F00F0000F00F0048EA000017
:101FA000384306F80B00BDF9140020EAE070A8429F
:101FB000D4BF03EB000A03EB050A14074FEA6A0BD0
:101FC00016F80B0000F1FF801AF0010F0BBF20F094
:101FD0000F0000F00F0048EA0000384306F80B003D
:101FE000BDF9180020EAE070A842D4BF03EB000A54
:101FF00003EB050A54074FEA6A0B16F80B0000F1D1
:102000009C801AF0010F0BBF20F00F0000F00F00B2
:1020100048EA0000384306F80B00BDF91C0020EA2E
:10202000E070A842D4BF03EB000A03EB050A940753
:102030004FEA6A0B16F80B0000F1BB801AF0010F93
:102040000BBF20F00F0000F00F0048EA00003843FB
:1020500006F80B0012F0010F029A22EAE2727BD11D
:10206000AA42D4BF9B185B195810325CDB074BBFE8
:1020700002F00F0322F00F033B4348EA03033354FB
:10208000009B994278D011F8012B08980CEB0103C2
:102090001BB24B45A8BF4B4623EAE37303EB830314
:1020A000DB0100EB030A4FEA6A0B140616F80B007B
:1020B00039D41AF0010F0BBF20F00F0000F00F0011
:1020C00048EA0000384306F80B000998540600EB74
:1020D000030A4FEA6A0B16F80B007FF51EAF1AF0E1
:1020E000010F40F0848020F00F004EEA000006F857
:1020F0000B001EE70398A842D4BF03EB000903EBD3
:1021000005094FEA690814F8080019F0010F15BF16
:1021100000F00F0020F00F004CEA00004EEA000033
:1021200004F80800C1E51AF0010F67D120F00F0094
:102130004EEA000006F80B00C7E71AF0010F78D14D
:1021400020F00F004EEA000006F80B0065E700BF24
:10215000A8C40010883F0020AA42D4BF9B185B1976
:102160005810DC07325C57D502F00F03019A134375
:102170003354009B994286D10A9B384908339BB25D
:102180000B80DDE90D2B1BF8014F0A9302F10803C8
:102190009AB2002C7FF48EAE11B0BDE8F08F1AF029
:1021A000010F4DD120F00F004EEA000006F80B00A1
:1021B000F9E61AF0010F28D120F00F004EEA0000D6
:1021C00006F80B0046E71AF0010F2BD120F00F00A4
:1021D0004EEA000006F80B0002E71AF0010F36D1B4
:1021E00020F00F004EEA000006F80B00BEE6019C4E
:1021F00000F00F00204306F80B009AE6019C00F067
:102200000F00204306F80B005FE7019C00F00F0071
:10221000204306F80B001DE722F00F034EEA0303EC
:1022200033542DE7019C00F00F00204306F80B000B
:10223000D6E6019C00F00F00204306F80B00ECE608
:10224000019C00F00F00204306F80B00ABE6019C58
:1022500000F00F00204306F80B0087E68C9B02205D
:102260002DE9F04FDFF88C9090F800B099F800A0BD
:1022700083B0BBF1000F31D01B4C1C4E0546D44639
:1022800020883388DFF87080194F01E099F800C08A
:102290005FFA83FE5A4698F80030B7F9001000B292
:1022A000CDE900CEFFF7B2FA208898F8003096F812
:1022B00000C001305A46B7F9001000B2CDE9003C29
:1022C000FFF7A4FA33882288C3EBC300104480B21E
:1022D000208015F801BFBBF1000FD7D189F800A00D
:1022E00003B0BDE8F08F00BF8C9B0220909B0220C2
:1022F0008E9B0220949B0220959B022010B44FF4E9
:1023000080740C4B53F8202003EB8003C00082F054
:10231000400200F1804003F5805C02F0C00200F54D
:10232000203003F54053CCF8002041601C605DF87C
:10233000044B70470480034010B4084CC90041EAC4
:10234000820154F8202004EB8003514003F58053B0
:1023500001F00C015DF8044B1960704704800340E4
:10236000064B402203EB800319B103F500531A60BA
:10237000704703F540531A60704700BF0480034064
:1023800030B44FF0000343EC440043EC400005251B
:102390004FF480740B4BC20053F8201003EB800005
:1023A00081F0400102F1804303F5203301F0C002C7
:1023B00000F5805100F540500A605D60046030BC5B
:1023C000704700BF048003400FB400B583B0049C85
:1023D000074803F027FD3CB105A92046019103F011
:1023E0005FFB044803F01EFD012003F071FB00BFFA
:1023F0000CC20010B0C10010EFF3108072B6064B93
:10240000D3E8CF1F01220029FAD1C3E8412F0029C8
:10241000F6D1BFF35F8F70477B1800200023034A7B
:10242000C2E88F3F80F31088704700BF7B18002000
:1024300070B58646EFF3108572B6124CD4E8CF6FB4
:102440000120002EFAD1C4E8460F002EF6D1BFF3CA
:102450005F8F4FF0010CC80801F007030CFA03F37B
:102460001EF800C01CEA030608D14CEA030C0EF863
:1024700000C0C4E88F6F85F3108870BD1046FFF769
:10248000A3FF00BF7B180020F8B5EFF3108572B6EC
:10249000234CD4E8CF7F0126002FFAD1C4E8476F40
:1024A000002FF6D1BFF35F8F9A4227D80126D708B5
:1024B00010F807E002F0070C06FA0CFC1EEA0C0FFD
:1024C00000EBD2070DD125E04FEAD20E10F80EE056
:1024D00002F0070C06FA0CFC1EEA0C0F00EBD20708
:1024E00018D001329342EFD24FF0FF300023C4E8FE
:1024F0008F3F85F31088984207DBF8BD0023C4E8BE
:102500008F3F85F310884FF0FF300029F5D00698F3
:10251000FFF75AFF4EEA0C0E104687F800E0E5E799
:102520007B180020044A1078431CDBB2182B28BF0C
:1025300010231370704700BF700900204FF0E02295
:10254000936843F000539360704700BF0021044B31
:1025500003F12002C3E88F1F01339342FAD1704781
:1025600070180020024B00221844C0E88F2F7047DB
:10257000701800204FF0E0234FF08032C3F80024A1
:10258000C3F80424C3F80824C3F80C24C3F81024A7
:10259000C3F81424C3F81824C3F81C24C3F8202457
:1025A000C3F82424C3F82824C3F82C24C3F8302407
:1025B000704700BF012300F01F029340400941B162
:1025C000800000F1604000F56140C0F88031036098
:1025D0007047024A203042F82030704700E100E0A6
:1025E0000123064A410952F8212000F01F008340D0
:1025F000134214BF01200020704700BF00E100E03B
:10260000F8B50D46EFF3108772B6124ED6E8CF2F0D
:102610000123002AFAD1C6E8423F002AF6D1BFF3CF
:102620005F8F0D4B00F110049B680C4A53F8243067
:10263000934203D0994201D000F028FF064B9B68DB
:1026400043F82450BFF35F8F0023C6E88F3F87F322
:102650001088F8BD7918002000ED00E01D01001081
:102660002DE9F04F83B0EFF3108A72B6744ED6E8BE
:10267000CF2F0123002AFAD1C6E8423F002AF6D123
:10268000BFF35F8F6F4B00F110089B686E4A53F8E1
:10269000285095423FD08D420C464AD06B4FEB1BE1
:1026A0002F2B38D801214FEA50194FEA890909F137
:1026B000604909F5614900F01F0301FA03F0D9F8F8
:1026C0000030C9F8800000EA030BBFF35F8FEFF31F
:1026D0000581C9B279B3884577D125F0010EDEF8BE
:1026E00008C0644505D17CE0D3F808C0644532D009
:1026F0009E469EF9062002EB4203002A07EB830365
:10270000F2DA644500F08180BBF1000F20D0C9F8F7
:102710008001C9F800004B4B9B6843F82850BFF379
:102720005F8F0023C6E88F3F8AF3108803B0BDE8AF
:10273000F08F1546EFE725F0010EDEF808C064457E
:10274000D7D19EF906407346002C08DA154666E09C
:10275000C9F88000DFE793F90640002C56DB04EB54
:10276000440C07EB8C0CDCF8082061009A609CF8A4
:102770000720DA719CF90620002A9A715DDBBCF80B
:102780000420520504D502F5FF1202F5FF521F3254
:10279000521502F1020C4FF0040E0C2212FB04E25F
:1027A00002EB4C026FF0070C3A44ACEB030C6244B2
:1027B000C2F34A0242F460429A80254B21441A78BF
:1027C00007EB81011C708A719EE7CDE9000100F0E2
:1027D0005DFEDDE9000125F0010EDEF808C064456C
:1027E00087D19EF906407346002CB8DA194A1A4C74
:1027F000D21A083AC2F30A316FEA01516FEA115155
:1028000044EA5202DA8099807EE773460029EDD1CE
:10281000FF228EF806204BF60152AEF804200C4C35
:102820004AF6AA2294F800C01946C91B49414A43F6
:10283000120D83F806C0227066E74BF60152BBE723
:102840007918002000ED00E01D010010740900203F
:10285000939B0220AE09002000F8FFFFF0B5EFF3D4
:102860000585EDB2EFF3108C72B62649D1E8CF2F73
:102870000123002AFAD1C1E8423F002AF6D1BFF372
:102880005F8F214E40F0010EB4684AF6AA2354F837
:1028900025701E4A0446A41A644163431B0D774504
:1028A0005BB21BD092F906409C421CD092F91240B8
:1028B0009C4223D092F91E409C4221D092F92A409A
:1028C0009C4208BF03240FD0114A002415781370CE
:1028D0008571C1E88F4F8CF31088F0BDB2680D4C44
:1028E00042F82540F0E7002404EB440402EB8402A4
:1028F000FF2494714BF601549480E5E70124F3E73B
:102900000224F1E77918002000ED00E074090020AE
:10291000939B02201D010010014B0B440360704784
:102920007018002070B5104C104DAC420ED2FF262E
:10293000236863B1FFF7F6FD01462046FFF7ECFF81
:10294000A680BFF35F8F0834AC42F1D370BDFFF7B0
:10295000E9FD01462046FFF7DFFF2671BFF35F8FD9
:102960000834AC42E4D370BDB4100020C410002081
:102970000D4B1A68EFF3108172B6D2E8CFCF012069
:10298000BCF1000FF9D1C2E84C0FBCF1000FF4D13B
:10299000BFF35F8F00221B68C3E88F2F81F310887D
:1029A00040BF0020002170477C3F00200000000055
:1029B0002DE9F04F2DED028B85B0EFF30583DBB2EF
:1029C000103B9A0818BF01224FF0010103F00300E9
:1029D00018BFAB4DAB4B08BFAB4D00EB820201FA09
:1029E00000FB53F8226005F541539FEDA38B019046
:1029F000C3F804B0CDF800B02AE0B388180440F161
:102A00008C80B379002B40F0D580B6F908100029EE
:102A1000C0F21581736901EB410103EBC103D3E9F6
:102A20000247B7F1FF3F08BFB4F1FF3F09D0019B58
:102A300005EB8301AB6A0A69D21AE31A934238BFE5
:102A40000C61284600F026FBA042B941C0F2F78095
:102A5000B6F90840009B002CEB63CEDBD6F814904F
:102A600004EB440A284609EBCA07D7E902B800F08C
:102A700011FB584571EB0801BFDBB8F1000FC0F244
:102A8000C180D7E90431814A934200F0EA807A8814
:102A9000B6F9080092B242EA0040984702460B4657
:102AA00052EA030100F0AE80002B80F2CE80BBEB37
:102AB000020B68EB030839F93A30C7E902B8002B7A
:102AC0009BDB716903EB430201EBC202D2E90270A6
:102AD000BB4578EB000C4FEA43028EDBB4462CF882
:102AE000083F0BE031F93230F446002B0DDB03EBED
:102AF000430001EBC0005A00D0E90270BB451A4404
:102B000078EB000001EBC20EECDA29F83A30ACF8B1
:102B10000040B38818043FF574AF3369EFF31082B7
:102B200072B6D3E8CF0F01210028FAD1C3E8401FC5
:102B30000028F6D1BFF35F8F4FF6FF74B0880023F3
:102B4000316900B2B480C1E88F3F82F310889842A7
:102B5000FFF657AF0746A946746906F1080807EB68
:102B6000470E04EBCE03D3E90250B6F90830C44651
:102B7000002BA8BFB34605DA0FE034F93A3094468B
:102B8000002B09DB03EB430A04EBCA02D2E9026122
:102B9000B54270EB0101F0DA5E46ACF8007034F932
:102BA0003E7024F83E30002FD9DAB3794D46002B21
:102BB0003FF42BAF0023B371B6F9083006F10808D3
:102BC000591C3CD01946776903E080465A1C3FF4F3
:102BD0001EAF03EB430207EBC200B0F802C01C4675
:102BE0001CF4004F9E4637F93230EED08C4280ED17
:102BF000028B05D0A8F80030318927F832103481D3
:102C00007146E3E739F83A3033813369EFF31082E4
:102C100072B6D3E8CF0F01210028FAD1C3E8401FD4
:102C20000028F6D1BFF35F8F7388316929F83A30F5
:102C300000237480C1E88F3F82F31088DDE640BF37
:102C400005B0BDEC028BBDE8F08F2846CDE902232C
:102C500000F020FA029A039B10EB020B43EB0108F1
:102C600029E708460B69029198470028CAD00299C3
:102C7000D1E9002314E700BFFFFFFFFFFFFFFFFFC5
:102C800000800B40183D002000000B40B1290010CF
:102C90002DE9F84F364C25692DB1BDE8F84F0A21D2
:102CA0003448FFF739BEDFF8E4800321404600F0E6
:102CB000DFF90326C4F80C80FFF734FC4FF0504CCA
:102CC0002D4B267003442361DCF800300F21637024
:102CD000636961801D834FF00405A3F878504FF0BD
:102CE0000505A3F890504FF00605A3F8A8504FF043
:102CF00007050E214FF6FF7208274FF00A0EA3F8C2
:102D0000C0504FF001094FF00C0C4FF0020B4FF088
:102D1000090A0D204FF00B05A3F868111749A2808E
:102D2000A3F808E1A160A3F848B0A3F8F0A0A3F8C5
:102D30002051A3F838C1A3F85001A3F83090A3F8AC
:102D40006060A3F8D8701A800D4B3046C8F8207028
:102D50000C49DC60FFF754FC49463046FFF72AFC7B
:102D6000094B0A211F640348BDE8F84FFFF7D4BDA3
:102D7000BC0900207C3F002070180020FFFF1000DD
:102D8000183D0020B129001000200B4000000B402E
:102D90000146F0B50069EFF3108772B6D0E8CF5F57
:102DA0000124002DFAD1C0E8454F002DF6D1BFF324
:102DB0005F8FB1F902E04C690EEB4E0CBEF1000FD3
:102DC0004FEACC0504EBCC0C3DDB605B0026488071
:102DD0000869C0E88F6F87F31088BCF80200CCE95F
:102DE00002230130C0F30E00012838BF0120059BEB
:102DF000ACF80200CCF81030069B40EA0E40CCF84C
:102E000014300B69EFF3108272B6D3E8CFCF0127ED
:102E1000BCF1000FF9D1C3E84C7FBCF1000FF4D135
:102E2000BFF35F8F8B886353A1F804E00B69C3E89D
:102E30008F6F82F310880122CB68097803F5015364
:102E40008A405A60F0BD00230A69C2E88F3F87F3C9
:102E500010884FF0FF30F0BD03464089B0EB214FA2
:102E600037DD58690A1402EB420210B500EBC200CC
:102E70001C69EFF3108C72B6D4E8CFEF0122BEF1DB
:102E8000000FF9D1C4E84E2FBEF1000FF4D1BFF30B
:102E90005F8F428889B292B28A4207D000221B69B2
:102EA000C3E88F2F8CF31088002010BD42F400423D
:102EB00042800121002218699971C0E88F2F8CF39C
:102EC00010881C78DA68084602F50153A140596061
:102ED00010BD0020704700BF2DE9F041861F41F171
:102EE000FF35B04271EB050338BF002682B038BF12
:102EF000354604460F4600F0D5F8301A65EB01035D
:102F0000012873F1000306DA2046394602B0BDE815
:102F1000F04100F003B900F0C5F8864265EB01010D
:102F200000290ADB0021174B3246009316482B4636
:102F30000191FFF72DFF0028E6DB4FF0000C13484E
:102F4000134A436A9D4204D8816AB142DCD29D4251
:102F5000DAD11368EFF3108172B6D3E8CF8F5FF048
:102F6000010EB8F1000FF8D1C3E848EFB8F1000F37
:102F7000F3D1BFF35F8F1368C3E88FCF81F310885D
:102F800020BFDEE771290010BC09002000000B40C3
:102F90007C3F002010B5044600F084F84FF47A73AB
:102FA0004FF0FF3C6FF00042E4FB0301BDE810402E
:102FB000844572EB01033CBF60461146FFF78CBFAE
:102FC000F0B506460D4683B0EFF30584E4B2002C5D
:102FD00035D1244F3A78F96804328B6A51F82220AF
:102FE000D21AC31A934207D320BF1F4B586AA84274
:102FF0001FD2002003B0F0BD00F054F8864265EB0C
:103000000101002911DB194B3846CDE90034324665
:103010002B46FFF7BDFE011E07DD134B5A6AAA427D
:1030200019D220BF0F48FFF717FF0F4B586AA8426D
:10303000DFD39B6A9E4209D8012003B0F0BD0A4B42
:10304000586A8842D5D39B6AB342F5D2401B18BF59
:10305000012003B0F0BD9B6A9E42E3D9AA42E1D1B0
:10306000DFE700BFBC09002000000B407129001001
:1030700010B4054B054C064AA04214BF1846581C14
:103080005DF8044BFFF7D4B9A420002000800B406A
:103090001CC200100346416A0A46986A596A8A426D
:1030A000FAD17047034B596A0A46986A596A9142A5
:1030B000FAD1704700000B4010B4174A536A9C467F
:1030C000946A536A6345FAD1001959414FF00002DE
:1030D00028BF01220346CAB10F4B596A4B1C08BFD7
:1030E0000B4608D04FF0FF310B460B48426A8A422C
:1030F000FCD38A4207D1084A02E0506A884202D1D2
:10310000906A9842F9D35DF8044B7047024A526ABC
:103110009142EAD8EDE700BF00000B40074A536A2E
:103120009942FCD8994207D1044B02E05A6A914275
:1031300002D19A6A8242F9D3704700BF00000B4067
:10314000F8B5054606200E4600F0E4F8002842D007
:10315000354A3648954214BF4FF080624FF0006206
:10316000334B344902601A608C6832EA0404FBD1A4
:103170002D4B4FF48071EB1AB3FA83F32E4A5B099F
:10318000062022F8131000F0C5F8C300B3FBF6F3D5
:103190000133DA0920D1402601216962AA622F6B2E
:1031A000FB0722D42B46002253F82C1F062003F5E0
:1031B000805422602F6300F0ADF840F20131032209
:1031C0008000B0FBF6F0EB6A83F0700303F07E033F
:1031D00023602963AA64F8BD4FF6FE718A421BD9A9
:1031E00022464FF6FF71154ED7E740F2013205F542
:1031F00040531A636B6AAC6A062004EB831400F038
:1032000089F80F4BA402A3FB0023DB0A0021B4FBC7
:10321000F3F0FFF751FFC5E7C3F34503114603EB96
:1032200082161A46B9E700BF00800740002002401E
:103230000030024000000240803F0020C0FF3F00FD
:10324000757B2B8F00EB400C4FEA8C0C0CF1804C03
:103250000CF5803CF0B51646DCF80420051FB2F5ED
:10326000803F38BF4FF48032EDB238BFCCF8042035
:10327000012D2AD94FF40067254C0CF540521760F8
:1032800054F82020B2B9DCF80020012D82EA461261
:1032900002F0E0020CF5805632602AD94FF400614A
:1032A00044F820304FF480330CF500521160CCF814
:1032B0000430F0BD6769B7FBF2FE0EF1010E0EEBB4
:1032C0004E0EBEF1030EFCD2DDE70129D2D103245C
:1032D0000CF540521460DCF80820D207FBD5DCF86E
:1032E00000200B4C82EA461202F0E0020CF58056F8
:1032F00032600122DCF800504D4005F003053560D6
:1033000002FA01F1DCF808200A42FBD0C6E700BF50
:10331000A8200020014B53F820007047A82000206F
:1033200070B4039D04682D0345EA03451B4B002C34
:10333000B3FBF1F3B2FBF3F61FDB194A194B9042D2
:1033400014BF4FF480424FF40042174C1A6003F54B
:1033500080531A60A36832EA0303FBD1212200F5EF
:1033600040530433016086601A600268002AFCDA68
:103370000822C5601A6070BC7047036803F03F0301
:103380008B42DAD18368C3F30B03B342D5D1C36850
:1033900003F4EE23AB42D0D1EDE700BF001BB70032
:1033A000008005400020024000000240012300EBA5
:1033B0004000800000F1804000F58410416003600F
:1033C000704700BF002370B5DB8A04460D4600221B
:1033D00042E800F2520254BF1021042144F252206C
:1033E000984786462B462246F446BDE870400A219F
:1033F0004FF48170604700BF0023DB8A002242E85F
:1034000000F2520201D4102118470421184700BFCE
:1034100008B503460846191E02DB1AB140F0300019
:10342000FFF7D0FF40F02000FAE700BF034AD2F8D0
:103430002838002BFBD0BFF35F8F704700000E4091
:103440000021044B044ABFF35F8F43F8041B9342EF
:10345000F9D170470C080E402C080E4010B42F20F4
:103460004FF42A64054A064B06491460D06019607F
:103470005368002BFCDA5DF8044B70470080044071
:1034800000A0044000B0FA00704700BF08B5014832
:10349000FEF79AFF40C2001038B5054C054DAC420E
:1034A00004D254F8043B9847AC42FAD338BD00BF6D
:1034B000F8BF001038C0001038B5054C054DAC42BF
:1034C00004D254F8043B9847AC42FAD338BD00BF4D
:1034D00024C0001038C0001010B40748074C084B37
:1034E000084A094904601A608B6832EA0303FBD179
:1034F0005DF8044B704700BF002002407F3BEFEFB8
:1035000000300240F6FFF30300000240044BDB6C86
:10351000B3F5004F03D14FF48022024BDA647047B9
:1035200000001150002011504FF0E022044BD2F85F
:10353000881D0B43C2F8883D10EE3004704700BF71
:10354000030330006FF06041044B054A1960936833
:10355000DB4333F06043FAD1704700BF00300240D4
:103560000000024010B545F25320FFF745FFBDE8CB
:10357000104003460420184710B545F25320FFF7CA
:103580003BFFBDE81040034601201847FEF7DEBFB1
:1035900010B5054B054C4FF488721846A16803F02E
:1035A00059FFA06010BD00BF0000002000ED00E04A
:1035B000002370B52B4C82B0C4F88430FFF74EFF67
:1035C0000122294BDA63636C012BFCD10321264ACB
:1035D000244B11639C6B012CFCD10226052521464E
:1035E0000523224A22480096FFF79AFE21462B46E1
:1035F000204A21480095FFF793FE0022042031461F
:103600001E4BFFF71FFE2146284600221C4BFFF7EA
:1036100019FE0022082011461A4BFFF713FE002264
:1036200009201146174BFFF70DFE00220620114618
:10363000134BFFF707FE0022114B07201146FFF73F
:1036400001FE0420FFF766FE00240F4BA3FB0035AC
:10365000AD0CE0B229460134FFF7A8FE062CF8D1E4
:1036600002B070BD0000014000300140002F6859D9
:1036700000000540008C864700800540001BB70015
:1036800080D1F008006CDC0283DE1B4386B003B4FB
:1036900051FC0804CDE9020151FC0904CDE9040103
:1036A00051EC0A04CDE9060103BCF047BDE8005027
:1036B0004EEC00C4BDE800504EEC01C4BDE8005023
:1036C0004EEC02C400BD000000B5FFF7DFFF02E0D2
:1036D00010FE30F4F8D441EC100443EC112400EE59
:1036E000010410EE010480EE200451EC1004704738
:1036F00000B5FFF7CBFF02E010FE30F4F8D441EC48
:10370000100443EC112400EE010410EE210480EEBD
:10371000200451EC3004704700B5FFF7B7FF02E01A
:1037200010FE30F4F8D410B541EC100443EC112431
:1037300051EC040453EC0524A0FB024C5FF0000E96
:10374000E0FB03CEE1FB02CE4CEC20440024E1FB85
:1037500003E444EC30E480EE200451EC5004BDE876
:103760001040704700B5FFF791FF02E010FE30F403
:10377000F8D441EC100443EC112451EC2104A0FBDB
:1037800001126FEA820252FB100052FB12F252FB4E
:103790001000A0EBD07C53EC04245CFB13F153EC41
:1037A0001524A1FB022001FB030053EC4424A2EBEF
:1037B000000050FB1CF24FEA111312EB017043EBB7
:1037C000E27140EA515020EA915020F0070053EC9A
:1037D0007524A0FB023C53EC752400FB03CC01FBD9
:1037E00002CC53EC0424ACEB824C40EA5C70A0F1B8
:1037F000010041EC400480EE200451EC700470475D
:1038000000B5FFF743FF02E010FE30F4F8D441ECBE
:10381000100480EE220410EEB204704700B5FFF7EA
:1038200035FF02E010FE30F4F8D440EC700400EEF6
:10383000010410EE210480EE200451EC30047047A6
:1038400000B5FFF723FF02E010FE30F4F8D440EC9F
:10385000600400EE010410EE210480EE200451EC1F
:103860003004704700B5FFF711FF02E010FE30F49E
:10387000F8D441EC800400EE010410EE010480EE67
:10388000400410EE1304704700B5FFF7FFFE02E09E
:1038900010FE30F4F8D441EC800400EE010410EE88
:1038A000010480EE400410EE3304704700B5FFF7CA
:1038B000EDFE02E010FE30F4F8D441EC100443ECCD
:1038C000112400EE010410EE3004C0F300707047C4
:1038D00000B5FFF7DBFE02E010FE30F4F8D441EC57
:1038E000100443EC112400EE010410EE3004C0F388
:1038F0008070704700B5FFF7C9FE02E010FE30F49B
:10390000F8D443EC102441EC110400EE010410EE55
:1039100030F48CBF01200020704700BF00B5FFF7D6
:10392000B5FE02E010FE30F4F8D443EC102441EC74
:10393000110400EE010410EE30F42CBF0120002031
:10394000704700BF00B5FFF7A1FE02E010FE30F4A3
:10395000F8D441EC100443EC112400EE010410EE05
:1039600030F42CBF01200020704700BF00B5FFF7E6
:103970008DFE02E010FE30F4F8D441EC100443EC6C
:10398000112400EE010410EE30F48CBF0120002061
:10399000704700BF000000000000000000000000B1
:1039A000DB60BE284A059193F4D5097F70374D7DC1
:1039B00066A5D83610E4104FEA58947F58F1AEF758
:1039C0008E1BC96DB8749390BA4B92018764748250
:1039D000C77A873FCF694A2C7D8D20BA21D1AE4B63
:1039E000091C673A90DF17AD8E75644E7DCED460AA
:1039F000E21721270E4A7EEFFF25FEC7036681F7F7
:103A000062C4CBFB479B82D6B39F4DDB6DC2F2C92C
:103A1000D98FD1D38BFA97A7B1EE495D5E7CF9FAC5
:103A20007DCE41CFBAA494E2ECD7FE9A4257E34749
:103A300011CC8015174B02F01F054FF00107AF4066
:103A40005FEA6218A7FB00450026E7FB015603EB7F
:103A50008803D3F81090A9FB06A7D3F80C90A9FB14
:103A600005A8E9FB6678D3F8089009FB0688E9FB0E
:103A70000578A9FB04A6D3F8049009FB0588E9FBA7
:103A80000478D3F8009009FB0488BF1948F10008B6
:103A9000704700009839001050EA013208BF41F029
:103AA000004141F400210B00020070470BB90020D7
:103AB0000021002240F20003C3F6F0731CF0020F55
:103AC0001CBF1046194670470022002300245FF0F7
:103AD000004504E14DF804CD5FF0000C0CF1040C3E
:103AE00002F10402FFF7A6FF98EAE879B9F1807FB6
:103AF00002D2BCF1400FF1D197EAE87741F2A61665
:103B0000C0F64636A9FB06A04DF21156C4F67E0655
:103B1000A7FB06A1E9FB66010626E7FB060109FBF8
:103B20000611DCF1200A57D421FA0CF320FA0CF22A
:103B300001FA0AF942EA0902A2FB0394A2FB0395E7
:103B4000E3FB6345A4FB0596A4FB0597E5FB6567CE
:103B5000F60856EA47764FF0AA39A6FB0967D4EB78
:103B6000070675EB45075FEA2739360B56EB075614
:103B700059F17F6717F14057C0B4A0FB0592A1FB34
:103B80000493E1FB6523A2FB0596A3FB0497E3FBEB
:103B900065674FF0AA39A2FB09A40025E3FB09459C
:103BA000641955F100054FF08839A6FB0923B4EBE1
:103BB000131465F10005B0EB940061EBA501B0EBC7
:103BC000857061F10001CCF58064A4F10E0400F071
:103BD00082F9BDE8C0100CE0CCF58064A4F10E04BD
:103BE00000F079F95DF804CB002640F20007C3F637
:103BF000F0775FEAD87868F3000C5FEA6C090FD4BD
:103C00005FEA690906D31CF0040C57EA4C713000D6
:103C1000BDE8F0879CEA9C0C51EACC71BDE8F087C6
:103C20001CF0040497EA4477C0B4A6E03CB500F069
:103C300004F830BC03C40CC530BD11F0004C5FEA81
:103C40005C0C5CF0004C06E05FEA517C1CF0040C5C
:103C500001E05FF0020CC1F30A53A3F2FF32B2F5A8
:103C6000806F3FF419AF12F1200FFFF61FAF012351
:103C700063F31F512DE9F04702F10C02FFF7DAFE62
:103C80005FEA987444F10004A8EB84780CEB440CD0
:103C90004CEAD87C97EAE87798EAE878B8F5800F9C
:103CA000FFF418AF41F2A619C0F64639A8FB09A0E7
:103CB0004DF21159C4F67E09A7FB09A1E8FB690181
:103CC0005FF00609E7FB090108FB0911B1F1007F6C
:103CD000FFF4FAAECA0E7C4B03EB02133CCB801A06
:103CE000994110D45FEA6C0636D476101CD200F0ED
:103CF0006CF800F0AFF800F0ECF89CEA9C0C51EA8C
:103D0000CC71BDE8F0875FEA6C0649D4761017D213
:103D100000F058F800F0ACF800F0D8F89CEA9C0CE1
:103D200051EACC71BDE8F08700F04FF800F0AFF831
:103D300000F0CCF81CF0040C51EA4C71BDE8F0879F
:103D400000F040F800F0B2F800F0C3F81CF0040CEA
:103D500051EA4C71BDE8F08700F037F8FCB400F090
:103D600096F800F0B3F81CF0040491EA4471FCBC2E
:103D700003B400F06FF800F0ACF89CEA5C0494EA3D
:103D80009C0491EAC4711CF0020F1DBF02460B4651
:103D900003BC0CBC1CF0804491EA4401BDE8F087F0
:103DA00000F010F8FCB400F081F800F092F81CF07C
:103DB000040491EA4471FCBC03B400F059F800F02B
:103DC00085F8DAE7404261EB4101A1FB0167A0FB06
:103DD00001237F084FEA3606F21847F10003A3FBE0
:103DE0000076E2FB01760027E3FB01674FF05538D0
:103DF000A6FB08964FF00009E7FB086916EB0906D9
:103E000059F10007861B71EB07074FEA033040EAC0
:103E10001250A0FB0009E9FB0809A9FB01084FF0BB
:103E20003330A8FB000858FB11FA4AF6AA20C2F664
:103E3000AA2060FB1A99B2EB491273EBD9635AFBC3
:103E400011FA4FF0C3606AFB108816EB481657EB67
:103E5000D8677047A2FB04804FF00001E3FB040128
:103E6000A6FB0583E7FB0534181A64EB01017047D4
:103E7000A2FB04804FF00001E3FB0401A6FB0583D5
:103E80006442E7FB0534181844EB01017047A2FBBC
:103E900005804FF00001E3FB0501A6FB04836D42A2
:103EA000E7FB0435181845EB01017047A2FB0580BC
:103EB0004FF00001E3FB0501A6FB0483E7FB04359B
:103EC000181A65EB01017047243F0010404261EB76
:103ED000410140F2F334B1FA81F20C2A0CD21532CE
:103EE00011FA02F3C2F12002D04021FA02F1224479
:103EF000584141EB0251704769B1C2F12B0230FACF
:103F000002F3C2F12002914090401943A4EB020257
:103F100001EB0251704701004FF00000A4F12004B2
:103F2000D9D170470B5C7325A974F50329B5FA0143
:103F30000015FC7FEB2FAA0054D9440CC8D22106EF
:103F40001F60DA7F3663E842CFD3D9133C5EEA09BB
:103F5000F0889D7F2FC46D04D9860A1C1F17FE0DA3
:103F6000D09E3B7FA79B50EC3EF5EB23BCE7E611D0
:103F7000C7EFBD7ED21C9C03B212F12B46F5DC15B7
:103F800049771E7ECA057A3DF493F23314C0CB19EB
:103F90009CAC5F7DA0A0EF7A1D32193C1D22C61D8E
:103FA0002F2F7D7CB50FFB1270EF5044530CC121B5
:103FB0003522787B5C8D6B4745A0F14B18DC6A2578
:103FC00016AD687AC14069576DD9EA53391636295A
:103FD0003C2D2F79DFEA4ED38942B35BD639E02CF2
:103FE0002526E0776950EA31D9071164C0D3C4307F
:103FF00070625876CB5667F3B3A2FD6B1C7E6834B3
:10400000227AC7740EED7A2F3175E073CCE7FA3758
:1040100027111C73C08EC4FC0E79147C0EA7A33B21
:104020008ECD417113B7043B8F7B5483D489D23E2C
:10403000EBD8856F9A365B13D96F0B8CD4EA944218
:10404000A3EF516D5F52CA4A26D33994706E0A4667
:104050004005236B8340C441340B0E9C3DB048495E
:1040600007EFF168BF086DA3FD6179A485F2B14C3B
:104070009D847A663616F8C8D247E5AB1E22A24F59
:104080002F623664ADC9C8D0E1ADFEB32470C3520F
:1040900086AFA461730E73646A35FEBB28F0C55504
:1040A000A3A3025FC6A58CB055B912C40892BA5832
:1040B000A394415C90005354372DB0CB19F46E5B40
:1040C000D88E9359367C8DA16E3CAAD325022E5EE4
:1040D000FC32AF56D0C7A248F619FFDB3253F3606B
:1040E0007EED9253949AAD7AE1AD22E4CADF8E63FD
:1040F000C72B7350FF15EF19BD85FBEBBB18FA6595
:10410000C7615C4DBD960F7E494B4CF4F7816F68DB
:10411000E617024AEB09EF1DFDBD4DFCC4D2B26AA1
:1041200013E4B4460022002950DA404261EB410119
:10413000C9B1B1FA81F30B3B17D4D3F1200C30FA9B
:104140000CFC9840994051EA0C011A44524202F288
:10415000324201EB025141F0004140F2FE739A42BB
:1041600038BF704721E011467EE003F1210310FAC9
:1041700003FCA3F1010301FA03FCC3F1200320FABD
:1041800003F021FA03F140EA0C00A3EB020202F271
:10419000324214D050F1000041EB025141F0004195
:1041A00040F2FE739A4238BF70474FF00001A8BF3B
:1041B000C7F6F0714FF00000704700217047EBD355
:1041C00050F1000020F00100E6E70022B9B1B1FA99
:1041D00081F30B3B16D4D3F1200C30FA0CFC984041
:1041E000994051EA0C011A44524202F2324201EB68
:1041F000025140F2FE739A4238BF704720E01146E8
:1042000000F066B803F1210310FA03FCA3F10103E7
:1042100001FA03FCC3F1200320FA03F021FA03F1B1
:1042200040EA0C00A3EB020202F2324212D050F13B
:10423000000041EB025140F2FE739A4238BF7047D2
:104240004FF00001A8BFC7F6F0714FF000007047B3
:1042500000217047EDD350F1000020F00100E8E7A5
:10426000002880F235804042B0FA80F30B3B11D435
:10427000984001EB0302524202F2124200EB02515B
:1042800041F000414FF0000040F2FE739A4238BF07
:10429000704713E0C3F1000330FA03FCC3F12002BE
:1042A0009040A3EB010202F212420CEB025141F0EA
:1042B000004140F2FE739A4238BF70474FF0004110
:1042C000A8BFCFF6F0714FF0000070470021704793
:1042D00060B3B0FA80F30B3B0FD4984001EB0302BC
:1042E000524202F2124200EB02514FF0000040F243
:1042F000FE739A4238BF704710E05B4230FA03FC0D
:10430000C3F120029040A3EB010202F212420CEB37
:10431000025140F2FE739A4238BF70474FF00001DD
:10432000A8BFC7F6F0714FF000007047002170473A
:104330000022A2F232425FEA215CACF10103A1EB60
:1043400003515B0513F5800F32D212EB535210D498
:104350000B2A36DA9140D2F1200330FA03F31943E5
:104360009040BCF1000FA8BF7047404261EB410193
:10437000704720320EDD01FA02F3D2F12002D14063
:10438000D0401843BCF1000FA8BF7047404261EB1A
:1043900041017047524282F3050231FA02F00021D6
:1043A000BCF1000FA8BF7047404261EB410170476C
:1043B00002D000200021704750EA013118BF4FF0B1
:1043C000000C6FF0004101EBDC716FEAEC7070479C
:1043D00038B50446094807F007FE204602F05CF9AC
:1043E0000546064807F0FCFD2DB1054B2C449C42C8
:1043F00001D8284638BD0348FDF7E6FFB410002079
:10440000000008204CC2001038B505460C460A488A
:1044100007F0EAFD2846214602F004FC054606485E
:1044200007F0DEFD2DB1054B2C449C4201D82846F7
:1044300038BD0348FDF7C8FFB41000200000082075
:104440004CC2001038B50446054D284607F0CCFD97
:10445000204602F029F92846BDE8384007F0C0BDE3
:10446000B41000209A4238BF88547047704700BF8C
:104470002DE9F04F83B09946DDE90DAB0F9B8846DF
:1044800011469A07074616D1DA453AD20C460D4630
:10449000ABEB0A060E4422464B464146202001342F
:1044A000B847B442F7D12946BAF1000F08D12046E7
:1044B00003B0BDE8F08F0C46BAF1000F10D00E46E5
:1044C00055460C9B2E449A440191721B4B46013D6C
:1044D00041461AF8010D3446B847002DF5D101992F
:1044E0000F9B9B07E3D5651AAB45E0D922464B46A7
:1044F000414620200135B8475D4504F10104F5D35C
:10450000D5E7BAF1000FDAD10C46D0E72DE9F04F2C
:104510000F9FDDF824E017F0020F0A9C9DF82C9005
:104520000E9DDDE90C8629D1002D6FD1B44225D234
:10453000202C07F0010B00F0128104F1FF3C4FF03A
:10454000300AF44401E0202C7AD00134A6420CF861
:1045500001AFF8D8BBF1000F10D0AC420ED2202C26
:1045600074D004F1FF3C4FF0300AF44401E0202CF9
:1045700029D00134AC420CF801AFF8D117F0100F7C
:104580003AD017F4806F28D11CBBB8F1100F00F09F
:10459000CA80B8F1020F00F0D48030248EF80040B9
:1045A0000124B9F1000F67D17E0740F1AA802B26C4
:1045B0000EF804600134CDE90B57CDE909E4BDE8FC
:1045C000F04FFFF755BFFC0640F189807C0535D4DC
:1045D0002024A6426AD0AC4268D0B8F1100F00F097
:1045E0008780B8F1020F5AD0202CE4D0264601343F
:1045F0004FF0300C0EF806C0202CD2D1CDE90B576D
:10460000CDE909E4BDE8F04FFFF732BF17F0010B29
:104610003ED0B9F1000F47D117F00C0F44D1B4428E
:104620009BD2202C89D1202D10D8FC0657D57C0593
:1046300055D4202E00F0B980202D10D02024CCE7B6
:10464000BBF1000F00F0A580202DBCD9FC0646D59B
:104650007C0544D4202E00F0A880202D3FD12C468C
:104660001F26B8F1100F7FD0B8F1020FC0D14FF064
:10467000620C0EF806C0B7E72D260EF80460013470
:10468000CDE90B57CDE909E4BDE8F04FFFF7F0BEE7
:10469000B442BFF473AF202C7FF44FAFD6E7202C89
:1046A00089D026460134E2E7013DB8E7661ED8D13D
:1046B000B8F1100F64D0B8F1020F7FF46EAF62262C
:1046C0008EF80060302644468EF80160B9F1000F84
:1046D0003FF46AAFD0E7B8F1100F7FF46CAF20243D
:1046E000CDE90B57CDE909E4BDE8F04FFFF7C0BEB7
:1046F000BE060ED4202CF2D078260EF804600134C9
:1047000072E73E077FF557AF20260EF804600134AC
:1047100051E7202CE3D04FF0580C0EEB040686F83E
:1047200000C0013460E7BE0617D558248EF800405B
:1047300030248EF801400224B9F1000F3FF434AF69
:104740009AE762248EF8004030248EF8014002245B
:10475000B9F1000F3FF428AF8EE77824F2E7BBF100
:10476000000F7FF462AF71E717F0200F0CBF4FF01E
:10477000780C4FF0580CA61E0EF806C0013C35E729
:10478000BC06EAD558248EF8004030248EF801404B
:10479000DDE717F0100F3FF40EAF17F4806F9AD1DA
:1047A000202E7FF418AF1F265BE734461F2658E7FC
:1047B00000B9704701F0F4BA10B1D1E900311847DF
:1047C000704700BF000000002DE9F04F9FB09DED45
:1047D000287BDDE92AA558EC177B83461E460D9100
:1047E000109243463A46384641468DED087B2C9C54
:1047F000FFF760F8002840F0D880384641464FF077
:10480000FF32754BFFF7B6F8002840F0CE803846EF
:1048100041464FF0FF326FF48013FFF76FF8002826
:1048200040F0C380DDE90878002238464146002385
:10483000FFF764F8002840F0C081CDE90A78DDE98F
:104840000A2390461F4614F4806308BF4FF0060AFF
:10485000139304F4006258EA0703119240F0C080F9
:10486000002A00F0A2819FED5A7B00278DED0E7B80
:104870004FF00009BA45CCBFAAEB070A4FF0000A77
:104880004F46C8BF0AF1FF3A44F480644D4594BFD7
:104890004FF00008A5EB090814F00203119304D0AF
:1048A000B9F1000F18BF4FF000083FB1DDE90A0170
:1048B000DDE90E23FEF75AFFCDE90A01DDE9080123
:1048C00000220023FFF71AF830B1DDE90A010246A1
:1048D00001F10043CDE90A239DED0A7BCDE902A851
:1048E000DDF834A024F4006304938DED007B33469F
:1048F00051465846109A00F097F98046B9F1000FDA
:104900004FD014F0200F024600F1010433460CBFD3
:10491000652045205146D84709F1FF3087EAE77CFA
:104920000DF1580900224B46DFF8B080ACEBE77C74
:104930004FEAD77E01E0202A10D0E246A8FB0C7196
:10494000C90801EB8107ACEB47073037BAF1090F13
:104950008C4602F1010203F8017BECD80523059097
:10496000069300200A230D9FCDE90330CDE9012EE7
:104970003346224639465846CDF80090FFF7C6FD2B
:10498000119B80466BB1109BC41AA54209D94246BF
:104990003346394620200134D847A54208F10108A2
:1049A000F5D840461FB0BDE8F08F9DED087B33463B
:1049B0005846109A0D998DED287BCDE92B54CDF8F2
:1049C000A8A01FB0BDE8F04F00F02EB9AFF30080F3
:1049D0000000000000000000FFFFEF7FCDCCCCCC3A
:1049E000C7F30A50A0F2FF30FEF71CFF8AA3D3E9F9
:1049F0000023FEF795FE8AA3D3E90023FEF768FEA5
:104A0000C7F31307CDE90E0147F07F51404600225E
:104A10007B4B41F44011FEF76FFE6BA3D3E90023FB
:104A2000FEF77EFE02460B46DDE90E01FEF750FE64
:104A3000FEF71CFF0746FEF7F5FE65A3D3E900234A
:104A400080468946FEF76CFE00226E4BFEF740FE64
:104A5000FEF70CFF03464946404612935EA3D3E996
:104A60000023FEF75DFE804612988946FEF7DAFEC7
:104A70005BA3D3E90023FEF753FE02460B464046F4
:104A80004946FEF739FE02460B4680468946FEF748
:104A900047FE42464B46CDE90E0140464946FEF7E9
:104AA00017FE0022CDE91401DDE90E01564BFEF799
:104AB0005DFE0022554BFEF70BFE02460B46DDE97C
:104AC0000E01FEF753FE0022514BFEF701FE024697
:104AD0000B46DDE90E01FEF749FE42464B46804695
:104AE000894600204FF08041FEF706FE02460B4645
:104AF00040464946FEF7ECFD02460B46DDE914014F
:104B0000FEF734FE0022434BFEF7E2FD129B00222B
:104B100003F2FF3C4FEA0C53FEF702FE8046894643
:104B2000DDE90A0142464B46CDE90E89FEF7E6FE75
:104B300068BB4346494607F16302C62A119A8CBFF7
:104B40004FF005094FF00409002A3FF49FAE0B43D4
:104B50003FF48EAEDDE90A0123A3D3E90023FEF77B
:104B6000F5FE48B1DDE90A0121A3D3E90023FEF7F0
:104B7000C5FE00287FF47CAEBAF1000F3FF486AE8C
:104B8000139B002B3FF482AE0AF1FF3A7EE600222F
:104B90001E4B40464946FEF7E9FD0A4601460346DC
:104BA000CDE90E12013F1146C5E79FED137B174675
:104BB0004FF004098DED0E7B68E608F100430A977B
:104BC0000B933CE6AFF3008061436F63A787D23F4E
:104BD00071A379094F930A401655B5BBB16B0240DA
:104BE000EF39FAFE422EE63F2D431CEBE2361A3F28
:104BF0000000000080842E41000000000000000042
:104C00000000F83F0000E03F00002C40000024407E
:104C1000000018400000F03FFB799F501344D33F41
:104C2000B3C8608B288AC63F2DE9F04F97B0DDE905
:104C30002089CDE90401DDE9224BCDE90623404678
:104C400042464B464946DDF890A0FEF733FE002869
:104C500040F0C581404649464FF0FF326FF4801363
:104C6000FEF74CFE002840F01D81404649464FF0BB
:104C7000FF32C14BFEF77EFE002840F0E380B8A370
:104C8000D3E9002340464946FEF774FE002840F071
:104C9000CB80B5A3D3E9002340464946FEF72EFE5C
:104CA000002840F0C1804046494600220023FEF71C
:104CB00025FE002840F0E0801AF480650D9000F099
:104CC000E980092C40F296810EAB1A460C933021F4
:104CD0000023A4F109050133202B02F8011BA4EBEA
:104CE000030600F03A81AB42F5D19FED9D7B8DED3F
:104CF000087B49464046FEF7B9FD0446FEF792FDA3
:104D000002460B4640464946FEF7F6FCDDE908231D
:104D1000FEF706FD02460B46CDE90A23FEF7B8FD75
:104D20000746FEF791FD02460B46DDE90A01FEF754
:104D3000E3FC02460B46CDE90A2300228F4BFEF727
:104D400019FE002800F0DB8001373846FEF77CFDB5
:104D5000DDE90823FEF7FAFD08B100270134002E33
:104D600040F0B1802046FEF75DFD02460B4640460E
:104D70004946FEF7C1FC0022804B06460F46FEF76F
:104D8000BDFD40B93046394600227C4BFEF7F2FDAE
:104D9000002800F015810C9B691E7948194410E029
:104DA00080FB0462C3EBA20303EB8302A4EB420487
:104DB00004F1300201351C4601F8012F002B00F0F0
:104DC000AB80202D4FEAE473EAD10AF00303012BF4
:104DD0001CD1BBF1000F19D00D9B002B40F0F980C6
:104DE0001AF00C0F40F0F580AB4540F2D380202D37
:104DF0000BD030220C996B1E0B4401355D4503F836
:104E0000012F00F08D80202DF7D12025DDE906232C
:104E1000DDE904010C9CCDE902BA01950094FFF78D
:104E200027FB17B0BDE8F08FCDE92089DDE9062327
:104E3000DDE90401CDE923BA229417B0BDE8F04FB3
:104E4000FFF7C2BC4F4DCDF88CA00AF0040ABAF1AE
:104E5000000F4D4C18BF2C46DDE90623DDE90401A7
:104E600020940CBF03240424CDF888B0219417B0FB
:104E7000BDE8F04FFFF7FCBA4B4642460020002148
:104E8000FEF73AFC01231AF48065804689460D93AB
:104E90007FF417AF9FED367B0EAB06268DED087BBA
:104EA0000C9326E70424DDE90623DDE90401374DF0
:104EB000CDF88CA0CDF888B02095219417B0BDE82E
:104EC000F04FFFF7D5BA0C9B681EDFF8C4C018443A
:104ED0000DE0ACFB0721C90801EB8102A7EB420200
:104EE0003032092F00F8012F27D90F461D46202DFB
:104EF00005F1010306F1FF36EBD120254BE7002237
:104F0000DDE90A011D4BFEF7F9FC00287FF427AF0D
:104F1000002F5AD1013722E70AF00303012B75D085
:104F2000202D3FF473AF0D9BBBB32D2205F1580329
:104F30006B4403F8202C013568E7202BDDD0AEB39D
:104F40000C9A1E441544302201E0B3422ED00133A6
:104F5000202B05F8012FF8D1CFE71D46C5E600BF8D
:104F60000000000065CDCD410000000065CDCDC141
:104F70000000000080842E41FFFFEF7F0000E03F33
:104F80006766666694C200109CC20010A4C200103E
:104F9000CDCCCCCC202D3FF439AF1AF0040F0DD17D
:104FA0001AF0080F3FF432AF2022BFE72E2103F1A1
:104FB00058026A4402F8201C5D1CECE62B22B5E77F
:104FC000E3077FF5E8AE0134E5E6FA077FF5C7AE03
:104FD000A0E70BF1FF3BAB453FF609AFA0E7032489
:104FE000DDE90623DDE904010A4DCDF88CA0CDF8FA
:104FF00088B061E7084B264603EBC40393ED007BC2
:105000000EAB8DED087B00250C9372E6BBF1000F13
:1050100086D0E1E6A0C2001058D200102DE9F04F72
:105020009A469BB0249C964D0B94964C0B1E18BF31
:10503000834625609AF80000934C0A9308BFA34664
:105040000992002800F0BC824FF000090AE04A46AD
:10505000099B0A9909F10109D8479AF8000000282C
:1050600000F0CE8025280AF1010AF0D10023524633
:1050700012F8010BA0F1200110290AD8DFE801F095
:105080004009093C090909090909093809340909CC
:105090003000A0F13001092940F28C802A2800F06C
:1050A000F58000210C912E2800F099800027A0F1B6
:1050B000680112292DD8DFE811F057012C005101A9
:1050C0002C0045012C002C002C002C002C002C0066
:1050D0002C0027002C002C002C002C002C0027007A
:1050E000924643F00103C2E7924643F00203BEE753
:1050F000924643F00403BAE7924643F01003B6E742
:10510000924643F00803B2E79AF8010043F4807333
:1051100001326728924600F28280242840F2C6803D
:10512000A0F12502422A00F2C180DFE812F05F01FF
:10513000BF00BF00BF00BF00BF00BF00BF00BF0077
:10514000BF00BF00BF00BF00BF00BF00BF00BF0067
:10515000BF00BF00BF00BF00BF00BF00BF00BF0057
:10516000BF00BF00BF00BF00BF00BF00BF002601DF
:1051700045012601BF00BF00BF00BF00BF00BF0048
:10518000BF00BF00BF00BF00BF00BF00BF00BF0027
:10519000BF00BF00D301BF00BF00BF00BF00BF0002
:1051A000BF00BF00BF00BF00D3016701D3012601CC
:1051B00045012601002100E0013201EB810100EBF5
:1051C000410110789246A0F13004092CA1F1300180
:1051D000F2D92E280C9102F101027FF467AF9AF800
:1051E00001001146A0F13006092E43F4806340F21D
:1051F00031812A2800F03E8192460027013256E78D
:105200004C46099B994501D303F1FF394A460020DA
:10521000099B0A99D84720461BB0BDE8F08FA0F142
:105220006902D2B20F2A41D8012649F241019640C3
:105230000E4040F001810A2A3FD0072A36D10B9C4C
:1052400054F8042B002A00F0288143F021010DF1CD
:10525000480E704603E0202E00F029811A4602F025
:105260000F052B46092D94BF303337330F2A00F832
:10527000013B06F101064FEA1213ECD817E100BF1B
:105280001D500010F03C00206D4400100B9C9AF85B
:10529000010054F8045B9246002DBDBF694243F003
:1052A00002030C910C950B940132FCE64A46099BD3
:1052B0000A9909F10109D847CFE60B9951F8048BF7
:1052C00098F800201046002F40F0E18072B16FF096
:1052D000010C0CF1010C4646C44401E0664503D0C4
:1052E00016F8014F002CF9D1A6EB080613F4806CD8
:1052F00002D0BE4228BF3E4613F0020400F0878170
:10530000002A00F02B81BCF1000F00F041810B94CA
:105310000D964A46DDE909540E464F4408E02B46F7
:105320002146D84718F8010F09F1010910B14A4682
:105330004F45F4D131460B9C0D9E002C40F00E8160
:105340000B918AE69AF801006C287FF4DFAE9AF898
:10535000020043F440730AF10302DAE69AF801000E
:1053600043F400730132D4E69AF80100682800F093
:10537000208143F080030132CBE6672800F0E7800C
:10538000472800F00081452800F0FF800B9C049323
:105390000C9B0734CDE9027324F007031C46DDE9BA
:1053A0000931F4E802674A465846CDE900670B9494
:1053B000FFF70AFA814650E646280B9C08BF43F0E7
:1053C000200304930C9B0734CDE9027324F00703F8
:1053D0001C46DDE90931F4E802674A465846CDE942
:1053E00000670B94FFF720FC814636E64A462520ED
:1053F000099B0A9909F10109D8472EE60B9A9C07E7
:1054000002F1040709F1010640F1E6801078099BDA
:105410004A460A99D8470C9B012B40F22C81DDE9C2
:105420000954994432462B46214620200136D8475C
:105430004E45F7D10B9710E66F2800F08B8040F2B5
:105440006581782800F008814FF00A0823F01003E6
:10545000C44647E0002707EB870700EB4700A0F1B1
:10546000300711F8010FA0F13002092AF3D98A465A
:105470004A1C1CE60B9C9AF8020054F8047B0AF1C3
:10548000020A0AF101020B9427EAE7770FE6002AE5
:105490003FF42CAF07F1FF3C1BE723F0100113F49E
:1054A000806241F021013FF4D2AE0DF1480E082395
:1054B0001020059300234A46CDE902300691584654
:1054C000DDE90931CDE900E60497FFF71FF80B94F9
:1054D0008146C2E5582879D0622840F051824FF0C9
:1054E0000208C44613F480606DD123F00C0313F45A
:1054F000007240F0C2800B9904310D9113F4807159
:1055000040F02E825E060B9A40F1AA801278002AA3
:1055100040F0DA8023F01003002800F0D580114617
:105520000DF1480E06930C9BCDF80CC0CDE9047329
:10553000019100234A4602935846DDE90931CDF82E
:1055400000E0FEF7E3FF0D9B81460B9385E543F4F6
:1055500000631BE74FF00808C446C3E70C9B4C46AA
:10556000B3427FF6EDAE0F464B44A3EB0609DDE9EF
:10557000096522463346294620200134D8474C4548
:10558000F7D13946DCE643F4006343F02003FDE63F
:105590000F460B94DDE909544A462B462146D8476D
:1055A00018F8010F09F101090028F5D139460B9CC3
:1055B000C3E69AF8020043F0C0030AF10302A8E52B
:1055C000044681461DE623F00D0390E74FF01008D6
:1055D00043F02003C44685E70C9B012B45D9DDE948
:1055E00009544E4609F1FF38984432462B4621466D
:1055F00020200136D8474645F7D10C9B32469944C6
:105600000B9B1878DDE90931D8470B9725E50C9BF2
:10561000B34240F2EE81CDE90D48DDE909548846F8
:105620004B449E1BCDF82CC04A462B4621462020D9
:1056300009F10109D847B145F6D14146DDF8388076
:105640000C9BDDF82CC00D9C98F800205E1C1046C9
:10565000002A7FF458AE73E64FF01008C44641E7C5
:105660001D064CBF1288126851E713464A46187847
:10567000DDE90931D847B146DCE60B9C073424F05C
:1056800007042246656852F8084B0B9254EA05025B
:1056900040F02C8123F01003002800F02781002621
:1056A0000DF1480E06930C9B4A46CDE90473002386
:1056B000CDE900E6CDF80CC002935846DDE909318A
:1056C000FEF724FF8146C8E413F0200F14BF4120E9
:1056D00061200DF1480E7646A0F10A0803E020296A
:1056E0003FF420AF2246B2FBFCF40CFB1425E8B2D9
:1056F000092D00F130058ABF4044E8B2C0B26245CE
:1057000006F8010B01F10101E9D20BE723F01002C9
:1057100069280D9240F06F8113F4806204D04FF439
:10572000806223F011030D930D9B13F4007640D19A
:105730000B9B03F104080D9B13F4807040F09880DC
:10574000590640F1C6800B9B19780C46CB0F0029F7
:1057500000F0B98022460DF1480E74461646DFF877
:10576000A0C201E020280FD03546ACFB0621C908B5
:1057700001EB8102A6EB42023032092D0E4600F108
:10578000010004F8012BEDD80D9ACDE90103069232
:105790000C9ACDE904720A234A4603935846DDE980
:1057A0000931CDF800E0FEF7B1FECDF82C8081463E
:1057B00053E40B9C073424F0070421460846636831
:1057C00050F8081BDC0F0B9051EA030000F0C38077
:1057D0000A46191E48DB13460DF1480EF446002612
:1057E000CDE90E94DFF8188201E0202E2DD05A1852
:1057F00042F10002A8FB025929F0030505EB9905C7
:10580000521B1C469B1A61F1000508464FF0CC3133
:1058100001FB03F108FB0511A3FB08531944052301
:1058200005F00109A9FB03399B180A2C03F1300389
:105830004FEA550570F100000CF8013B06F1010636
:1058400045EAC1734FEA5101CFD2DDE90E940D9BB9
:105850004A4606930C9BCDE90164CDE904730A2303
:10586000CDF800E0039328E7524261EB4101B2E733
:105870000B9B1968CB0F002900F0AB8081EAE17225
:10588000A2EBE1720DF1480E7046DFF874C101E041
:10589000202E10D01546ACFB0241C90801EB810453
:1058A000A2EB440404F13002092D00F8012B06F1AB
:1058B00001060A46ECD80D9ACDE9016306920C9ACE
:1058C000CDE9047267E7002A3FF445AF0DF1480EB9
:1058D0005AE713F0800F0B9B00F08180B3F90010A2
:1058E00081EAE174A4EBE174A4B22FE713F0200F76
:1058F00014BF412261220DF1480E0A3ACDE90D97FD
:10590000CDF844B000267746F3469146CDE90F3CEA
:1059100003E0202E17D004460D46294642460023B8
:10592000204606F059FBD2B2092A02F1300388BFA3
:1059300002EB09034445DBB275F1000507F8013BB2
:1059400006F10106E5D2DE46DDE90D97DDE90F3C03
:10595000DDF844B0A6E6002A47D1134611463BE7DE
:105960000B990968A1B923F0100388B10DF1480E15
:1059700006930C9BCDF80CC0CDE904730192D8E5D9
:1059800013F480627FF4CBAE23F010030D93CBE6CB
:1059900013F0200F14BF412061200DF1480E764610
:1059A000A0F10A0802E0202AE2D02146B1FBFCF473
:1059B0000CFB1415E8B2092D00F130058ABF4044F4
:1059C000E8B2C0B2614506F8010B02F10102EAD269
:1059D000CEE7002A3FF456AF0DF1480E6BE7196889
:1059E00081EAE174A4EBE174B0E600260DF1480E03
:1059F0002DE701362BE64FF00A081346C44671E541
:105A0000CDCCCCCC0EB410B585B007AC54F8043B6B
:105A100001464FF0FF32009404480394FFF7FEFA6A
:105A200005B0BDE8104003B0704700BF65440010EA
:105A300070B594461E4605460C4684B04FF0FF32C2
:105A4000634602A900960348CDE90254FFF7E6FA3F
:105A500004B070BDB94700100FB410B50E4B84B040
:105A600006A91C6851F8043B03915CB100914FF00A
:105A7000FF3202A90948A047012004B0BDE8104048
:105A800004B07047184600F0CDF9204604B0BDE8D8
:105A9000104004B0704700BFF03C0020B147001038
:105AA00010B5094B84B01C684CB1034600914FF00F
:105AB000FF3203A90548A047012004B010BD00F043
:105AC000B1F9204604B010BDF03C0020B1470010F1
:105AD00000BEFDE7074A0346106838B10649034493
:105AE0008B428CBF4FF0FF3013607047034908466C
:105AF0001160F3E7E430002000000820989B0220AA
:105B000008B5FFF7E5FF00BF9C46144600B50B46FD
:105B10000246614683B044B1054D064801940095A4
:105B2000FFF79AFF0120FFF7D3FF034D2C46F4E760
:105B3000ACC20010BCC2001018C1001038B5064C31
:105B4000064DFDF7A9FCAC4204D254F8043B98473B
:105B5000AC42FAD338BD00BF38C0001040C00010BE
:105B60000368084611461847437D2DE9F0478146F2
:105B70000F461646002B43D0002A3BDD037D002054
:105B80004D1E014615F8012FDFF884800A2A01F125
:105B900001040ED0A6421CD02B782146A3F10D03A0
:105BA000B3FA83F315F8012F5B090A2A01F1010406
:105BB000F0D1002BEED18142A1EB000138441BDC77
:105BC00002214046D9F800309847A64208D0204626
:105BD000E2E7864204DD311AD9F8003038449847AC
:105BE000374417F8013CA3F10D03B3FA83F35B09C3
:105BF00089F81430BDE8F087D9F800309847DFE71E
:105C00003846D9F800301146BDE8F047184700BFC4
:105C1000A8D200100B682DE9F041802B0D460646F6
:105C200005D05A1C2B442A601E71BDE8F0810F4B31
:105C30001C68A4B10E4F01F1040801E0246974B19D
:105C40002368002BFAD03B680BB1A342F6D1204663
:105C500041462A68FFF788FF2469002CF0D1002311
:105C600001222B442A601E71BDE8F081D42400205B
:105C7000DC2C00202DE9F04782B00D469246994673
:105C80000746FDF70FFA4FF0FF366FF000442F4A3A
:105C9000821841F10003964274EB03013CBF324687
:105CA00023462B4806F0A4F96B1C804603D13846E6
:105CB00001F046FC0546274B274E1C68274BB9F1DF
:105CC000000F18BF1E46B4B1BAF1000F1AD1DFF8A9
:105CD000909001E0246974B12368002BFAD0D9F8C0
:105CE00000300BB19C42F5D120462A463946B047D8
:105CF0002469002CF0D1B8F1000F1FD1284602B062
:105D0000BDE8F0874FF00A0ADFF8549002E02469FA
:105D1000002CF0D02368002BF9D0D9F800300BB15B
:105D2000A342F4D12A4639462046B04701222046F4
:105D30000DF107018DF807A0B047E8E7044806F029
:105D40004FF9284602B0BDE8F08700BF40420F007F
:105D5000BC100020D4240020615B0010695B00109F
:105D6000DC2C00200A4A13684BB1834202D109E0BF
:105D7000984207D003F110021B69002BF8D101B142
:105D8000106070470029FCD10369136001617047FE
:105D9000D424002008B500F0A5F9012008BD00BFFB
:105DA000F0B583B006468DF80700FDF77BF94FF09C
:105DB000FF356FF00044174A821841F10003954205
:105DC00074EB03013CBF23462A46134806F010F942
:105DD000124B07461C689CB1114D01E024697CB14F
:105DE0002368002BFAD02B680BB19C42F6D12046D9
:105DF00001220DF10701FFF7B7FE2469002CEFD156
:105E000017B9304603B0F0BD034806F0E9F8304654
:105E100003B0F0BD40420F00BC100020D42400208D
:105E2000DC2C002038B5044601F08AFB012305462E
:105E30001A4620462946FFF71DFF084B1C682CB167
:105E400063682BB198472469002CF9D1284638BDE6
:105E50002469002CF4D1284638BD00BFD42400208A
:105E60002DE9F041A2B004460D46FDF71BF94FF0B5
:105E7000FF376FF00046274A821841F1000397422E
:105E800076EB03013CBF3A463346234806F0B0F8B0
:105E900000262B4607462246204801A90196FFF717
:105EA000C7FD019B06467BB91D4B1C682CB163687E
:105EB00043B198472469002CF9D10FBB304622B07A
:105EC000BDE8F0812469F1E7DFF85480D8F800508C
:105ED000EDB1144C01E02D6975B12B68002BFAD09F
:105EE00023680BB1AB42F6D12846019A02A9FFF70D
:105EF0003BFE2D69002DF0D1D8F800400195D5E783
:105F0000054806F06DF8304622B0BDE8F0810195F5
:105F1000D3E700BF40420F00BC100020155C00100A
:105F2000D4240020DC2C00200FB400B583B004A9D9
:105F300051F8040B0191FFF793FF03B05DF804EBF8
:105F400004B07047B1F1000C1DDD0F4A0F4B126811
:105F500030B5D31AB3FA83F30D240D4D5B09411EFE
:105F600035F913E08C4411F8010F864506D093698A
:105F70009B06FCD461451060F5D130BD93699D0648
:105F8000FCD41460F3E77047843F00200080074092
:105F9000803F0020224BB1F1000C10B41C682EDDB4
:105FA000034600201F4A591E12689369DB0617D466
:105FB00001309369DB06FCD41368844501F8013F86
:105FC000F3D14CB150211346916353F8342F02F0B2
:105FD000380203F580531A6060465DF8044B704741
:105FE0004CB150211346916353F8342F02F038021C
:105FF00003F580531A6078B15DF8044B70475CB1CB
:10600000084B50211A681346916353F8342F02F05D
:10601000380203F580531A606FF00200ECE700BF0E
:106020009C200020843F0020054B1B6833B10021D9
:10603000044A05481268006891631847704700BF1A
:106040009C200020843F0020A0200020024B1A68E2
:1060500093691B07FCD47047843F0020F8B51C4FA0
:106060001C4D3A681C4EAA4214BF21252225044625
:10607000D6F800C018B1BCF1000F10D0F8BDBCF1CB
:10608000000FFBD0014690632846FCF793FA2846A0
:106090001249FCF7E5FA124B34601C60F8BD0B4660
:1060A0000F4A0E49306028461360FCF7A9FA012117
:1060B0002846FCF77FFA3A6850211346916353F85B
:1060C000342F02F0380203F580531A60F8BD00BF88
:1060D000843F0020008007409C20002029600010A1
:1060E000A020002010B50E490E4C0F480F4A104B4F
:1060F000007821600020022112781B78FCF7FEF85E
:1061000002210120FCF7FAF84FF4E1312068FDF795
:1061100017F8BDE8104001210648FFF723BE00BF75
:1061200000000740843F00202C410110284101104D
:1061300024410110D40900200B4B10B5DB6ADB07AA
:1061400009D40124094B0021DC620948FCF7B4FFA3
:10615000084BDC6210BD01210022064B4FF0FF30DE
:10616000D9621146FDF754F900001040002010409C
:10617000400D0300003010402DE9F04789460546E8
:10618000FCF73AF9012399F8042099F905C005F1C3
:106190002F4EDFF8D8800EF5600E93404FEA1E5E5A
:1061A000BCF1000F58F82E7003F1FF3346DBC2F14B
:1061B00020018C45644631DC03FA0CF139422DD1C3
:1061C0006646D5F868A199F80710BAF1000F2CD0EF
:1061D000C9072CD4BCF1000F01DB664527D1B340C1
:1061E0001F423CD1D9F8001082B1B44601EB4209FC
:1061F00031F8022B0CF1120AB2F5005F38BF921988
:1062000049450CF1010C45F82A20F1D13B4348F8EF
:106210002E30FCF703F92046BDE8F0874FF0FF343D
:10622000FCF7FCF82046BDE8F0874907D2D56FF0AF
:106230000A04FCF7F3F82046BDE8F087D2F1200409
:106240000DD403FA04F13942264603D1B9E73942A5
:106250002646B6D0013C661C03FA04F1F7D16FF074
:106260000804FCF7DBF82046BDE8F0879018002012
:106270002DE9F041D0F868419DF81860121B1F2AE3
:1062800038D84EF29F044EF280054FF4003801EBEF
:10629000410C002E18BF254600EBCC0404F54354F6
:1062A00000EBCC0C052BDCF8DC704FEA410EDCF87F
:1062B000CC60C4F80C800CD95401053B44F0A054C8
:1062C0000532052BCCF8DC4002F01F02CCF8D85088
:1062D000F2D8714400EBC1010020520142EA83630D
:1062E000C1F8DC30C1F8D850C1F8DC70C1F8CC601E
:1062F000BDE8F0816FF00400FAE700BFF0B50125BA
:1063000004688D4024EA05040460B3B3D3E9015660
:106310001F68DC6801EB410300EBC303C3F8C870DE
:106320004FEA410CC3F8D060C3F8CC50C3F8DC404E
:106330000CEB01034FF0013500EBC30C4FF00046AE
:1063400000EBC30E01230EF5865E0C1D01F108075C
:106350008D40CEF8106003FA04F4CEF8106002F01D
:106360001F028560BB4000F5005004600EF1100E66
:1063700003600020CCF8D820F0BD4FF480374FF4F4
:1063800040264FF4F83501EB410400EBC404C4F897
:10639000C8704FEA410CC4F8D060C4F8CC50C4F8BF
:1063A000DC30C5E710B5054C82B001460F23002252
:1063B00000940348FCF768F802B010BD30C3001029
:1063C0008A9B0220012307480749084A03600B60A3
:1063D0009368D907FCD50123054A13601368DB05D0
:1063E000FCD570470020024000300240000002400F
:1063F00000000A402DE9F84F374B0746984214BF7A
:106400004FF400234FF480230E46344D344C354A6C
:106410002B602360946833EA0404FBD10620FCF768
:1064200079FF3946022351F8042F4FEA462E4FEAEE
:10643000D65B704502EA030801F5405974EB0B0284
:10644000C9F8003011D34FEA965CB20201E052461F
:10645000AC460233B3F5807F07D01EEB020A4BEB4C
:106460000C05904274EB0C0CF1D24FF48072C3EB2C
:1064700003249446013A2DD0B0FBF4F5AE42A4EBD0
:106480000304F6D20CFB03FC120202243B613B46E0
:1064900003253E6801F500517240B0FBFCF002F4A8
:1064A0007F4207F5805CCCF80020C1F800807E6850
:1064B000C9F8004053F8242B264082F0070202F06E
:1064C000CF0203F50053CCF800200E601D600C6075
:1064D000BDE8F88F9C46D8E7000008400020024045
:1064E000003002400000024003BD00BF10B504466A
:1064F000FCF7E2FF2346BDE8104018474FF08071DB
:10650000124B134A10B559605368D801FCD51920B5
:10651000FCF766F8002104461920FCF74BF84FF011
:1065200080714FF050420B4B5960136DD90703D463
:1065300020BF136DDB07FBD54FF050432146BDE86C
:10654000104019209B6DFCF735B800BF00A001403A
:106550000080014000B00140F0B5054687B0192029
:1065600017460E46FCF73CF8002104461920FCF7BC
:1065700021F80021CDE904650397002600270122B8
:106580004FF050438C46CDE900670292B9B11A6DC5
:106590009507FCD5596540BF1A6DD00703D420BFBD
:1065A0001A6DD207FBD59A6D8A420DD04FF0000CC0
:1065B00006AA02EB8C0252F8181CE7E79A6D1A6DD6
:1065C000D607FBD440BFE2E70CF1010CBCF1060F8B
:1065D000EED12146192007B0BDE8F040FBF7EABF35
:1065E0000C4B0D4A93420ED39C4603F2F4710B4AB6
:1065F0009268CCF8F4070A48CCF8F837CCF8FC07D6
:106600000848FFF7A9BF4FF0FF3340F2F3719C46F3
:10661000EDE700BF000808200000082000ED00E0C2
:10662000ED640010E964001038B5A1FB021434BB1E
:1066300000F042F8054630B350F8042C22F0030273
:10664000043A242A0CD8132A0FD91B2AC0E9004483
:1066500012D9242AC0E9024418D000F1100205E042
:10666000214600F04DFD284638BD0246002328464D
:10667000C2E90033936038BD00F10802F6E700F08C
:10668000F3FD0C2303600025284638BD00F11802F5
:10669000C0E90444EAE700BF024B0146186800F075
:1066A0000BB800BF000E0020024B0146186800F036
:1066B000D1BF00BF000E002001F10B03162B2DE906
:1066C000F04F074683B023D8102900F2AF8000F0C6
:1066D0009DFA102518230220BC4E33445C68A3F1B8
:1066E0000802944200F080816368384623F0030377
:1066F000D4E902122344CA6091605A68083442F017
:1067000001025A6000F088FA204603B0BDE8F08F1D
:10671000002B23F00705C0F28980A94200F2868091
:1067200000F074FAB5F5FC7FC0F0B4816B0A00F09C
:106730008180042B00F27E81AB0903F1390003F163
:10674000380EC300A14E3344A3F1080C5C68A44585
:1067500007D10DE0002AE16880F232818C450C46B9
:1067600006D0636823F003035A1B0F2AF2DD70463C
:10677000DFF870823469444500F0E780636823F0F5
:10678000030CACEB05030F2B00F39481002BC6E93F
:10679000048880F28381BCF5007FD6F804E080F0A5
:1067A00029814FEADC0301224FEA5C1C013302FA23
:1067B0000CF256F833104EEA020E06EBC302083A0A
:1067C000C6F804E0C4E9021246F83340CC608310F6
:1067D0004FF0010C0CFA03FCF44531D81CEA0E0F03
:1067E00007D120F003004FEA4C0C04301CEA0E0FD6
:1067F000F9D006EBC00A8146D646DEF80C300BE035
:106800005A681C46DB6822F00302511B0F2900F373
:106810001D81002980F231819E45F1D109F10109E4
:106820000EF1080E19F0030FE7D167E10C233B606E
:10683000002469E74FF4007340204FF03F0E81E7DA
:10684000B468636823F00309A9EB05030F2B02DD8D
:10685000A94580F0A4805E4B08201B6803F1100856
:1068600004EB0903009300F009FD5A4AA84483464B
:106870001368013305D008F1FF384342804403EA2E
:1068800008084146384600F0DDFCB0F1FF3F824683
:10689000504A79D0009B83425AD9B44274D14E4BAE
:1068A0000BF1FF3C186800EB080EC3F800E011681C
:1068B000013100F07381009AAAEB020272441A605F
:1068C0001AF00702CDE9002300F04281C2F108026C
:1068D000384692445A44D04408EA0C01521A02EA5B
:1068E0000C0B594600F0AEFC421C019B00F06E817F
:1068F000A0EB0A0000EB0B08196848F00102B44253
:10690000C6F808A05944CAF80420196032D0B9F179
:106910000F0F40F20C816068A9F10C024FF0050CDA
:1069200022F0070200F0010010430F2A606004EB20
:106930000200C0E901CC1DD904F1080138460093DA
:1069400000F088FE009B196814E0D6F804E03EE7EA
:10695000214B0BF1FF3C196841448E461960A6D1CA
:10696000009810EA0C0FA2D109EB0803B26843F0BB
:1069700001035360194B1A688A4238BF1960184BDB
:106980001A688A4238BF1960B468626822F003024C
:10699000531B0F2B40F3CE80954200F2CB8062193F
:1069A00045F0010543F00103083444F8045C38461F
:1069B000B260536000F030F9204603B0BDE8F08FBC
:1069C000A26823443846D1608A6096E6F809002020
:1069D00034170020EC090020041700202C17002099
:1069E00030170020000A0020DC68A3427FF47CAE50
:1069F0000230BDE6BCF5206F4FEA5C226CD3142A4E
:106A000000F2B98002F15C035B32DB00F118F3584D
:106A10000839994203D191E09B68994204D05A68A1
:106A200022F003026245F7D8D968C4E902318C60CC
:106A3000DC60CCE6142B56D9542B00F2A5802B0B2E
:106A400003F16F0003F16E0EC3007BE6D4F808C0BB
:106A50003846671945F001056560CCF80C30C3F87D
:106A600008C041F00103C6E90477C7E902887B60EA
:106A7000A150083400F0D0F846E622443846516868
:106A800041F00101516054F8082FD3609A6000F082
:106A9000C3F839E6E80805F108031DE6A4443846C2
:106AA0000834DCF8043043F00103CCF8043000F083
:106AB000B3F829E6621943F0010145F001053846B3
:106AC0006560C6E90422C2E90288516044F80C30CE
:106AD000083400F0A1F817E64FEA9C1202F13903DE
:106AE0003832DB0092E703F15C0003F15B0EC30078
:106AF00028E65AF80839534540F0858010F0030F16
:106B000000F1FF30F5D1736823EA0C0373604FEA9C
:106B10004C0C0CF1FF329A4204D391E64FEA4C0C34
:106B200009F104091CEA030FF8D0484661E6012385
:106B3000CAF80430384600F06FF879E692104FF04A
:106B4000010C0CFA02F24EEA020EC6F804E06CE701
:106B50000AEB0802384602EA0C02ABEB020B0BEA26
:106B60000C0B594600F06EFB431C019B7FF4C0AE3A
:106B7000DDF800B0C0E6542A13D84FEA1C3202F107
:106B80006F036E32DB0041E7B3F5AA7F13D8EB0B3E
:106B900003F1780003F1770EC300D3E5C2F800A03B
:106BA0008EE6B2F5AA7F19D84FEADC3202F17803FB
:106BB0007732DB002AE740F25452934219D8AB0CEB
:106BC00003F17D0003F17C0EC300BBE5009A4FF09A
:106BD000000B083A9044A8EB0A088DE640F25453A3
:106BE0009A420CD84FEA9C4202F17D037C32DB00D2
:106BF0000CE74FF47E737F204FF07E0EA2E54FF43A
:106C00007E737E2202E7736881E700BF014800F0CF
:106C100031BB00BF00170020014800F02DBB00BFB2
:106C200000170020024B0A460146186800F002B81F
:106C3000000E00202DE9F04F164683B0002900F029
:106C40009E800C4606F10B058046FFF7DFFF54F8E7
:106C5000040C162DA4F1080920F0030762D81022B5
:106C600000231546B542C0F0A280002B40F09F8063
:106C7000974261DADFF828B309EB0701DBF8083047
:106C8000D1F804C08B4200F097802CF001030B4434
:106C90005B68DB0768D42CF0030C07EB0C03934212
:106CA00045DAC30712D454F8083CA9EB030ADAF812
:106CB000043023F0030084440CEB070B5A4540F3E7
:106CC000FE8007EB000B5A4540F3D4803146404626
:106CD000FFF7F2FC0646002800F0298154F8043C36
:106CE000A0F1080223F001034B44934200F0B1806D
:106CF0003A1F242A00F2DF80132A00F2B0800346F4
:106D00002246116819605168596092689A6021465C
:106D1000404600F09FFC4046FFF77EFF304603B040
:106D2000BDE8F08F25F007052A46EB0F9AE71F46CE
:106D3000D1E90223D3609A60781BD9F8043009EBBB
:106D400007020F2803F001031FD83B43C9F80430A2
:106D5000536843F00103536026464046FFF75CFF4B
:106D6000304603B0BDE8F08FC307AFD454F8083CF9
:106D7000A9EB030ADAF8043023F00300A1E7114677
:106D800003B0BDE8F04FFFF797BC2B4309EB0501BB
:106D900040F00100C9F80430083141F8040C4046C5
:106DA000536843F00103536000F054FCD4E70C2314
:106DB000C8F800300026D3E72CF0030C05F11001D1
:106DC0000CEB07038B4280F29280C0073FF57EAF49
:106DD00054F8083CA9EB030ADAF8043023F0030066
:106DE00084440CEB070399423FF76BAF3A1F5646BA
:106DF000DAF80C1056F8080F242AC160886000F2F7
:106E0000B080132A40F2AB8021681B2ACAF8081010
:106E10006168CAF80C1000F2AB8008340AF1100265
:106E20002168116061685160A16891605B1B0AEB89
:106E30000502404643F00103CBF808205360DAF81E
:106E4000043003F001032B43CAF80430FFF7E4FEDB
:106E500086E750F8043C23F003031F446CE72368E3
:106E60001B2A03606368436036D804F1080200F10E
:106E7000080346E73A1F5646DAF80C30242A56F83B
:106E8000081FCB60996022D8132A1ED923681B2AB9
:106E9000CAF808306368CAF80C303CD808340AF1E4
:106EA000100322681A6062685A60A2689A603446C9
:106EB0005F46D14640E7214600F0A2F827E7D1E936
:106EC00002133A1FCB609960D5E73346E9E72146C4
:106ED000304600F095F8EAE7A368242A8360E36867
:106EE000C36028D004F1100200F1100309E75B1B16
:106EF00009EB05024046264643F00103CBF8082083
:106F0000536054F8043C03F001032B4344F8043C61
:106F1000FFF782FE24E7A368242ACAF81030E3684A
:106F2000CAF8143010D010340AF11803B9E74046FB
:106F3000FFF772FE3EE7236904F1180203616369FB
:106F4000436100F11803DCE623691834CAF81830ED
:106F500054F8043CCAF81C300AF12003A1E7324679
:106F60005EE721463046019300F04AF8019B5DE759
:106F7000A168242ACAF81010E168CAF8141003D0D6
:106F800010340AF118024BE722691834CAF81820A5
:106F900054F8042CCAF81C200AF1200240E700BF74
:106FA000F80900200EB470B59DB000254FF40172B1
:106FB00021AC1B95ADF8142054F8046B0290069098
:106FC00000F0BEFA0B4903464FF6FF7032460A91B5
:106FD0000949ADF81600039307932346086802A9F0
:106FE0000E951395019400F073FD1DB0BDE870403F
:106FF00003B07047FD6F0010000E002000207047A6
:1070000088420ED98B1883420BD900EB020C002A60
:107010006ED0624613F801CD994202F801CDF9D144
:1070200070470F2A0FD8034602F1FF3C002A5FD0B9
:107030000CF1010C013B8C4411F8012B614503F864
:10704000012FF9D1704740EA01039B0751D1A2F10A
:10705000100301F1200C70B523F00F0501F1100EA3
:1070600000F110041B09AC445EF8105C0EF1100E28
:10707000103444F8205C5EF81C5C44F81C5C5EF83C
:10708000185C44F8185C5EF8145CE64544F8145C3F
:10709000EAD1013312F00C0F02F00F0C01EB0311D7
:1070A00000EB031329D0ACF1040C1C1F8E462CF00E
:1070B00003064FEA9C0C1E445EF8045B44F8045F30
:1070C000B442F9D10CF1010402F0030203EB840392
:1070D00001EB840102F1FF3C4AB10CF1010C013BD0
:1070E0008C4411F8012B614503F8012FF9D170BDD3
:1070F000704702F1FF3C03469AE76246EAE700BFA9
:1071000070B5860747D0541E002A3ED0CAB2034647
:1071100001E0013C39D303F8012B9D07F9D1032C81
:107120002CD9CDB20F2C05EB052505EB054535D93E
:10713000A4F1100C03F1100E1A462CF00F064FEAC2
:107140001C1CB644C2E90055C2E902551032724512
:10715000F8D10CF1010214F00C0F04F00F0C03EB4A
:10716000021213D0ACF1040323F0030304331344DD
:1071700042F8045B9342FBD10CF003042CB1C9B27A
:107180001C4403F8011BA342FBD170BD64461346A7
:10719000002CF4D1F9E703461446C0E71A46A4468A
:1071A000E0E700BF38B511F0FF040CD0034600251E
:1071B00001E0431C05462146184602F06DF90028FF
:1071C000F7D1284638BD2146BDE8384002F064B901
:1071D000024A01231268503200F002B8000E00206B
:1071E00018B3F0B407468C4617F8015B01E0A542DE
:1071F00014D01CF8014B002CF9D1DDB13E460C46F1
:1072000016F8015B00E063B114F8013B9D42FAD12E
:107210004DB100233B701660F0BC704773B1384627
:10722000E0E73746EAE72E46F5E710680028D8D1B0
:107230000020704700201560F0BC70471760037095
:10724000EAE700BF38B50022064D044608462A602A
:10725000FEF740FC431C00D038BD2B68002BFBD050
:10726000236038BDD8240020014B1868704700BF48
:10727000000E0020704700BF704700BF082802D1F1
:107280004FF48050704708B5FFF7EEFF1622034613
:107290004FF0FF301A6008BD80EA010C1CF0030FAC
:1072A00037D110F0030C20F0030021F0030150F857
:1072B000042B08BF51F8043B0ED08CF0030C6FF088
:1072C0007F434FEACC0C23FA0CFC51F8043B42EA12
:1072D0000C0243EA0C0300BFA2F1013C9A4201BF39
:1072E0002CEA020C1CF0803F50F8042B51F8043BB0
:1072F000F2D04FEA02604FEA1222012828BFB0EB19
:10730000036F08BF1B0AF4D003F0FF03000EC01A7E
:10731000704710F0030F0AD010F8012B11F8013B51
:10732000012A28BF9A42F4D0A2EB030070474DF81F
:10733000045D50F8042B01F0030521F0030151F81E
:10734000043B022D26D04DD822F07F45B5EB132FFC
:10735000A2F1013C2CEA020C0DD11CF0803C08BFCC
:1073600051F8043B0AD185EA0205B5EB036F0CD155
:1073700050F8042BE8E74FEA13235BE03CF07F4C26
:1073800054D10B784FEA126554E04FEA126503F0CE
:10739000FF034FE04FEA0245A2F1013C4FEA1545D9
:1073A0002CEA020CB5EB134F18D11CF0803C08BF3F
:1073B00051F8043B07D185EA0205B5EB034F09D12B
:1073C00050F8042BE6E75FEA0C4C2FD10B884FEA0C
:1073D00012452FE04FEA03434FEA12454FEA1343A9
:1073E00028E000BF02F0FF05B5EB136FA2F1013CEE
:1073F0002CEA020C0DD11CF0803C08BF51F8043B74
:107400000AD185EA0205B5EB032F0AD150F8042B07
:10741000E8E74FEA13630DE012F0FF0F06D051F8D2
:10742000043B4FEA122523F07F4303E04FF00000B6
:1074300020BC704705F0FF0203F0FF00012828BFC1
:10744000904204BF2D0A1B0AF4D0A2EB000020BC1E
:10745000704700BF844641EA000313F0030349D19B
:10746000403A23D30B6803604B6843608B688360AA
:10747000CB68C3600B6903614B6943618B698361AE
:10748000CB69C3610B6A03624B6A43628B6A836296
:10749000CB6AC3620B6B03634B6B43638B6B83637E
:1074A000CB6BC36340304031403ADBD230320BD338
:1074B0000B6803604B6843608B688360CB68C36074
:1074C00010301031103AF3D20C3205D351F8043B8E
:1074D00040F8043B043AF9D2043208D0D2071CBF6A
:1074E00011F8013B00F8013B01D30B880380604693
:1074F000704700BF082A13D38B07B1D010F00303E5
:10750000AED0C3F10403D21ADB071CBF11F8013B54
:1075100000F8013BA4D331F8023B20F8023B9FE77F
:10752000043AD9D3013A11F8013B00F8013BF9D2F2
:107530000B7803704B7843708B788370604670478C
:1075400020F0030110F00300C0F1000051F8043BEB
:1075500000F1040C4FEACC0C6FF000021CBF22FAC1
:107560000CF213434FF0010C4CEA0C2C4CEA0C4C7F
:10757000A3EB0C0222EA030212EACC1204BF51F878
:10758000043B0430F4D0C2F1000102EA0102B2FA75
:1075900082F2C2F11F0200EBD20070472DE9F843DE
:1075A0000646DFF8AC8008208946FFF767FE0546EF
:1075B0003046FFF72BFBD8F808305F6827F0030749
:1075C000A7F11104A4EB09042C44B4FBF5F4013C2D
:1075D00005FB04F4A54208DC00213046FFF732FE2B
:1075E000D8F808303B44984205D03046FFF714FBEA
:1075F0000020BDE8F88361423046FFF723FE0130EA
:107600000FD03F1B104AD8F80830304647F001072A
:107610005F6013681B1B1360FFF7FEFA0120BDE8D3
:10762000F88300213046FFF70DFED8F80820831AB2
:107630000F2BDADD43F0010303495360034B1B6852
:10764000C01A0860D1E700BF04170020EC09002031
:10765000F809002000297CD02DE9F0410C46804635
:10766000FFF7D4FA764F54F8043CA4F10805BE683D
:1076700023F0010168184268864222F0030200F0FC
:107680008380DE0700EB020C426033D454F8084CD0
:10769000DCF8043007F1080C2D1B214403F0010332
:1076A000AC68644564D0D5F80CE0C4F80CE0CEF8C2
:1076B0000840002B00F0818041F001036B60016005
:1076C000B1F5007F22D2CB080122490901338A405B
:1076D00079680A4357F833107A6007EBC302083A17
:1076E000C5E9021247F83350CD604046BDE8F0418D
:1076F000FFF792BADCF80430DB072BD541F0010329
:10770000B1F5007F44F8043C0160DCD3B1F5206F93
:107710004FEA512353D28B0903F1390003F13802A8
:10772000C300F818FB580838984203D161E09B6801
:10773000984204D05A6822F003028A42F7D8D868E7
:10774000C5E9023085604046DD60BDE8F041FFF7E5
:1077500063BA7047114407F1080C836863453FD052
:10776000C268DA60936041F001036B606950A7E77B
:10777000002B5FD10A44D0E90213CB60996042F03C
:1077800001036B60AA50B0E7DB070A4407D454F842
:10779000083CED1A1A44D5E90213CB60996042F017
:1077A00001036B60274BBD601B6893429DD8264B3D
:1077B00040461968FFF7F2FE97E71144CDE7142B16
:1077C00008D9542B1DD80B0B03F16F0003F16E0287
:1077D000C300A6E703F15C0003F15B02C300A0E76E
:1077E00041F00103C7E90455C5E902CC6B6069505B
:1077F0007BE70121921001FA02F279680A437A606C
:107800009EE7B3F5AA7F06D8CB0B03F1780003F10E
:107810007702C30085E740F25452934206D88B0C9E
:1078200003F17D0003F17C02C3007AE74FF47E731D
:107830007E2276E741F001036B60016055E700BFEF
:10784000F8090020F0090020341700202DE9F04746
:1078500080460C464548264614F801EB10F80EC049
:107860001CF0080CF7D1BEF12D0F5BD0BEF12B0F31
:107870003AD0654633F010003ED04FF0FF379A46BD
:10788000B7FBF3F703FB07F96FEA09090026304657
:107890000EE0AEF1370C63451DDD002E04DBB8426F
:1078A00002D833D1CC4531DD4FF0FF3614F801EB6F
:1078B000AEF1300CBCF1090FEDD9AEF1410CBCF1C9
:1078C000190FE6D9AEF1610CBCF1190F03D8AEF176
:1078D000570C6345E1DC731C1CD005B140420AB172
:1078E000F6B91160BDE8F08733F0100094F800E0BD
:1078F000654606F10204C0D1BEF1300F17D06BBB54
:107900000A234FF005091A4F9A46BFE700FB0AC049
:107910000126CBE722233046C8F80030002AE1D008
:10792000611EDEE794F800E00125B41CA2E7207890
:1079300000F0DF00582807D083B908234FF007096B
:107940006FF060479A46A1E7102394F801E04FF0EA
:107950000F0902346FF070479A4697E710234FF0F3
:107960000F096FF070479A4690E700BFD5D200101C
:1079700099999919FFF76ABF38B54B1C1AD09389AA
:1079800014465268CDB223F02003A381236BA3B128
:10799000636B934209DD23685A1E226003F8015C81
:1079A000636801336360284638BD214601F03AFD23
:1079B0000028F0D04FF0FF35F5E7236921682BB19F
:1079C0008B4203D211F8013CAB420ED0234604F1A6
:1079D0004000C4E90E12032101222063284661639E
:1079E00003F8425FC4E9003238BD01390132C4E90D
:1079F0000012D8E710B50C46096B69B104F14003D9
:107A0000994201D0FFF726FE0020E36B20636360FC
:107A100013B1A36B236010BDA289002123694FF02D
:107A2000FF3042F020026160A281F3E72DE9F04FC0
:107A3000834685B002FB03F00E9C0193A0B38846F9
:107A40000646D4E90015A84223D94FF0000904F1F5
:107A5000400ACDE9020240462A46FFF7FBFC2168B6
:107A6000236B58464F19A8441946C4F80490276060
:107A70003746761BDBB1534501D0FFF7EBFDE06BDA
:107A8000C4F83090606090B1A16BB04205462160AF
:107A9000E1D332464046FFF7DDFC0198D4E90032DD
:107AA000921B3344C4E9003205B0BDE8F08FDDE934
:107AB0000202A389284443F02003C01BA3810023B2
:107AC000B0FBF2F02269C4E9002305B0BDE8F08FF5
:107AD0002DE9F04FADF5377D8A4602AFC7E91202B6
:107AE000B1F90C20FB6296044B6E05D442F40052AF
:107AF00023F400538A814B669D04C3F3403401F1A3
:107B00008C80A1460822214607F15800FFF7F8FAB9
:107B1000BC63FC617C633C64BC62954BD3F8E4407D
:107B200001F0A2FD07F15802034607F1540100924B
:107B3000FA6CB86CA04700285CDBFB6C024603447F
:107B4000FB647B6D002B00F0D480012861D0252BD5
:107B500068D00028E1D0FB6C01389E1ADAF80430B6
:107B60001A463418751E002A16DDDAF80030691C32
:107B70006A7818780133904240F0BB80DAF804202C
:107B80008C42CAF8003002F1FF32CAF8042000F03B
:107B9000BB80002A0D46E8DC5146B86CFFF72AFF8F
:107BA0000028E2D03B6C002B40F09E80BB6B002B8A
:107BB00001F03380BB6BDE8818687EB10024051F9E
:107BC0008146A04655F8043F01341868FCF73AFC9A
:107BD0002B68A642C3F80080F4D148464FF0FF332B
:107BE0003B6408B1FCF72EFC386C07F53577BD46D1
:107BF000BDE8F08F4FF6FD730822002107F1580011
:107C00007B65FFF77DFAFB6C0133FB647B6D002B1A
:107C10006FD0584AD25C140700F1F1840120252B63
:107C2000024698D10024FE6C25463178A1F1250347
:107C300006F1010B552B5CD8DFE813F04F075B0012
:107C40005B005B005B0031075B005B005B005B007F
:107C50005B001E061E061E061E061E061E061E06CD
:107C60001E061E061E065B005B005B005B005B00E1
:107C70005B005B002B065B00570477002B062B068E
:107C80002B065B005B005B005B0070005B005B0031
:107C900066045B005B005B00AC045B005B005B00A8
:107CA0005B003C065B005B0039075B005B005B0030
:107CB0005B005B002B065B00590479002B062B064A
:107CC0002B060107530770005B0043070D071B07D6
:107CD00068042E075B005B00AE046B00FA065B00D5
:107CE0005B003C065B006B00BAF80C305A063FF5AF
:107CF0005DAFBB6B002B3FF477AFBB6B18683B6C81
:107D000001337FF46EAF55E702354D44A5EB06090C
:107D100003E72307EDD171785E4687E72107E8D1B5
:107D2000717844F002045E4680E744F00104124B8F
:107D30000326BB620A237B63DAF80430002B00F3CE
:107D4000EF835146B86CFFF755FE00287FF42AAF49
:107D5000C7F84CB0600641F10682731E032B01F296
:107D60006981DFE813F02D02DE0134010B0000BF52
:107D7000480F0020D5D2001061A70010B86C44F461
:107D8000F06801F077FC03683B626B1EB3F5AE7FD1
:107D900040F232876FF4AE7405EB040C40F25D15CF
:107DA00007F5B87B0023C7F80CC05C467B64FB6317
:107DB0003B63BB61C7F824B0C7E90433DAF80010AD
:107DC0000A78A2F12B034E2B50D8DFE813F03903C9
:107DD0004F0039034F004F007D039D009D009D0023
:107DE0009D009D009D009D009D009D004F004F0047
:107DF0004F004F004F004F004F002E039A009A0093
:107E00009A00600355034F004F0040034F004F009E
:107E10004F004F000E034F00EE024F004F004F0087
:107E2000E7024F004F004F00D20227034F004F00E0
:107E30004F004F004F004F004F002E039A009A0052
:107E40009A00600355034F004F0040034F004F005E
:107E50004F004F000E034F00EE024F004F004F0047
:107E6000E7024F004F004F00D202270318F4007FB3
:107E700067D0386A0378934263D183460026C7E906
:107E800001545546C24606E029609BF8000091F86F
:107E900000E086451BD11BF8010F3446C84601316E
:107EA000013609F10109002800F09186686801385F
:107EB00000286860E8DC2946B86CFFF79BFD30B904
:107EC00029689BF8000091F800E08645E3D043461E
:107ED000D046AA462246BC689146D7E9085B7C6238
:107EE0002E443B623446BE6C14F8011D52463046A7
:107EF000FFF742FDA542F7D13B6A7C6AA3EB090973
:107F000021E018F4006F1CD0FB6B796C5B1818D162
:107F100028F4C0787B64FB6304F8012B013DDAF898
:107F2000043009F10109013B002BCAF8043040F389
:107F30005B83DAF800300133CAF80030002D7FF49B
:107F40003DAFD7F824B03B6B0BB128F48078FB6BC6
:107F5000013B012B41F2DE807B6C013B062B40F2A2
:107F60007C8618F4807F00F06A8418F4806F40F0FB
:107F7000948714F8011C01F0DF03452B40F097862D
:107F8000651E09F1FF395246B86CFFF7F5FC18F091
:107F900010037FF4C2AD2B707B69002B40F0A087EB
:107FA00000225946B86C02F04FFBFB6A18F0010F33
:107FB000024605460E4603F1040400F06D861B6878
:107FC000C3E900563B6CFC6201333B64A5E56B1EC4
:107FD00044F45864B3F5AE7F40F2A9836FF4AE72F7
:107FE000A91840F25D1507F5B87B4FF000087A6BD1
:107FF0005E46CB46D146C246B046F963D9F800008A
:1080000090F800C0ACF12B034D2B62D8DFE813F0E1
:1080100056026100560261006100C702AB01AB016C
:10802000AB01AB01AB01AB01AB0143024302610009
:108030006100610061006100610061004E004E005E
:108040004E004E004E004E00610061006100610074
:108050006100610061006100610061006100610018
:10806000610061006100610061004A02610061001D
:108070006100610061006100610061004E004E001E
:108080004E004E004E004E00610061006100610034
:1080900061006100610061006100610061006100D8
:1080A000610061006100610061004A020A2A10DD7E
:1080B00024F4386406F801CBD9F80430013B002BD6
:1080C000C9F8043040F386820130C9F80000013D50
:1080D00094D14346E105D0467A63CA46D9469B46C9
:1080E00005D59E4200F29B845E453FF402AE14F03B
:1080F000100211D17B6B5946BD6A3270B86CA8472B
:10810000FB6AA20603F1040540F1E1831B681860D5
:108110003B6CFD6201333B64A6EB0B064644B14465
:10812000FBE4002D04F0100208BF4FF0FF35E0071C
:1081300040F1FF82002A40F01D85FE6A210656F8B4
:1081400004BB40F1D7867A64BBF1000F3FF4D1AD98
:108150008020FCF73DF97A6C0346002800F0D587B3
:10816000B96BCBF80000CC88B1F80480444580F0AE
:10817000D9850868B96B9E4640F824B04FF0200CB2
:108180000134FE62CC80DAF80010DFF8BC83097895
:1081900018F8016016F0080600F0B883002A7FF492
:1081A000BCAC1A60A3EB0E03991001318C4503D9C6
:1081B000BBF1000F40F028863B6C01333B64ACE41C
:1081C000002D04F0100308BF4FF0FF35E0073B63BC
:1081D00040F13582D7F82CB0002B40F0C2845BF818
:1081E000043B21063B6240F18C86002B3FF481ADBD
:1081F0008020FCF7EDF88046002800F086873B6A77
:108200001860BB6BDC889A88944280F0A58518685A
:108210003B6AC7F82C8040F824300134BB6BDC800B
:1082200020237B62C7F818B00024FE69CB467D642A
:1082300001F01AFAA0423FF4B5AC032E07F1600931
:10824000DAE9003202F1FF3213F8011BCAF8042008
:1082500007F5B872CAF80030115504F1010403D1D2
:10826000D9F80030042B04D0082200214846FEF73C
:1082700047FFCDF8009007F5B87223464146B86C29
:1082800002F008FC421C06463FF48CAC002840F08B
:1082900079840346C8F800000822002107F168002D
:1082A000FB63FEF72DFFFB6BB86C07F150011A461C
:1082B000A24BD3F8E0301D4607F16803A847012818
:1082C0000CBF97F85030002307F17002D35C002BED
:1082D00000F02386032EA34400F05D847B6C013BF9
:1082E0007B643B6BBBB908F10408F86A7D6AA8EBB4
:1082F0000004B5EBA40F0ED83B6A63B1E900FCF7AC
:1083000083F8F862002800F0008769003B6A00EB00
:10831000040879621860DAF804300024002B40F376
:1083200046847B6C002B83D1D946D7F818B0FE6108
:108330003B6BA3B9C8F80030FB6A7A6AA8EB03016B
:108340008B1001339A4207D93C6A2CB10431206862
:10835000FCF75AF800B120603B6C01333B64C7F86E
:108360002CB0FFF7DABB764B24F4386433F91220D3
:10837000A0E608F41863B3F5807F7FF4E2AD3B6BB1
:10838000012B7FF4DEAD302328F48078013D04F822
:10839000013B002348F400683B63BDE57B6C062B82
:1083A0007FF4CFAD07237B64B6E518F4006F3FF48C
:1083B000C8AD08F4A063B3F5806F07D018F4806FE0
:1083C0003FF4BFAD3B6B002B00F0B38618F4007F89
:1083D00004D13B6BB9695B1AC7E9044328F4786898
:1083E000002348F4C0783B6396E5FB6B002B40F01C
:1083F00075823B6B002B40F0718208F4E063B3F5AB
:10840000E06F00F0A1857B6C012B02D0042B7FF480
:1084100098AD7B6C0133DBB27B647DE57B6C072B15
:108420007FF48FAD08237B6476E518F4006F40F08D
:108430003A82FB6B012B7FF484AD0223FB636BE577
:1084400018F0800F3FF47DAD28F0800864E57B6C68
:10845000002B40F04B823B6B002B40F0478208F42E
:10846000E063B3F5E06F00F077850023D7F824B020
:108470007B6400233B636AE518F4006F40F00C82D4
:108480007B6C022B7FF45DAD03237B6444E518F421
:10849000006F8ED038E52A4B33F91220082A3FF7B7
:1084A00007AE16E604F4C063B3F5007F7FF411AEA7
:1084B00024F40074102244F4A064FBE523067FF545
:1084C00008AE24F08004F5E518F4807F3FF41CAD7D
:1084D0003B6B28F0800801333B63FB68002B3FF4C3
:1084E0001DADFB68013BFB6019E544F0010444F05D
:1084F00040040026C7F84CB0DAF80430002B3FF7F0
:1085000029ACD7F84CB01CE444F001040D4B032611
:10851000BB6208237B63DAF80430002B7FF711ACD1
:10852000DAF80020DFF82080137818F803301907F4
:1085300040F124854346D0469A460EE0480F00207D
:10854000D8D3001075790010D5D20010C8F80020DB
:1085500013781AF803301B0717D5D8F8043009F13F
:1085600001090132013B002BC8F80430EEDC414622
:10857000B86CFFF73FFA002840F04883D8F8002095
:1085800013781AF803301B07E7D4C246C7F84CB07B
:10859000FFF7E3BB44F001040226FFF7CDBB230540
:1085A0007FF588AD12B944F400740822610500F12A
:1085B0008A81FB6B24F4607413B1013B0135FB63CA
:1085C000D9F804300AF1010A013B002BC9F8043044
:1085D0003FF77AAD4946B86C7A64FFF70BFA7A6CCC
:1085E00000283FF474AD74E55146B86CFFF702FA09
:1085F00000287FF4A6AC002D7FF4E0ABA1E4DAF80C
:108600000420BC6C11E0DAF80030BD491A7801335F
:108610008A5C10077FF581AADAF8042009F10109C4
:10862000CAF80030013ACAF80420002AEBDC5146AF
:108630002046FFF7DFF90028E5D0FFF76EBA3B6B65
:10864000002B40F05682FB6A53F8042B3B6314F076
:1086500080031646FA6300F05C84002A3FF449ABBD
:108660002020FBF7B5FE044600283FF49FAABB6B11
:108670003060B3F80480DE88464580F03A8318689D
:10868000FB6B40F826300136BB6BDE802023DAF826
:10869000000007F170020178515C00293FF429AB1A
:1086A000F96B2646C7F82C909046B1F1000B99461D
:1086B00018BF4FF0010B07E0DAF80000027818F855
:1086C0000220002A00F0B282DAF80420411C013AAC
:1086D000CAE90012027804F8012BA21B4A457A6409
:1086E00010D33046BBF1000F0CD04FEA4909494680
:1086F000FBF78AFE064600283FF458AA7A6CFB6B0B
:1087000084181860013D00F09182DAF80420002AF4
:10871000D2DC5146B86CFFF76DF90028CCD0B442DA
:108720004B46D7F82C903FF43DAAA61B84E20021CB
:1087300059E4002A40F07483FA6A14F0800452F875
:10874000043B7B64FA6300F0C0831C46002B3FF4BB
:10875000D0AA2020FBF73CFE064600283FF426AABC
:10876000BB6B2060B3F80480DC88444580F0AA82AB
:1087700018687B6C4FF0010B40F824300134BB6B60
:10878000DC802023DAF80000DFF87481017818F823
:108790000110090700F1AB82424634463146984643
:1087A0002E464B469146DAF804200D46013ACAF8A7
:1087B0000420421CCAF80020027805F8012B2A1B6D
:1087C00042453A6312D32046BBF1000F0ED04FEA68
:1087D0004808FB624146FBF717FE044600283FF4B9
:1087E000E5A97B6C3A6B18608518FB6A013E0CD0DA
:1087F000DAF80420002A40F3B783DAF800002946AB
:10880000027819F802201207CDD59946291B434654
:108810002E468944013100208B42307008D9BBF1CB
:10882000000F05D07C6C2068FBF7EEFD00B12060E6
:108830003B6C01333B64FB6BFB62FFF76EB918F0D6
:1088400010037FF46AA9237008F4C063B3F5806F46
:108850007FF4A2ABBB693A6B93423FF4A1AB9A1A87
:1088600007F2C32327499C4228BF07F2C2242046AF
:10887000FDF7C8F8FFF794BB14F08F0F7FF439AA07
:1088800005EB850501EB450571785E46303DFFF748
:10889000CDB90426FFF750BAFB6B796C5B187FF4F7
:1088A000EFADFFF735BBFB6B796C5B187FF4C1ADA7
:1088B000FFF72EBB44F40074134B0326BB62102356
:1088C0007B63FFF739BA24F4B064FFF7F3BB2107E9
:1088D00040F16282FB6A1B68187019E4FB6B022B83
:1088E0007FF491AD0323FB63FFF716BB7B6C032B77
:1088F0003FF48FAD052B3FF48CADFFF722BB00BFDB
:10890000D5D2001050C3001075790010C7F824B0FC
:10891000C7F82080A846D7F81CB01D46C7F830E03D
:10892000C7F83CC07A6400F09FFEB0423FF43AA919
:10893000BBF1030F07F16804DAE9003202F1FF32FC
:1089400013F8011BCAF8042007F5B872CAF8003002
:10895000915506F1010602D12368042B04D00822A8
:1089600000212046FEF7CCFB0094334607F5B87291
:108970002946B86C02F08EF8B0F1FF3F83463FF411
:1089800011A9002800F02F8210F1020F2CD02868C6
:1089900002F0AAF8002840F01E83BBF1030FB14497
:1089A00002D12368042B01D008F1FF387E6C002E21
:1089B00040F089820435386BFB6B2C1AB3EBA40FA3
:1089C00000F281827A6A002A00F07D82D900FBF7EA
:1089D0001BFD01463863002800F09783FB6B0519E7
:1089E00058007B6AF8631960DAF80430002B40F312
:1089F000C982DAF800303A6A1B78D35C1B0702D4CC
:108A0000B8F1000F8FD1C7F81CB02B46D7F824B0AF
:108A1000D7F830E0D7F83CC07A6CFFF7BFBB16F848
:108A2000011C5246B86C013EFEF7A6FFFFF75CBB87
:108A3000BA4B0326BB620A237B63FFF77DB923078A
:108A40007FF457A97178682900F0A08144F00404EC
:108A50005E46FFF7EBB814F08F037FF44AA9B96BB9
:108A6000002900F03782717844F080045E46FFF7F9
:108A7000DDB8E10600F1C680FA6A52F8043BFA62FA
:108A8000220700F1BD80660740F19282A3F80090B2
:108A9000C7F84CB0FFF741B844F408740CE725431D
:108AA0007FF427A9717810245E46FFF7BFB85946B6
:108AB00007F1700000F066FC44F040040126F86401
:108AC0001AE521077FF415A971786C2900F0588107
:108AD00044F001045E46FFF7A9B8C7F84CB0FFF7B1
:108AE00038B88F4B0326C7F84CB0BB6200237B63BA
:108AF00002E5DAF8003007F170021978515C0029BC
:108B00003FF4F7A80133012DCAF80030DAF8043039
:108B100003F1FF33CAF804303FF401ABBC6C90465C
:108B200014E0DAF800301A78013318F80220002A2D
:108B30003FF4F5AA0136CAF80030DAF80430B5423D
:108B400003F1FF33CAF804303FF4E9AA002BE8DC54
:108B500051462046FEF74EFF0028E2D0B144FEF712
:108B6000DCBF002307F154027B629046FB623B624C
:108B7000FFF758BB4FF0000C07F15403E646E346FD
:108B8000FFF701BB831C0DD0D8F800305D1C7FF4CB
:108B900083ABFFF799BBD9F80030042B7FF49EAB71
:108BA000FFF79FBBDAF80430002B3FF741AB51468B
:108BB000B86CFEF71FFF00283FF4B3ABD946FE6147
:108BC000D7F818B0002C3FF4B3ABFEF7EBBFBC688E
:108BD0003246396A2046C7F81880D046AA467D68D2
:108BE00000F002FDBB6928F42078013D0446994657
:108BF0003B6BBB61FFF793B94FF0000CFFF7D0B8A8
:108C000083F80090C7F84CB0FEF787BF3B6CC246B4
:108C1000002B3EF4CBAFFFF767B84FF0FF333B6458
:108C2000386C07F53577BD46BDE8F08FA61B4B467F
:108C3000D7F82C903FF45DA8711C00228B42227063
:108C400003D9BBF1000F40F0D680B1443B6C013337
:108C50003B643B6BFB62FEF760BF7B6C022B40F218
:108C60006C82032B3FF47DA97B6C1E1FF6B2F5438B
:108C70007E6426462544BC6C16F8011D52462046EB
:108C8000FEF77AFEAE42F7D1344609F1FF397E6C29
:108C9000A9EB0609FFF765B9FB6A18F0020FD3F8D4
:108CA00000B000F09380CBE90056FFF78BB9524635
:108CB000B86CFEF761FEA9F10209A51E14F8021CAA
:108CC000FFF761B94FF6F67188453EF673AF08F1CC
:108CD0000808BB6B4FEA88011868FBF795FB002872
:108CE0003EF468AFBB6BA3F80480186041E5012136
:108CF00091E54FF6F67398453EF65CAF08F108082B
:108D0000BB6B4FEA88011868FBF77EFB00283EF436
:108D100051AFBB6BA3F804801860B1E47579001003
:108D200061A700104FF6F671FA637864884500F287
:108D3000EC8108F10808BB6B4FEA88011868FBF763
:108D400063FB002800F0E181BB6BFA6BA3F80480A1
:108D500018607B6CFFF70EBA4FF6F6739A4200F27A
:108D6000D48102F10806BB6BB1001868FBF74CFB1D
:108D7000002800F0CA81BB6B9E801860FFF748BADC
:108D8000B17844F002040236FEF750BFB17844F0E7
:108D900008040236FEF74ABF620779D414F00102D4
:108DA00040F01081A30740F10D819F4BB96AB86C68
:108DB00099427B6B594600F0CE8101F0A1FD0B4634
:108DC000FA6A1168C1E90003FFF7A2B90B46FAF786
:108DD00071FD002870D128463146FAF715FDCBF811
:108DE0000000FFF7EFB8286001F07EFE002840F099
:108DF000F280B144D8E5FC6B2068FBF705FB002846
:108E00003FF423AF206020E7191DDBF80000FBF7DB
:108E1000FBFA00283FF4D0A9CBF80000FFF7CCB94B
:108E2000DAF80030DFF808821A7818F80220140700
:108E30003EF573AE0133012DCAF80030DAF8043084
:108E400003F1FF33CAF8043000F089810124BE6CBD
:108E500013E0DAF800301A78013318F8022010070E
:108E600013D40134CAF80030DAF80430A54203F113
:108E7000FF33CAF8043000F0AB80002BE9DC514628
:108E80003046FEF7B7FD0028E3D0A144FEF745BE0B
:108E9000FB6A1B681880FFF73BB95C455E467EF6AF
:108EA00028AFBD6C14F8011D52462846FEF764FD3C
:108EB000B442F7D1FEF71DBF5C4800F0DFFBCBF8F2
:108EC0000000FFF77FB800268EE57E6CA3462346A0
:108ED0007C6457E482B0CDE9023302ABBB63C2E5E8
:108EE0003C690A230022B86C611C01F039FC7B69E3
:108EF000C21AB5E45B46944696469346FE62FFF777
:108F000042B93B6BD7F820807B62FB623B62FFF784
:108F100089B9FC6BFB63FFF7BABBD946FE61D7F892
:108F200018B02646002C3FF403AA07F5B873BD6CB1
:108F30001C19013E524614F8011D2846FEF71CFD7F
:108F4000002EF6D1FFF7F4B9012328F4F068FB6393
:108F500000233B63FEF7E0BF012328F4F0687B6445
:108F600000233B63FEF7D8BF5146B86C3B63FEF766
:108F700041FD3B6B00283FF440AC46E4C7F84CB0E1
:108F8000FEF7EBBE5146B86CFEF734FD00283FF407
:108F900030ADC7F81CB02B46D7F824B0D7F830E076
:108FA000D7F83CC07A6C002E7EF4FCADFFF7F6B823
:108FB000E5070AD4A40708D54FEAE972C3F8009080
:108FC0005A601FE6FB6AFFF7A1B8C3F8009019E6E4
:108FD000A944FEF7A2BDC7F81CB02B46D7F824B0B1
:108FE000D7F830E0D7F83CC07A6C002E3FF4D6A812
:108FF00007F5B871C7F84490FD63F0468C19E14657
:10900000BD6C3A63013E524614F8011D2846FEF736
:10901000B3FC002EF6D1CC46FB6BC646D7F8449085
:109020003A6BFFF7BBB800BF7579001018C100108C
:10903000D5D20010012D04F0100238BF012514F024
:1090400001037A6400F09380FB6A002A40F0DE801E
:1090500053F804BB24063B6300F10281D846D7F8DD
:1090600044B05B46DC46C7F83CB0002664469B46ED
:1090700000F0FAFAB0423EF495ADDAE90032013A76
:1090800013F8011BCAF8042007F5B872CAF80030BB
:10909000731C915507F16806FA69032A02D13268F8
:1090A000042A06D0082200213046FB62FEF728F889
:1090B000FB6A009607F5B8724146B86CFB6201F096
:1090C000E9FC0246F861501C3EF46CADFB6A002AD4
:1090D00040F00A8199447B6C013D002B40F01281E5
:1090E000C8F80030A8EB0406BBEBA60F00F23D81E8
:1090F000FB6B002B00F0398120464FEACB01FBF7D8
:1091000083F90446002840F02A814FF0FF333B6486
:10911000FEF7EFBD5C455E467EF6EBADBD6C14F828
:10912000011D52462846FEF727FCB442F7D1FEF750
:10913000E0BDD7F824B0FFF79CB95C457EF6D9AD09
:109140005D4614F8011D5246B86CFEF715FCAC42A2
:10915000F7D1FEF7CEBD01F09BFC0B4630E609F1DE
:109160000109FEF7DABCD7F84CB0FFF7D9B97A6C31
:10917000002A51D1D7F82C80240658F8046B62D508
:10918000002E3EF4B6AD2846FBF722F90246002831
:109190003EF40CADBB6B3060B3F806B09C88A345C1
:1091A000C0F093804FF6F67378649C423EF602ADB1
:1091B0000834BB6BA1001868FBF726F900283EF4C1
:1091C000F9ACBB6B7A6C9C801860B96B0BF1010336
:1091D00040F82B60CB801146CDF800A02B46012231
:1091E000B86CFEF723FC0446002870D0854205D9F0
:1091F00001463068FBF708F900B130603B6CA144D0
:10920000C7F82C8001333B64FEF787BC3B63002327
:109210009C469B46984626E71C46DAE900239D4279
:1092200002EB030147DDCAF800105146B86C1C443C
:10923000ED1AFEF7DFFB0028EFD0002C3EF4B2ACB5
:10924000A144FEF76ABCCDF800A02B4631460122AE
:10925000B86CFEF7EBFB04460028CFD1FEF7A2BCAA
:10926000BBF1000F3EF445AD8020FBF7B1F880461E
:1092700000283FF44AAFBB6BCBF80000DE889C8827
:10928000A6422FD34FF6F6739C423FF63EAF08340A
:10929000BB6BA1001868FBF7B7F800283FF435AFA7
:1092A000BB6B9C801860BB6BC44640F826B001368F
:1092B000DE802023D7E65B1B2A442C44CAF8043006
:1092C000A144CAF80020FEF728BC18687DE73B6C73
:1092D000002B3EF46FACBAF80C305B067EF50DAD9A
:1092E000FEF768BC1868DEE7FA69911C23D0032AF0
:1092F000994402D13368042B00D0013D7B6C002BD4
:109300003FF4F0AEDAF804300026002B19DD002D12
:109310007FF4AEAE5B46A446D7F83CB0A8EB0C0198
:10932000B3EBA10F02D9BBF1000F21D17B6C002B55
:109330007FF48FAC8AE4DAF804201E46002A3FF757
:1093400097AE5146B86CFEF755FB0028DFD05B4660
:10935000A446D7F83CB0002EE0D0FEF723BCFB6B50
:1093600000EB06084FEA4B0B186008F10408C9E748
:10937000DBF80000FBF748F80028D7D0CBF8000056
:10938000D4E700BF70B50C7884465E2C24D000234F
:10939000481C9E4600220CF5807163F3070263F3BC
:1093A0000F2263F3174263F31F62634643F8042BF3
:1093B0008B42FBD174B18EF00101451C0CF80410F6
:1093C00015F8013C2D2B0ED05D2B0AD01BB11C468D
:1093D0002846F2E7013870BD0123881C4C789E4670
:1093E000D8E7284670BD90F801E0BEF15D0F15D0BA
:1093F000744513DC661C02300CEB060202F8011BFC
:10940000A2EB0C03013B9E45F8DCAEEB04030235F6
:10941000013B7445A8BF00239C19D1E72D242846A1
:10942000CBE700BF2DE9F0410C46096B04F1400386
:10943000994214D0666B77003A46FDF7FBFB054670
:1094400030B300EB0608014632464046FEF702F80C
:10945000C4F80080C4E90C570020BDE8F0814FF447
:109460008061FDF729F998B194F842204FF48061AA
:10947000206300F2FD33616380F8FF2394F84120FC
:1094800080F8FE2394F8402080F8FD232360E3E772
:109490004FF0FF30E1E700BF11F0FF01034600F09D
:1094A000030239D08ABB10B501EB012E02680EEB26
:1094B0000E4EA2F101338EEA020423EA0203A4F164
:1094C000013222EA0402134313F0803F0FD150F817
:1094D000044F84EA0E0CA4F10133ACF1013223EA0B
:1094E000040322EA0C02134313F0803FEFD0037809
:1094F00023B936E010F8013F002B32D09942F9D160
:1095000010BD8A4228D09A0729D01A78184601330C
:10951000002AF6D110467047CAB90268A2F1013399
:1095200023EA020313F0803F08D150F8042FA2F180
:10953000013323EA020313F0803FF6D003785BB1D6
:1095400010F8013F002BFBD17047990705D0184652
:1095500013F8012B002AF8D170471846DDE71846AA
:10956000A1E7184610BD00BFCAB384460B4630B50C
:1095700004460843800719D09CF800000C78A042EC
:1095800012D150B3012A28D0E64603E01CEB030FAA
:1095900023D010B31EF8010F11F8014FA2EB0E03F8
:1095A000A04203F1FF33F1D0001B30BD032A07D8DE
:1095B000E2E7043A11D01EF0803F0ED1032A10D901
:1095C0002068194653F8045BA446A0F1013E043418
:1095D000A8422EEA000EECD0CEE7002030BD1046A7
:1095E0007047A4461946C7E740EA01039B0710B439
:1095F000044601D1032A1CD801F1FF3C07E01CF806
:10960000011F501E03F8011B41B102461C462346B0
:10961000002AF4D120465DF8044B7047F8B1A01839
:1096200003F8011B8342FBD1002CF3D15DF8044BFE
:1096300070478C4604E0043A44F8040B032A0CD922
:10964000DCF8000061460CF1040CA0F1013323EAC0
:10965000000313F0803FEED0CEE76146CCE718461A
:10966000002CD7D1E2E700BF014B93F828017047E7
:10967000480F00200048704738100020004870470D
:109680000000C07F82B049B15AB16BB113780B6052
:109690001278101E18BF012002B0704701A9002ADD
:1096A000F3D1104602B070476FF00100F4E700BF3D
:1096B0002DE9F04F88469FB0002183460792002293
:1096C0001A910021CDE9041242461746199212F868
:1096D000019BB9F12D0F5FD801A151F829F000BF0E
:1096E0002D980010999700109997001099970010E5
:1096F000999700109997001099970010999700106A
:1097000099970010CB960010CB960010CB960010C6
:10971000CB960010CB9600109997001099970010E7
:109720009997001099970010999700109997001039
:109730009997001099970010999700109997001029
:109740009997001099970010999700109997001019
:109750009997001099970010999700109997001009
:10976000CB960010999700109997001099970010C8
:1097700099970010999700109997001099970010E9
:109780009997001099970010999700109B9D0010D1
:1097900099970010B39D001000220892B9F1300F84
:1097A0007ED000230A93A9F13003092B00F2348400
:1097B000002538462E462C460130082C05EB850244
:1097C00004F1010406EB8601199090F80090CCBFDB
:1097D00003EB420503EB4106A9F13003092BEBD95A
:1097E0000122A349FFF7C0FE58BB199BA24609906E
:1097F0005A1C19925B78A3F13002092A09D801306A
:1098000091461999002A40F0D4844B1C19934B7847
:10981000F1E74FF0010923F02002452A40F0B7821A
:1098200044EA00030A9A134340F05082079B002643
:1098300000270BB1C3F80080304639461FB0BDE8A1
:10984000F08F29F0200200204B46A246452A81468F
:10985000099000F03B820E90002C35D10A9A024309
:1098600040F08382B9F1000FE0D1692B00F0CC8485
:1098700000F31F83492B00F0C7844E2BD6D17D49BE
:1098800019A801F047FD0028D0D0199B1B78282B80
:1098900000F08385784801F017FA06460F4666E225
:1098A0007A7802F0DF02582A00F03F8401371997D6
:1098B00097F80090B9F1300FF8D0B9F1000F00F02F
:1098C000548201230A936EE7099ABAF1000F08BF88
:1098D000A2460E9B102C3046A046A3EB0203A8BF65
:1098E0004FF010080D93F9F7AFFF092C02460B4615
:1098F000CDE9042317DD614B03EBC80353E91223C1
:10990000F9F70EFF02460B462846CDE90423F9F786
:109910009BFF02460B46DDE90401F9F7D9FE0F2C47
:10992000CDE9040124DC0D9B002B00F0B5830D9BD9
:1099300040F3AD82162B40F38484C4F125030D9AC5
:10994000934215DBC4F10F044C4D05EBC401DDE976
:109950000423D1E90001F9F7E3FE0D9B1C1B05EB85
:10996000C405D5E90023F9F7DBFE06460F46FEE104
:10997000A4EB08030D9A9D18002D40F32B8215F0DF
:109980000F000AD03D4901EBC001DDE90423D1E914
:109990000001F9F7C5FECDE9040135F00F034BD006
:1099A000B3F59A7F00F35A84102B4FEA231540F346
:1099B000B385DFF8DCE04FF0000C0A96F046E14694
:1099C0007646DDE9042315F0010F1046194607D04D
:1099D000D8E90023F9F7A4FE4FF0010C02460B462C
:1099E0006D1009F1010908F10808012DEBD1B64607
:1099F0000A9EBCF1000F01D0CDE90423059B0EEBBC
:109A0000C901A3F154730593DDE90423D1E90001F1
:109A1000F9F786FE1A4B0A460B40CDE904011949B5
:109A20008B4200F21B8418498B4240F2C9844FF0EC
:109A3000FF32164BCDE9042300230C9323465246F4
:109A400039465846009601F0E1FD1590002800F0D7
:109A500005840E9A099B9B1A0D9A002A22EAE2724B
:109A6000A8BF002314920E9300239A460993EBE0BB
:109A700058C30010ACC3001018C10010580A0110E0
:109A80000000F07F0000A07C0000907CFFFFEF7FD3
:109A9000300A0110D21A1F2AA4EB020400F37C82C0
:109AA0000123002593401E46A0444C440C9BA14535
:109AB00098444B46A8BF23464345A8BF4346002BC6
:109AC00004DDE41AA8EB0308A9EB03090E9B002BA5
:109AD00000F30382002C00F319820D9B002B00F38E
:109AE0004C82B8F1000F00F33C82B9F1000F08DDA1
:109AF00051464A46584601F06FFF8246002800F062
:109B000039823A461A99584601F0FCFF099000281C
:109B100000F03082099A0023D168D3600F9151463A
:109B200001F0CEFF0028C0F27984DDF8149000F037
:109B3000E7835146099802F08DF900224FF08043E7
:109B400004460D46F9F7EEFE002800F0B6810F9BA3
:109B5000002B40F02882049B002B40F01283C9F3B5
:109B60001303002B40F09B820022954B2046294690
:109B7000F9F7C4FE002840F0BA830022914B20463A
:109B80002946F9F7CDFD0A460146109002F100433F
:109B9000CDE912121193DFF834828B4B09EA0808E1
:109BA0009845DDE9104500F00A820C9B1BB3B8F123
:109BB000D46F20D880A3D3E90023DDE91201F9F79F
:109BC000B1FEA0B1DDE91201F9F762FE012838BF4C
:109BD0000120F9F739FE0F9BCDE91201002B40F06F
:109BE000E38201F1004316901793DDE9164505F174
:109BF000D663A3EB0805DDE90A0102F043F802464B
:109C00000B4620462946F9F78BFDDDE90A23F9F7D3
:109C10005FFD0C46CDE904016C4B2340434503D165
:109C20000C9B002B00F05C821A99584601F092FCC4
:109C30003946584601F08EFC5146584601F08AFCE0
:109C40000999584601F086FC159C5846616801F058
:109C50005BFC0746002800F08D81226904F10C01AD
:109C60000C3002329200FDF7F5FB1CAB5846019315
:109C70001BAB9DED047B009353EC172B8DED0A7B02
:109C800002F088F81A90002800F049810121584616
:109C900001F068FD8246002800F06C811B9B002BC0
:109CA000C0F259810E9ADDF8508003EB02090C9A3C
:109CB0001C9C9B1A464A2344C4F13604013B934240
:109CC000FFF6E8AE012300251E46EDE6DDF86480D0
:109CD00008F10103199398F801302B2B00F09981BA
:109CE0002D2B57D14FF0010E08F10203199398F86C
:109CF0000230A3F1300CBCF1090F00F24881199A2F
:109D0000302B0C920BD1013219921378302BFAD0F0
:109D1000A3F131010C92082939D8A3F1300C0C9B26
:109D2000591C19915B78A3F13002092A00F2818253
:109D300001310CEB8C0C199103EB4C0C0B78ACF152
:109D4000300CA3F13002092AF2D90C9A891A082999
:109D500040F36F8244F61F620E92BEF1000F3FF493
:109D60007BAD0E9A52420E9276E500260027079AA6
:109D70000AB1199B1360089B002B3FF45DAD07F1FE
:109D8000004330461F4639461FB0BDE8F08F002221
:109D90000E9261E54FF0000EABE7002208927A1CAC
:109DA000199297F80190B9F1000F3FF43FAD1746B3
:109DB000F4E401220892F2E70000C0FFFFFFDF4158
:109DC0000000F03F0000E03F0000E07F0000F07F77
:109DD00002FCFFFF3FF430AE6D4215F00F020AD0D7
:109DE000B74B03EBC203DDE90401D3E90023F9F724
:109DF000BDFCCDE904012D113FF41EAE1F2D40DC4A
:109E000015F01003DFF8D4824FF0000C18BF6A235E
:109E10000C93DDE9042315F0010F1046194607D015
:109E2000D8E90023F9F77CFC4FF0010C02460B4601
:109E30006D1008F10808EED1BCF1000F01D0CDE99A
:109E400004230C9BA3B1DDE90401C1F30A52C2F162
:109E50006B03002B0ADD1F2B40F382830020342B81
:109E6000049040F3B8834FF05C7305936A230C931E
:109E700000220023DDE90401F9F72EFD00283FF45C
:109E8000DDAD222300260027CBF800306FE7163324
:109E9000FFF66EAD099B0E9A9A1A894B03EBC2032B
:109EA000DDE90401D3E90023F9F760FC06460F461B
:109EB0005DE76E2B3FF4E3ACB8E4824B20462946C5
:109EC0000022F9F72DFC0F9BCDE91201002B71D177
:109ED00001F10043109011935DE651461A46584631
:109EE00001F020FD8246002844D001461A9A5846C7
:109EF00001F066FC00283DD00F9058461A9901F0F9
:109F000029FB0F9B002C1A937FF7E7AD22461A9985
:109F1000584601F061FD1A9000287FF4DEADB94685
:109F2000054622230026684FCBF8003029465846C4
:109F300001F010FB4946584601F00CFB51465846CB
:109F400001F008FB1599584601F004FB09995846A1
:109F500001F000FB0BE7149ADDF83890A2EB030840
:109F6000A5E639464246584601F036FD0746002828
:109F70007FF4BBADB9461A9DD3E73946149A5846CB
:109F800001F0D0FC074600287FF4ABADF2E70022D9
:109F9000CDF864800E925FE44C4AD31A012202FA93
:109FA00003F5164680E59FED427B8DED107B8DED30
:109FB000127BF0E59DED127B8DED107BEBE5A9F1B9
:109FC0005473DFF804910593DDE9044520462946E2
:109FD00001F058FEDDE91023F9F7A2FB2B462246DB
:109FE000F9F776FB3A4B01EA09099945CDE90401F5
:109FF00040F2D68003F15473DDE90A01994202D19F
:10A0000006460136B6D04FF0FF33324CCDE904346A
:10A010000AE64FF0000E67E601222F493846FFF7A7
:10A02000A3FA824658B14FF0000A4B4655465646B1
:10A0300050465446D146CDF824A0FFF7ECBB199901
:10A040004B1C19934B78302B40F04F818A1C1046E3
:10A05000199201320378302BF9D0401A0138A3F15C
:10A060003102082A0FD8199F0026A3F130090124D4
:10A07000431C39463546099306EB8606002009EB5A
:10A080004606FFF7C2BB00224FF0010916461446F0
:10A0900015460992FFF7BFBBDDE9046767E69FED50
:10A0A000067B8DED107B9FED027B8DED127B72E5C3
:10A0B000000000000000F03F000000000000F0BFC2
:10A0C000580A01100000E03F0000F07FE2FBFFFFB4
:10A0D000FFFF9F7CFFFFEF7F58C3001028D40010C4
:10A0E000DDE9125628463146FAF722F9FAF71AF84E
:10A0F0000B46024631462846F9F7FEFA049D0F9EAC
:10A10000C4F3130C04462E430D4656EA0C0326D125
:10A11000C0A3D3E90023F9F7F1FB00283FF484AD95
:10A12000B946DDE904671A9D00E7029319A9089B67
:10A130005846AF4A01931AAB00931BAB00F01CFECC
:10A1400010F00F0504463FF410AE062D40F08A8053
:10A150007B1C0022002600270892199307E69CA387
:10A16000D3E90023F9F7CAFB0028D9D120462946B4
:10A1700099A3D3E90023F9F7FDFB00283FF454AD80
:10A18000CEE7049B012B8AD1B9F1000F87D1B946E4
:10A190001A9C2223254600260027CBF80030C5E66E
:10A1A00001F15474059437E59DED127B8DED167B1E
:10A1B0001BE5012840F33B8204EB000E0C900EF1EE
:10A1C000FF3C02E0460064450BD0082C06EB8600FD
:10A1D00004F10104F6DD05EB8503102CD8BF5D000A
:10A1E000F1E70C987446099BBCF1080F03440993EE
:10A1F0007FF742AF102C4FF00000DCBF05EB850568
:10A2000002EB4505FFF701BB7A4919A801F082F876
:10A2100000283FF40BAB199B19A87749013B199310
:10A2200001F078F810B9199B013319930026734F88
:10A230009DE544F61F629445A8BF9446CDF838C00A
:10A240008BE50D986E4901EBC001DDE90423D1E9EE
:10A250000001F9F765FA06460F4688E52223CBF898
:10A260000030E3E71A9A3AB135211CA801F020FE2C
:10A2700058461A9901F06EF9013D1B9B042D00F21E
:10A28000D981DFE805F0032C291E030003F23342D5
:10A290001C9B04931D9B23F4801343EA02530593F4
:10A2A000E20502D543F000430593544A1A40DDE924
:10A2B0000467002A7FF45BADFCF7D6FF222303601E
:10A2C00055E54FF0FF326FF00043CDE90423E3057D
:10A2D0007FF5E2AE059BE5E7484B0593F7E7DDE93F
:10A2E0001C121D9BCDE90412DAE75046B7E69FED3C
:10A2F0003C7B8DED107B9FED3C7B8DED127B4AE42A
:10A300004B460F98B646B946AC463E49C3F31302D6
:10A31000DDE90A67002800F0B5808A4200F00A8172
:10A32000A5BB049A1EEA020F33D030463946049387
:10A3300001F0A8FC0C9B002B00F02581049BC3F3CB
:10A340000A53C3F16B0CBCF1000F40F365812E4C36
:10A35000002204EB0C53F9F7E3F902460B463046B2
:10A360003946F9F7B5F906460F4630463946274BC8
:10A370000022F9F7D5F9214B06460F460B40002B7A
:10A380007FF4D1AE2223CBF80030CCE61CEA030FD9
:10A39000CBD10C9B002BE8D1C5E619A81CAA1C49FF
:10A3A00000F0D2FF05287FF475AA1D9B43F0FF4300
:10A3B00043F4E00305931C9B0493DDE90467D6E4B2
:10A3C00002F154730593FFF737BB00BFAFF3008072
:10A3D0009535A094FFFFDF3F35E5AF350000E03F46
:10A3E000000000000000E0BF000000000000E03FAF
:10A3F00010D40010A0C30010A4C300100000F07F10
:10A40000580A0110FFFF0F000000F03F0000503914
:10A41000FCD300109535A094FFFFCF3F0F9BB946AA
:10A42000DDE90401DDE90A670343B2D1C1F3130397
:10A43000002BAED121F00044240D2405B4F1D66FD9
:10A440002546A6D9099A536913B91369012BA0DDD2
:10A4500009990122584601F0BFFA5146099001F0CE
:10A460002FFB002895DD0C9BD3B1A5F580136FEA77
:10A4700013536FEA035305934FF0FF330493DDE961
:10A48000046772E7D2B9DDE904452246002C49D1C0
:10A490000C9A002A40F08E8025F00044240D2405FB
:10A4A000A4F580141A9D6FEA14536FEA03530593C1
:10A4B0004FF0FF330493DDE9046737E5ADBB049A41
:10A4C0001EEA020F3FF465AF30463946049301F0AF
:10A4D000D9FB0C9B002B00F08680049BC3F30A532E
:10A4E000C3F16B0CBCF1000F40F39E80524C002274
:10A4F00004EB0C53F9F714F902460B463046394683
:10A50000F9F7FAF80022002306460F46F9F7E4F9B6
:10A5100000283FF42AAF3BE64FF00009DFF824E1C2
:10A52000FFF76CBABCF1000FCAD01CEA030F3FF46E
:10A5300030AFC9E70C9A049CD2B1404A1A40B2F13C
:10A54000D46F15D8100D4FF0FF31C0F16B00814072
:10A550008C4227D0002D62D01D423FF406AFE4E6C6
:10A560004FF0FF3202FA03F3049A1A4004927DE49A
:10A57000621C12D0BCF1000F7FF408AF14EA0E0F7A
:10A580003FF407AFD1E602460B4630463946F9F7AD
:10A590009FF81A9D06460F46C8E4294A934234D0D4
:10A5A00001321A4002F58013059300230493DDE97C
:10A5B0000467EEE6214D1D40B5F1D66F3FF655AF6D
:10A5C000B5F15C7F3FF6D1AE22231A9D002600270D
:10A5D000CBF80030AAE4C2F14B024FF0FF339340B6
:10A5E0000B40059342E402460B4630463946F9F7E4
:10A5F00083F81A9C0022002306460F462546F9F7E9
:10A600006BF900283FF492ACC3E522231A9D002683
:10A610000A4FCBF8003089E402460B469FE614EA65
:10A620000E0F3FF4A2AE80E602460B4666E7A44654
:10A630000134D8E5002333E60000F03F0000F07F4E
:10A64000FFFFEF7F300A0110014BFFF731B800BF69
:10A65000480F00202DE9F04F82468E463F48754650
:10A660001EF801BB10F80B4014F00804F7D1BBF141
:10A670002D0F5BD0BBF12B0F6FF0004904BF9EF88C
:10A6800000B005F1020E33F0100010D1BBF1300F15
:10A6900004D0002B5ED10A231F4609E09EF800007B
:10A6A00000F0DF0058284ED0002B53D108231F465E
:10A6B0000025B9FBF7F6284607FB16980EE0ABF12C
:10A6C000370C63451DDD002D04DB864202D321D10A
:10A6D000E0451FDA4FF0FF351EF801BBABF1300C3F
:10A6E000BCF1090FEDD9ABF1410CBCF1190FE6D962
:10A6F000ABF1610CBCF1190F03D8ABF1570C6345FA
:10A70000E1DC6B1C0AD004B140420AB1CDB9116042
:10A71000BDE8F08F07FB00C00125DDE72223CAF862
:10A7200000305AB10EF1FF314846F0E79EF800B014
:10A730004FF0004905F1020E0124A4E74846BDE8A8
:10A74000F08F8146EEE710239EF801B00EF1020E65
:10A750001F46ADE710231F46AAE700BFD5D2001061
:10A76000242B03D8012B01D0FFF774BF10B5FCF7E1
:10A770007BFD16230360002010BD00BF034649B1D6
:10A78000FF2A02D801200A7070478A224FF0FF305A
:10A790001A607047084670472DE9F04F924685B021
:10A7A00089461E460D46554A0390294615F8014B29
:10A7B000135D13F00803F8D12D2C7CD02B2C4ED038
:10A7C0004FF0FF3102936FF00043CDE9001336F0F4
:10A7D000100851D037464FEAE6783A464346DDE95D
:10A7E000000101F0F9FB002383468E461846194606
:10A7F000A44613E0ACF13704A6421FDD002B09DBB1
:10A8000083457EEB010305D38E4508BF83453BD1CD
:10A81000A24239DA4FF0FF3315F801CBACF1300426
:10A82000092CE9D9ACF14104192CE3D9ACF161044C
:10A83000192C03D8ACF15704A642DFDC5A1C2FD0E8
:10A84000029A12B1404261EB4101BAF1000F03D00C
:10A85000002B48D1CAF8009005B0BDE8F08F4FF04A
:10A86000FF30029336F010086FF000432C7801F1AE
:10A870000205CDE90003ADD1302C25D0002E3AD110
:10A880000A27B0463E46A8E700FB08F307FB013362
:10A89000A0FB07010B44201843EBE4710123BBE745
:10A8A0002223039A1360BAF1000F17D005F1FF3984
:10A8B000DDE90001CEE74FF00047009301232C783B
:10A8C0008D1CCDE9017382E72B7803F0DF03582B51
:10A8D0000CD086B90827B0463E467EE7DDE9000188
:10A8E00005B0BDE8F08FCDE90001DFE710276C78F7
:10A8F00002353E4671E710273E466EE7D5D200107E
:10A90000FFF74ABF2DE9F04F85B08B461E460D4636
:10A9100001925D4A0390294615F8014B135D13F02F
:10A920000803F8D12D2C00F082802B2C51D00293FB
:10A9300036F0100A54D04FEAE67A32464FF0FF3034
:10A940004FF0FF315346B14601F046FB3246074611
:10A95000884653464FF0FF304FF0FF3101F03CFB8B
:10A96000944600221046114613E0A4F137039E429C
:10A970001FDD002A09DB874278EB010205D3414540
:10A9800008BFB8423BD1634539DD4FF0FF3215F8BF
:10A99000014BA4F13003092BE9D9A4F14103192B90
:10A9A000E3D9A4F16103192B03D8A4F157039E4204
:10A9B000DFDC531C30D0029B13B1404261EB4101FC
:10A9C000019B1BB182BB019BC3F800B005B0BDE881
:10A9D000F08F36F0100A2C78029301F10205AAD10B
:10A9E000302C29D0002E44D14FF00A09B2464FF046
:10A9F000050C4FF09937DFF894804E46B1E709FB1C
:10AA000001F100FB0A11A9FB0002114418184FF0D4
:10AA1000010241EBE371BAE72223039910460B6070
:10AA20001146019B002BD1D005F1FF3BCBE7012361
:10AA30002C788D1C02937BE72B7803F0DF03582BD7
:10AA40000BD0B6B94FF00809B2464FF0070C4FF0E3
:10AA5000FF376FF060484E4683E74FF010096C787F
:10AA60004FF00F0C02354FF0FF376FF070484E4635
:10AA700077E74FF010094FF00F0C4FF0FF376FF0F2
:10AA800070484E466DE700BFD5D2001099999919CC
:10AA9000FFF738BF70B582B00446069D55B1104827
:10AAA000D0F8E4606AB120460095B047431C10D04E
:10AAB00002B070BD00F1F4050948D0F8E460002A46
:10AAC000F1D1012311462046064A0095B047431CA8
:10AAD000EED100228A232A60236002B070BD00BF3D
:10AAE000480F002018C10010002100F001B800BF7D
:10AAF00010B500F0B7F8044601F036FAA0F11A03D9
:10AB0000DBB2022B01D8012010BDA4F109000428FA
:10AB10008CBF0020012010BD0229C0F307235FFA7B
:10AB200080FC25D0032903D083F080038CF0800CB7
:10AB300003F15002D2B21F2A0BD903F13002D2B274
:10AB4000242A3BD84FF2A64290422CD94FF0FF3036
:10AB500070474CF6D3729042F8D8B03BACF1A10CE0
:10AB6000384AC3EBC3130CEB430332F813007047AE
:10AB7000BCF19E0F11D90CF1230C80225FFA8CFCE2
:10AB80009F2B94BF703B503302EB4302D3B203F1CF
:10AB90005002D2B21F2AD0D8DBE7ACF17E0C7F2264
:10ABA0005FFA8CFCECE7D03BACF1A10C264AC3EB7E
:10ABB000C3130CEB430332F813007047A13B072B80
:10ABC000C4D8DFE803F0382E241D17120D04BCF1A1
:10ABD000C00FBBD81D4AACF1A10332F81300704777
:10ABE000BCF1F10FB2D81A4A1CE0BCF1D80FADD8B5
:10ABF000184A17E0BCF1F60FA8D80CF54050704782
:10AC0000BCF1F30FA2D842F6A07060447047124B1B
:10AC1000634413F8A13C002B98D04FF66060604469
:10AC200070470E4AACF1A10332F81300002808BFA8
:10AC30004FF0FF3070470A4AACF1A10332F813001D
:10AC4000704700BFCCEE001050D40010F805011082
:10AC500038060110DC0601104C070110A80701108E
:10AC60006408011038B50546B9B101F5957412496B
:10AC70002046FCF711FB28B928460121BDE83840E1
:10AC8000FFF74ABF0D492046FCF706FB38B92846B6
:10AC90000221BDE83840FFF73FBF094CE7E709490B
:10ACA0002046FCF7F9FA28B928460321BDE83840C8
:10ACB000FFF732BF284638BDB0C30010B4C3001040
:10ACC00072100020BCC3001000200149704700BF73
:10ACD0000000F87F2DE9F0410469B4EB611F05DC49
:10ACE0000023036100234361BDE8F08100F11405F6
:10ACF0004E1111F01F0C05EB840E05EB860321D0DD
:10AD0000043355F82610CCF120089E4521FA0CF1A9
:10AD10002DD92F461A6802FA08F20A4347F8042B85
:10AD200053F8041B9E4521FA0CF1F3D8A31B9B009A
:10AD3000053B9B08013305EB830445F8231071B1F3
:10AD400004340CE09E45CBD900F1100253F8041BEB
:10AD50009E4542F8041FF9D8A41B05EB8404631B2D
:10AD6000AC424FEAA3030361BCD0BDE8F08141616E
:10AD70000029B5D02C46E3E72DE9F04F8A4685B08F
:10AD8000096803938B78302BCDE9002040F0EE81E9
:10AD9000CA1C137814460132302BFAD0A4EB0109F7
:10ADA000A9F10209DFF8108318F80330002B00F036
:10ADB000D3802378002718F803303D46002B00F09D
:10ADC0006D81264616F8013F18F80330002BF9D1A3
:10ADD0000122B8493046FEF7C7FB8346002843D01E
:10ADE0003278002D00F0A381AB1B4FEA830B02F0F9
:10ADF000DF023546502A43D0CAF80060002F54D1F4
:10AE00002A1B3946013A072A03DD52100131072A6D
:10AE1000FBDC019800F078FB8246002800F06A8293
:10AE200000F11406A542029640F2CC810027B946F3
:10AE30000CE03A4604372B78AC4218F8033003F0A4
:10AE40000F0303FA02F349EA030940D015F8013D64
:10AE50002E2B01D1AC4231D9202FEAD1002246F865
:10AE6000049B04279146E6E7002D00F070813278BC
:10AE7000AB1B354602F0DF024FEA830B502ABBD1F1
:10AE80006A782B2A00F051812D2A40F0C5800120DC
:10AE9000AA78AE1C18F802104A1E182A40F2C48084
:10AEA0002E46CAF80060002FAAD0B9F1000F0CBFDF
:10AEB00006250025284605B0BDE8F08F01227D4912
:10AEC0002846FEF751FB0028C6D1AC42BED1029BFA
:10AED000484646F8049BF61AB610CAF81060760188
:10AEE00000F0ECFB009B361A1C68A64277DCC0F22F
:10AEF00020810027009B9A685A45C0F25881009B28
:10AF00005A685A454BDDA2EB0B0B5C4500F3A7805A
:10AF1000DB68022B00F0F980032B00F06A81012B23
:10AF200040F0F7805C4540F0F480012C08D0611EB1
:10AF3000504600F0EBFF002800F0EB80009B5A68C1
:10AF40000399012362250A60029ACAF8103013603F
:10AF50000E9BC3F800A0ADE7012256492046FEF73C
:10AF600003FB0746002840F09B806378651C18F8B7
:10AF70000320002A00F09680302B2C4640F04481BC
:10AF800014F8013F302BFBD018F803304FF00109C3
:10AF9000B3FA83F77F09002B7FF413AF7EE001251E
:10AFA0009FB1009BDA68022A00F08880032A00F033
:10AFB0008980012A07D1B90705D5029B1A68174372
:10AFC000FA0700F1838045F010050E9B2846C3F870
:10AFD00000A0039BC3F800B005B0BDE8F08F361B9E
:10AFE0005046314600F092FF074678B1711E029B31
:10AFF00001274A1153F8220001F01F0207FA02F25A
:10B00000024203D0B94200F3E7800227314650469E
:10B01000B344FFF75FFE6DE718F802106E1C0020C6
:10B020004A1E182A3FF63CAF72781039013618F8DC
:10B03000022002F1FF3CBCF1180F0CD801EB81019A
:10B0400016F8013F02EB4102A2F1100118F80320AB
:10B05000531E182BF2D900B149428B44CCE60BF1B8
:10B06000FF36002F40F0AC80002E40F0AF8073110F
:10B07000029A06F01F06594652F823200123504633
:10B08000A4EB0B04B3400225134218BF47F002079C
:10B09000FFF720FE009BD3F804B081E7264697E631
:10B0A0002378254603F0DF03502B00F09E80CAF87A
:10B0B0000050FAE658C30010200901100F9BC3F19D
:10B0C00001030F930F9B002B3FF47DAF029B0026E3
:10B0D000DAF8107098461A464FEA870903EB8700A2
:10B0E00003E0904242F8046C44D9944652F8041BA1
:10B0F0004B1CF6D00131022DCCF800107DD014F09D
:10B100001F0440F0AB8021255FE70F9B002B3FF42D
:10B1100017AF50250198514600F01CFA00230E9AF3
:10B120002846136005B0BDE8F08F0020B0E6AB46BE
:10B130005DE6A61B5146019800273246ABEB060B95
:10B1400000F04AFC00F1140382460293D2E67278C2
:10B15000751C18F802102E4600293FF448AE16F868
:10B16000012F18F80230002BF9D13DE68C1C4FF06E
:10B17000000917E6DAF80820974248DA7A1C01211C
:10B180000AEB8707022DCAF81020DDF808807961E4
:10B1900033D0002A6FDC0022CAF810200022CAF83F
:10B1A0001420009B0BF1010B9A685A45ABDA51460B
:10B1B000019800F0CFF900230E9AA325136079E6D9
:10B1C000012754E7029E4FF0000980E631465046C1
:10B1D00000F09CFE07464AE7B11E504600F096FE7E
:10B1E00000283FF412AF032710E74FF0000B0127B0
:10B1F00046E60F9B002B8CD0A2E6009B1A68013A12
:10B20000A24263D02225E0E64FF00109D9E5DAF841
:10B2100004100198013100F077F9064600286FD03C
:10B22000DAF810200AF10C010C3006F11408023291
:10B230009200FCF70FF951460198B24600F08AF9E6
:10B2400031690120022D01EB000206EB8101326120
:10B250004861D2D09742BFF652AF9AE7C144C4F1D9
:10B26000200459F8040C00F029FAA042BFF64BAFB5
:10B27000DAF810208DE708EB82000AF11804DAF8FA
:10B280001420A0424FEA52022CD94546236842EAD4
:10B29000C37245F8042B54F8042BA0424FEA520223
:10B2A000F4D8A0EB0A0119398908013148F82120A6
:10B2B00008EB810102B10431A1EB080241454FEADC
:10B2C000A202CAF810207FF46CAF67E7621104F0A5
:10B2D0001F0458F822100122A2400A4214BF21255F
:10B2E000222572E6C8F800200AB14146E3E7CAF811
:10B2F000102053E70246054BE4210548FAF704FC09
:10B300000246024B84210248FAF7FEFBC4C3001038
:10B31000D8C3001010B504688646013409E014F85B
:10B32000013BA3F1410CBCF1190F98BF20339342AC
:10B3300007D111F8012B002AF1D10120CEF80040ED
:10B3400010BD002010BD00BF09682DE9F04F4B1162
:10B3500085B011F01F01044602EB8303029140F017
:10B360009A80181F19462568002641F8046C01359B
:10B370002B78002B00F0A780B44601910646864644
:10B38000DFF88081E1466746E346AA46014603941A
:10B3900018F8030000285CD1202B00F28E804F4566
:10B3A00020DD76451AD9BCF1070F17DCCCF1080473
:10B3B000DEF800307046CDF800E0A400C4F1200CA7
:10B3C000A646446804FA0CF51D4324FA0EF3056002
:10B3D00040F8043F8642F4D8DDF800E0724551D3CE
:10B3E0004FF0080C1AF8013F002BD1D10846019903
:10B3F000002F68D0B64502D2BCF1070F67DD724559
:10B400004CD2141F734653F8045B834244F8045F24
:10B41000F9D9A0EB0E03441C0EF1010E23F0030337
:10B420000433A64588BF04230024134443F8044B87
:10B430008342FBD951F8044C1CB106E050F8043D9E
:10B440001BB98242FAD101230360052005B0BDE893
:10B45000F08F0CF1010C0137BCF1080F08DCDEF8AD
:10B4600000301B0100F00F001843CEF80000B9E7D0
:10B470007245B7D24EF804BC0023AEF1040E4FF073
:10B48000010CEFE7AEF104064EF804BCB9464FF0EC
:10B49000000CB646A6E7191D184664E7029B51F852
:10B4A000044C002BC8D0C3F120034FF0FF3525FA20
:10B4B00003F31C4041F8044CBEE7292B08465546CF
:10B4C0000199039C1BD0042005B0BDE8F08FCCF19E
:10B4D0000803DEF8004077469B002546C3F12008AC
:10B4E0009C467B6803FA08F42C4323FA0CF53C6075
:10B4F00047F8045FBE42F4D8724582D3CEE70135E7
:10B50000256075E72009011038B5436C05460C46E7
:10B510004BB153F8240080B1026843F82420002383
:10B52000C0E9033338BD21220421FBF77DF803462F
:10B5300068640028EDD1002038BD0121284601FAB9
:10B5400004F56A1D9200FBF76FF80028F3D0C0E9FC
:10B550000145E4E731B1436C4A6853F822000860C2
:10B5600043F82210704700BF2DE9F04107460E4610
:10B570001C460D6901F1140E0020DEF800100130A8
:10B580008BB285424FEA114102FB03434FEA134C51
:10B590009BB202FB01CC03EB0C434FEA1C444EF878
:10B5A000043BEADC3CB1B368AB4207DD06EB850344
:10B5B00001355C6135613046BDE8F081716838461F
:10B5C0000131FFF7A1FF8046A8B1326906F10C01F5
:10B5D0000C3002329200FBF73DFF7B6C726853F82F
:10B5E0002210316043F82260464606EB85030135A0
:10B5F0005C613561DFE70246024BBA210248FAF787
:10B6000083FA00BFC4C300103CC400102DE9F84306
:10B610001E4617460833264A0C46092E82FB0312A3
:10B620004FEAE3730546C3EB620338DD4FF0010CCC
:10B6300000214FEA4C0C01316345FADC2846FFF744
:10B6400063FF014668B3089B092F43614FF0010374
:10B65000036112DC0A340927BE420BDDF61B2644C7
:10B6600014F8013B0A222846303BFFF77DFFB44225
:10B670000146F5D10846BDE8F88304F109093C44C8
:10B68000C84618F8013B0A222846303BFFF76CFFFA
:10B69000A0450146F5D1A7F108044C44DCE70021A0
:10B6A000CCE70246034BD3210348FAF72DFA00BF3B
:10B6B000398EE338C4C300103CC40010B0F5803F9D
:10B6C000034618D203041020B3F1807F01D2083062
:10B6D0001B02B3F1805F01D204301B01B3F1804F34
:10B6E00003D3002B06DB013070479B0005D45B00C1
:10B6F00005D4202070470020E6E702307047033071
:10B70000704700BF0368014613F0070207D0DA074D
:10B710001FD4980721D55B0801200B60704798B2B1
:10B72000A0B11046DAB20AB908301B0A1A0701D1D3
:10B7300004301B099A0701D102309B08DA0703D4B1
:10B740005B0800F1010006D00B6070471B0C102055
:10B75000E8E700207047202070479B0802200B601C
:10B76000704700BF38B5436C04460D464BB158686E
:10B77000B0B102685A60002201234561C0E9032389
:10B7800038BD21220421FAF74FFF034660640028E8
:10B79000EDD1094B002240F245110848FAF7B4F9FF
:10B7A0001C2201212046FAF73FFF0028F1D0012298
:10B7B0000223C0E90123DEE7C4C300103CC400102B
:10B7C0002DE9F04FD1F8108085B015690E469246EC
:10B7D000A84505DB2A46534645468A4690461E46FE
:10B7E00005EB0804DAE90113A342B8BF0131FFF702
:10B7F0008BFE002800F08B8000F1140707EB840E0D
:10B80000774505D23B46002243F8042B9E45FBD8E2
:10B8100014360AF1140906EB880809EB850546453C
:10B8200068D2A5EB0A030AF1150ACDF808E0AE4686
:10B83000153B039423F00303043355452CBF9B466B
:10B840004FF0040B824605E0090C2CD1B04507F1FE
:10B8500004074CD956F8041B8DB2002DF4D0CC4609
:10B860003C46002301965CF8040B216886B2E6454D
:10B870008AB24FEA104005FB06224FEA11411A44F2
:10B8800005FB001101EB124192B24FEA114342EA6B
:10B89000014244F8042BE6D8019E47F80B3056F8D5
:10B8A000041C090CD2D03B68002248463D461C4689
:10B8B000944602889BB201FB02C202EB144243EAA7
:10B8C000024345F8043B50F8043B2C684FEA134C04
:10B8D0007045A3B201FB0C3303EB12434FEA134C48
:10B8E000E7D3B04547F80B3007F10407B2D850460C
:10B8F000DDE902E4002C02DC05E0013C03D05EF847
:10B90000043D002BF9D0046105B0BDE8F08F02467C
:10B91000024B4FF4B1710248FAF7F6F8C4C30010B5
:10B920003CC4001012F003032DE9F0411446074611
:10B930002CD10D46A4101CD03E6C86B3E3074FF00B
:10B94000000806D4641014D03068A8B10646E30796
:10B95000F8D5324629463846FFF732FF35B17B6CC1
:10B96000696853F821202A6043F821506410054685
:10B97000EAD12846BDE8F081324631463846FFF725
:10B980001FFF30600646C0F80080E0E7013B0F4A29
:10B9900052F823200023FFF7E7FD0546CAE70121FF
:10B9A0003846FFF7B1FD064640B1012340F271224F
:10B9B000C0E90432002338640360BFE70246044B49
:10B9C00040F245110348FAF79FF800BF200A011022
:10B9D000C4C300103CC400102DE9F0470C4690464B
:10B9E00006464FEA62192769A36807EB62174968A0
:10B9F0007D1C9D4203DD5B0001319D42FBDC304636
:10BA0000FFF782FD002850D0B9F1000F00F1140CAF
:10BA10000EDD09F10502634600214FEA820E00EBBC
:10BA2000820243F8041B9342FBD1AEF114039C4401
:10BA300004F11403216918F01F0803EB81012BD0D6
:10BA4000C8F12009E6464FF0000A1A6802FA08F227
:10BA500042EA0A024EF8042B53F8042B994222FAC8
:10BA600009FAF2D80B1B04F11502153B23F003036E
:10BA70000433914238BF04234CF803A0BAF1000FFD
:10BA800000D13D46736C6268056153F82210216055
:10BA900043F82240BDE8F087ACF1040C53F8042BC6
:10BAA00099424CF8042FF9D8EBE70246024B4FF4C9
:10BAB000EF710248FAF728F8C4C300103CC4001024
:10BAC00084460B690069C01A16D10CF1140C1431AC
:10BAD0000CEB830201EB830310B401E0944508D220
:10BAE00052F8044D53F8041D8C42F7D005D24FF0A4
:10BAF000FF305DF8044B7047704701205DF8044B40
:10BB0000704700BF2DE9F04F15460A6983B088469B
:10BB10002B69D21A002A40F08B8001F1140605F13E
:10BB2000140101EB830106EB830302E09E4280F0E7
:10BB3000828053F8044D51F8042D9442F6D078D306
:10BB40002B460024454698466968FFF7DDFC00282F
:10BB500000F08C802E6905F1140B08F1140ED8F852
:10BB6000103000F1140A05F110020EEB83094FF0BA
:10BB7000000C0BEB86015746C460CDF804B05EF8AC
:10BB8000044B52F8045F1FFA84FBF145ABB24FEA55
:10BB90001444A3EB0B03C4EB1544634404EB2344AC
:10BBA0009BB24FEA244C43EA044347F8043BE6D8EF
:10BBB000A9EB080408F11508DDF804B0C145A4F1AB
:10BBC000150434BF4FF000084FF00108A408B8F185
:10BBD000000F04F101024FEA820208BF04220BEBBE
:10BBE00002055244A94231D917462C4654F8043B69
:10BBF0001FFA83F8A1424FEA134E6344C4449BB238
:10BC00000EEB2C4C43EA0C434FEA2C4C47F8043B18
:10BC1000ECD80139491B21F003010A4423B952F839
:10BC2000043D013E002BFAD0066103B0BDE8F08F61
:10BC300086DA012488E70021FFF766FC78B101224B
:10BC40000023C0E9042303B0BDE8F08FB8F1000F72
:10BC50004FEA840408BF00240AEB0402DEE7024630
:10BC6000064B40F237210648F9F74EFF0246034BD8
:10BC700040F245210248F9F747FF00BFC4C3001056
:10BC80003CC40010114B0B40A3F15073002B03DD9B
:10BC900000221946104670475B42B3F1A07F4FEA7D
:10BCA000235106DA4FF4002300220B4110461946B7
:10BCB000704714391E2904DD01220023104619465D
:10BCC00070474FF00042CA40F7E700BF0000F07F26
:10BCD0002DE9F041026900F1140707EB820252F8E6
:10BCE000046CA2F104083046FFF7E8FCC0F1200321
:10BCF0000A280B6035DD4745A0F10B011BD252F835
:10BD0000083C31B3C1F1200C8E40A2F1080023FAA7
:10BD10000CF48B40874246EA040646F07F5545F412
:10BD200040151AD252F80C2C294622FA0CF2134371
:10BD30001846BDE8F0810B280AD006FA01F100236D
:10BD400041F07F55184645F440152946BDE8F0817D
:10BD5000002346F07F5545F4401518462946BDE8B6
:10BD6000F081C0F10B03474526FA03F141F07F55FE
:10BD700045F4401509D3002200F11503294606FABF
:10BD800003F313431846BDE8F08152F8082CDA405B
:10BD9000F2E700BFF0B5012183B016461F46FFF75A
:10BDA000B3FB0546002849D0C7F30A54C7F3130371
:10BDB0000CB143F48013002E019315D101A8FFF7B5
:10BDC000A1FC0199012200F1200369612A611CB3E1
:10BDD000A4F23344C3F135001C44089B1C60099B4A
:10BDE0001860284603B0F0BD68460096FFF78AFC4D
:10BDF000019A034600B3C0F1200102FA01F1C240EA
:10BE0000009801920143002AC5E905120CBF0122E6
:10BE100002222A61002CDBD1A3F23243089805EB01
:10BE2000820103600869FFF749FC099BC0EB4210DF
:10BE30001860284603B0F0BD0099E4E70246034BC2
:10BE400040F20F310248F9F75FFE00BFC4C3001093
:10BE50003CC400102DE9F04383B088468146694612
:10BE6000FFF736FF04460D46404601A9FFF730FFB5
:10BE7000D9F81030D8F81020A3EB020CDDE900321D
:10BE80009B1A03EB4C13002B0BDD05EB03573D46D0
:10BE900002460B4620462946F7F768FC03B0BDE88A
:10BEA000F083C3EB033301EB03594946F0E700BFCE
:10BEB000013902F114034FEA611C116903EB81019E
:10BEC0000CF1010C8B4200EB8C0C16D210B5A0F1DA
:10BED000040E53F8044B99424EF8044FF9D88B1ACC
:10BEE000153B23F0030304331844844504D900238D
:10BEF00040F8043B8445FBD810BD844505D9002398
:10BF000040F8043B8445FBD87047704703694A11E9
:10BF10001430934209DA00EB830302E053F8042D56
:10BF2000AAB98342FAD80020704700EB8203F8DDFB
:10BF300011F01F01F5D010B450F8224024FA01F29C
:10BF40008A40944209D001205DF8044B70470120DB
:10BF5000704753F8042D002AF5D18342F9D8002008
:10BF60005DF8044B704700BF154B984226D840F649
:10BF7000F90C70B54FF0000E124D03E004F1010E04
:10BF8000F44519DB1CEB0E0248BF013222F001031D
:10BF9000541003EB620305EB43015B004A784E88C3
:10BFA000898842EA062211448842E7D8904204F187
:10BFB000FF3CE5D3E85C70BDFF2070BDFF207047FB
:10BFC000EF010E00200B0110F8B500BF00000000CB
:10BFD0005FF800F0710500205FF800F021060020F6
:10BFE0005FF800F06D0200205FF800F01101002002
:10BFF0005FF800F00102002065350010D934001010
:10C000000D350010B13500104535001041340010D9
:10C010008D3500102D3400102529001091350010A9
:10C02000912C00108934001079350010293500104A
:10C030003D2500107525001019020010396100100F
:10C040004646542F69464654000000005261737002
:10C050006265727279205069205069636F323A20AC
:10C0600065636534373630004272756365204C6114
:10C070006E643A2042524C3440636F726E656C6C51
:10C080002E6564750000000048756E74657220416D
:10C0900064616D733A5648413340636F726E656CEC
:10C0A0006C2E65647500000050726F746F74687256
:10C0B00065616473207270323335302076312E33EF
:10C0C00000000000313620636F6C6F7220564741CC
:10C0D00000000000316B0000326B0000336B000089
:10C0E000346B0000696E707574207265636F7264E2
:10C0F00020706C61796261636B3A200025642025B1
:10C10000640000000A0A436F6D70696C65642070FA
:10C11000726F6772616D3A20000000002F0000000E
:10C12000557365727300000057696E646F777320F2
:10C1300055736572206E616D653A2000436F6D70B6
:10C14000696C652074696D652F646174653A2000BF
:10C150004A616E20313120323032350031303A358B
:10C16000353A3235000000002573202025730A007F
:10C1700050726F746F746872656164733A205250C4
:10C18000323335302076312E332074776F2D636F44
:10C1900072652C207072696F7269747900000000FA
:10C1A0004170706C69636174696F6E3A2025730A1F
:10C1B0000A000000433A2F55736572732F313630F1
:10C1C00037332F4F6E6544726976652F446F637500
:10C1D0006D656E74732F5069636F2D76322E302F1C
:10C1E00076676131365F6666742F76676131365FD8
:10C1F0006666745F696666742E6300004646542F57
:10C200006946465420746573740000000A2A2A2A7D
:10C210002050414E4943202A2A2A0A00486172646C
:10C220007761726520616C61726D20256420616C9C
:10C23000726561647920636C61696D6564000000FA
:10C240004861726420617373657274004F75742065
:10C250006F66206D656D6F727900000052656C65C8
:10C2600061736500626F6F74325F77323571303899
:10C2700030000000322E312E300000007069636FF4
:10C280003200000067726170686963735F74657380
:10C2900074000000666E692B00000000666E690085
:10C2A0006E616E00666E692D000000002C206675C0
:10C2B0006E6374696F6E3A200000000061737365ED
:10C2C0007274696F6E2022257322206661696C6525
:10C2D000643A2066696C6520222573222C206C69E3
:10C2E0006E65202564257325730A0000554152545C
:10C2F00020737464696E0000554152542073746455
:10C300006F7574005541525420737464696E202F08
:10C31000207374646F757400646F75626C6520724D
:10C3200065736574202D3E20424F4F5453454C0099
:10C330004E6F20444D41206368616E6E656C7320C2
:10C3400061726520617661696C61626C65000000F4
:10C3500065256C64000000002E0000004C435F4324
:10C360004F4C4C41544500004C435F435459504599
:10C37000000000004C435F4D4F4E45544152590060
:10C380004C435F4E554D4552494300004C435F546A
:10C39000494D45004C435F4D45535341474553007C
:10C3A0006E660000696E697479000000616E0000BD
:10C3B0004A495300534A4953000000004555434A37
:10C3C0005000000042616C6C6F632073756363659D
:10C3D00065646564000000002F646174612F6A6504
:10C3E0006E6B696E732F776F726B73706163652FFD
:10C3F000474E552D746F6F6C636861696E2F617263
:10C400006D2D31332F7372632F6E65776C69622DDA
:10C4100063796777696E2F6E65776C69622F6C69D7
:10C4200062632F7374646C69622F6764746F612D2B
:10C430006765746865782E63000000002F6461747E
:10C44000612F6A656E6B696E732F776F726B737095
:10C450006163652F474E552D746F6F6C636861691A
:10C460006E2F61726D2D31332F7372632F6E65776E
:10C470006C69622D63796777696E2F6E65776C6979
:10C48000622F6C6962632F7374646C69622F6D70C4
:10C490007265632E630000000000010002000300CB
:10C4A0000B000F000F000000000000000000000063
:10C4B0000000000000000000FFFF0000000000007E
:10C4C000000000000000000000000000000000FF6D
:10C4D000FF00000000000000C0C0C0C0C0C0C0C05D
:10C4E000C0C0C0C0C0C0C0C018181818181818188C
:10C4F0001818181818181818C0C0C0C0C0C0C0C07C
:10C50000000000000000000000000000000000002B
:10C51000C0C0C0C0C0C0C0C000000000000000F823
:10C52000F818181818181818000000000000001F4C
:10C530001F18181818181818181818181818181F6D
:10C540001F0000000000000018181818181818F82C
:10C55000F80000000000000018181818181818FF3C
:10C56000FF1818181818181818181818181818FF7D
:10C57000FF0000000000000000000000000000FFBD
:10C58000FF1818181818181818181818181818F864
:10C59000F818181818181818181818181818181F34
:10C5A0001F181818181818180080C0E0F0F8FEF8C6
:10C5B000F0E0C080000000000002060E1E3EFE3EBD
:10C5C0001E0E0602000000000000183C7E1818181D
:10C5D0007E3C180000000000000066666666666625
:10C5E000660066660000000000007FDBDBDB7B1B73
:10C5F0001B1B1B1B00000000007CC660386CC6C6FD
:10C600006C380CC67C000000000000000000000038
:10C61000FEFEFEFE000000000000183C7E18181808
:10C620007E3C1800000000000000183C7E1818181E
:10C63000181818180000000000001818181818180A
:10C64000187E3C18000000000000000000180CFEDE
:10C65000FE0C18000000000000000000003060FE2A
:10C660007E30180000000000000000000000C0C084
:10C67000C0FE00000000000000000000002466FF73
:10C680006624000000000000000000001038387C24
:10C690007CFEFE000000000000000000FEFE7C7C2E
:10C6A000383810000000000000000000000000000A
:10C6B00000000000000000000000183C3C3C18187E
:10C6C00018001818000000000066666624000000CC
:10C6D00000000000000000000000006C6CFE6C6CAC
:10C6E0006CFE6C6C0000000018187CC6C2C07C0692
:10C6F0000686C67C1818000000000000C2C60C1890
:10C700003060C686000000000000386C6C3876DCB3
:10C71000CCCCCC760000000000303030600000004F
:10C72000000000000000000000000C183030303025
:10C730003030180C00000000000030180C0C0C0CFD
:10C740000C0C1830000000000000000000663CFFE8
:10C750003C66000000000000000000000018187E89
:10C760001818000000000000000000000000000099
:10C770000018181830000000000000000000007EC3
:10C7800000000000000000000000000000000000A9
:10C7900000001818000000000000000002060C183D
:10C7A0003060C0800000000000007CC6C6CEDEF60F
:10C7B000E6C6C67C0000000000001838781818187B
:10C7C0001818187E0000000000007CC6060C183007
:10C7D00060C0C6FE0000000000007CC606063C06E5
:10C7E0000606C67C0000000000000C1C3C6CCCFE61
:10C7F0000C0C0C1E000000000000FEC0C0C0FC06B7
:10C800000606C67C0000000000003860C0C0FCC600
:10C81000C6C6C67C000000000000FEC606060C1856
:10C82000303030300000000000007CC6C6C67CC638
:10C83000C6C6C67C0000000000007CC6C6C67E06D8
:10C8400006060C7800000000000000001818000028
:10C850000018180000000000000000001818000078
:10C860000018183000000000000000060C183060AE
:10C8700030180C060000000000000000007E0000E0
:10C880007E000000000000000000006030180C0670
:10C890000C1830600000000000007CC6C60C1818A0
:10C8A000180018180000000000007CC6C6C6DEDEB6
:10C8B000DEDCC07C00000000000010386CC6C6FE44
:10C8C000C6C6C6C6000000000000FC6666667C6640
:10C8D000666666FC0000000000003C66C2C0C0C086
:10C8E000C0C2663C000000000000F86C6666666628
:10C8F00066666CF8000000000000FE6662687868FA
:10C90000606266FE000000000000FE6662687868F3
:10C91000606060F00000000000003C66C2C0C0DE45
:10C92000C6C6663A000000000000C6C6C6C6FEC6FF
:10C93000C6C6C6C60000000000003C18181818182B
:10C940001818183C0000000000001E0C0C0C0C0C09
:10C95000CCCCCC78000000000000E666666C7878ED
:10C960006C6666E6000000000000F06060606060D9
:10C97000606266FE000000000000C3E7FFFFDBC34B
:10C98000C3C3C3C3000000000000C6E6F6FEDECE4F
:10C99000C6C6C6C60000000000007CC6C6C6C6C625
:10C9A000C6C6C67C000000000000FC6666667C60AF
:10C9B000606060F00000000000007CC6C6C6C6C60D
:10C9C000C6D6DE7C0C0E00000000FC6666667C6C41
:10C9D000666666E60000000000007CC6C660380C93
:10C9E00006C6C67C000000000000FFDB991818187E
:10C9F0001818183C000000000000C6C6C6C6C6C60F
:10CA0000C6C6C67C000000000000C3C3C3C3C3C3C6
:10CA1000C3663C18000000000000C3C3C3C3C3DBEF
:10CA2000DBFF6666000000000000C3C3663C181808
:10CA30003C66C3C3000000000000C3C3C3663C18CB
:10CA40001818183C000000000000FFC3860C1830C6
:10CA500060C1C3FF0000000000003C3030303030C7
:10CA60003030303C0000000000000080C0E0703832
:10CA70001C0E06020000000000003C0C0C0C0C0C0C
:10CA80000C0C0C3C0000000010386CC600000000CC
:10CA90000000000000000000000000000000000096
:10CAA0000000000000FF000030301800000000000F
:10CAB00000000000000000000000000000780C7C76
:10CAC000CCCCCC76000000000000E06060786C66A2
:10CAD0006666667C0000000000000000007CC6C0A6
:10CAE000C0C0C67C0000000000001C0C0C3C6CCCDC
:10CAF000CCCCCC760000000000000000007CC6FE1C
:10CB0000C0C0C67C000000000000386C6460F060AB
:10CB1000606060F000000000000000000076CCCCF7
:10CB2000CCCCCC7C0CCC78000000E060606C7666ED
:10CB3000666666E600000000000018180038181845
:10CB40001818183C0000000000000606000E06063B
:10CB50000606060666663C000000E06060666C78CB
:10CB6000786C66E6000000000000381818181818E5
:10CB70001818183C000000000000000000E6FFDB71
:10CB8000DBDBDBDB000000000000000000DC666691
:10CB9000666666660000000000000000007CC6C6F5
:10CBA000C6C6C67C000000000000000000DC66660F
:10CBB0006666667C6060F000000000000076CCCC09
:10CBC000CCCCCC7C0C0C1E000000000000DC766697
:10CBD000606060F00000000000000000007CC660A3
:10CBE000380CC67C000000000000103030FC3030F3
:10CBF0003030361C000000000000000000CCCCCC1F
:10CC0000CCCCCC76000000000000000000C3C3C301
:10CC1000C3663C18000000000000000000C3C3C34E
:10CC2000DBDBFF66000000000000000000C3663C84
:10CC3000183C66C3000000000000000000C6C6C625
:10CC4000C6C6C67E060CF8000000000000FECC1828
:10CC50003060C6FE0000000000000E1818187018A2
:10CC60001818180E000000000000181818181818DE
:10CC700018181818000000000000701818180E1876
:10CC80001818187000000000000076DC000000009A
:10CC900000000000000000000000000010386CC61A
:10CCA000C6C6FE000000000000000000003E5B4F12
:10CCB0005B3E3E6B4F6B3E1C3E7C3E1C183C7E3CFC
:10CCC000181C577D571C1C5E7F5E1C00183C18000A
:10CCD000FFE7C3E7FF0018241800FFE7DBE7FF309A
:10CCE000483A060E2629792926407F050507407F08
:10CCF00005253F5A3CE73C5A7F3E1C1C08081C1C7B
:10CD00003E7F14227F22145F5F005F5F06097F0170
:10CD10007F006689956A606060606094A2FFA2945B
:10CD200008047E040810207E201008082A1C080829
:10CD30001C2A08081E101010100C1E0C1E0C303877
:10CD40003E3830060E3E0E06000000000000005F78
:10CD500000000007000700147F147F14242A7F2A94
:10CD60001223130864623649562050000807030056
:10CD7000001C2241000041221C002A1C7F1C2A08A2
:10CD8000083E080800807030000808080808000005
:10CD900060600020100804023E5149453E00427F79
:10CDA000400072494949462141494D331814127FC8
:10CDB0001027454545393C4A494931412111090768
:10CDC0003649494936464949291E000014000000E9
:10CDD00040340000000814224114141414140041BB
:10CDE00022140802015909063E415D594E7C121178
:10CDF000127C7F494949363E414141227F414141B0
:10CE00003E7F494949417F090909013E414151732A
:10CE10007F0808087F00417F41002040413F017F9B
:10CE2000081422417F404040407F021C027F7F0463
:10CE300008107F3E4141413E7F090909063E4151AC
:10CE4000215E7F09192946264949493203017F019C
:10CE5000033F4040403F1F2040201F3F4038403F9D
:10CE6000631408146303047804036159494D4300B3
:10CE70007F4141410204081020004141417F0402EA
:10CE80000102044040404040000307080020545481
:10CE900078407F284444383844444428384444285F
:10CEA0007F385454541800087E090218A4A49C78B2
:10CEB0007F0804047800447D40002040403D007F0E
:10CEC0001028440000417F40007C047804787C08EE
:10CED0000404783844444438FC18242418182424C2
:10CEE00018FC7C08040408485454542404043F44A7
:10CEF000243C4040207C1C2040201C3C4030403CD6
:10CF000044281028444C9090907C4464544C440035
:10CF10000836410000007700000041360800020199
:10CF20000204023C2623263C1EA1A161123A404085
:10CF3000207A385454555921555579412154547803
:10CF400041215554784020545579400C1E5272129C
:10CF50003955555559395454545939555454580024
:10CF600000457C410002457D420001457C40F0299E
:10CF70002429F0F0282528F07C54554500205454ED
:10CF80007C547C0A097F4932494949323248484831
:10CF900032324A4848303A4141217A3A4240207878
:10CFA000009DA0A07D39444444393D4040403D3C73
:10CFB00024FF2424487E4943662B2FFC2F2BFF0996
:10CFC00029F620C0887E090320545479410000448A
:10CFD0007D413048484A32384040227A007A0A0A75
:10CFE000727D0D19317D2629292F282629292926E8
:10CFF00030484D4020380808080808080808382F2D
:10D0000010C8ACBA2F102834FA00007B00000814B6
:10D010002A142222142A1408AA005500AAAA55AAE2
:10D0200055AA000000FF00101010FF00141414FF98
:10D03000001010FF00FF1010F010F0141414FC008A
:10D040001414F700FF0000FF00FF1414F404FC1494
:10D050001417101F10101F101F1414141F0010108D
:10D0600010F0000000001F101010101F1010101002
:10D07000F010000000FF101010101010101010FF22
:10D0800010000000FF140000FF00FF00001F101739
:10D090000000FC04F414141710171414F404F40022
:10D0A00000FF00F714141414141414F700F71414E8
:10D0B00014171410101F101F141414F4141010F06F
:10D0C00010F000001F101F0000001F14000000FCE3
:10D0D000140000F010F01010FF10FF141414FF14CF
:10D0E0001010101F00000000F010FFFFFFFFFFF006
:10D0F000F0F0F0F0FFFFFF0000000000FFFF0F0F57
:10D100000F0F0F38444438447C2A2A3E147E020212
:10D110000606027E027E0263554941633844443C60
:10D1200004407E201E2006027E020299A5E7A599F2
:10D130001C2A492A1C4C7201724C304A4D4D303029
:10D1400048784830BC625A463D3E494949007E0114
:10D1500001017E2A2A2A2A2A44445F444440514A33
:10D16000444040444A51400000FF0103E080FF007A
:10D170000008086B6B083612362436060F090F06B6
:10D18000000018180000001010003040FF010100DE
:10D190001F01011E00191D1712003C3C3C3C000001
:10D1A00000000000ACD1001009FF0100A08047A0E2
:10D1B00000E022A0C123A0800464046245000000B6
:10D1C000C8D100100EFF0100A08027A0C02001C020
:10D1D000420049E0C020860000E0C020C0205FE09F
:10D1E000C0388C00ECD1001009FF0100A08027A0FE
:10D1F000420000FF00FF00FF01FF01EC00C1000042
:10D2000006005250D3F075425CC200100600525026
:10D21000E182887F64C2001006005250ABB36053B5
:10D2200074C2001006005250BBFF3CB67CC2001016
:10D2300006005250861C030284C2001006005250A1
:10D240005422A29D50C1001005005250DE65F468C2
:10D25000F850011000000000000000000000F03F46
:10D2600000000000000024400000000000005940C1
:10D270000000000000408F40000000000088C34014
:10D2800000000000006AF8400000000080842E4189
:10D2900000000000D01263410000000084D79741D5
:10D2A0000000000065CDCD410D0A0000060052507F
:10D2B00053B4F4A104C3001008005250120000003F
:10D2C00008005250921000000600525053B4F4A1CE
:10D2D00018C30010002020202020202020202828F3
:10D2E0002828282020202020202020202020202026
:10D2F0002020202020881010101010101010101066
:10D300001010101010040404040404040404041095
:10D310001010101010104141414141410101010123
:10D3200001010101010101010101010101010101ED
:10D3300010101010101042424242424202020202F9
:10D3400002020202020202020202020202020202BD
:10D35000101010102000000000000000000000006D
:10D3600000000000000000000000000000000000BD
:10D3700000000000000000000000000000000000AD
:10D38000000000000000000000000000000000009D
:10D39000000000000000000000000000000000008D
:10D3A000000000000000000000000000000000007D
:10D3B000000000000000000000000000000000006D
:10D3C000000000000000000000000000000000005D
:10D3D00000000000000000000A000100020003003D
:10D3E0000400050006000700080009000A000B0001
:10D3F0000C000D000E000F001000000034000000B3
:10D40000CEFBFFFFCB030000010000000000000086
:10D4100035000000CEFBFFFFCB0300000100000041
:10D420000000000000000000BC89D897B2D29C3CEC
:10D4300033A7A8D523F649393DA7F444FD0FA532FB
:10D440009D978CCF08BA5B25436FAC6428066811A2
:10D450000C5F104E154E2A4E314E364E3C4E3F4E0E
:10D46000424E564E584E824E854E6B8C8A4E1282DC
:10D470000D5F8E4E9E4E9F4EA04EA24EB04EB34EAE
:10D48000B64ECE4ECD4EC44EC64EC24ED74EDE4EDA
:10D49000ED4EDF4EF74E094F5A4F304F5B4F5D4F09
:10D4A000574F474F764F884F8F4F984F7B4F694F5D
:10D4B000704F914F6F4F864F964F1851D44FDF4F9B
:10D4C000CE4FD84FDB4FD14FDA4FD04FE44FE54F1F
:10D4D0001A50285014502A50255005501C4FF64F12
:10D4E000215029502C50FE4FEF4F11500650435001
:10D4F000475003675550505048505A5056506C5042
:10D50000785080509A508550B450B250C950CA508B
:10D51000B350C250D650DE50E550ED50E350EE50BF
:10D52000F950F5500951015102511651155114513C
:10D530001A5121513A5137513C513B513F514051C1
:10D5400052514C5154516251F87A69516A516E519D
:10D5500080518251D8568C5189518F51915193519C
:10D5600095519651A451A651A251A951AA51AB511E
:10D57000B351B151B251B051B551BD51C551C9515D
:10D58000DB51E0515586E951ED51F051F551FE5115
:10D5900004520B5214520E5227522A522E52335218
:10D5A00039524F5244524B524C525E5254526A526C
:10D5B0007452695273527F527D528D5294529252DC
:10D5C000715288529152A88FA78FAC52AD52BC5263
:10D5D000B552C152CD52D752DE52E352E652ED98C7
:10D5E000E052F352F552F852F95206530853387587
:10D5F0000D5310530F5315531A5323532F533153B5
:10D6000033533853405346534553174E49534D53A4
:10D61000D6515E5369536E5318597B5377538253D7
:10D620009653A053A653A553AE53B053B653C3530A
:10D63000127CD996DF53FC66EE71EE53E853ED533E
:10D64000FA5301543D5440542C542D543C542E5400
:10D65000365429541D544E548F5475548E545F546F
:10D6600071547754705492547B548054765484543B
:10D6700090548654C754A254B854A554AC54C454BE
:10D68000C854A854AB54C254A454BE54BC54D85427
:10D69000E554E6540F551455FD54EE54ED54FA5428
:10D6A000E2543955405563554C552E555C554555FA
:10D6B00056555755385533555D5599558055AF5486
:10D6C0008A559F557B557E5598559E55AE557C5530
:10D6D0008355A9558755A855DA55C555DF55C45505
:10D6E000DC55E455D4551456F7551656FE55FD55E0
:10D6F0001B56F9554E565056DF7134563656325633
:10D7000038566B5664562F566C566A568656805657
:10D710008A56A05694568F56A556AE56B656B4564F
:10D72000C256BC56C156C356C056C856CE56D15620
:10D73000D356D756EE56F9560057FF560457095799
:10D7400008570B570D57135718571657C7551C57DF
:10D750002657375738574E573B5740574F576957FB
:10D76000C057885761577F5789579357A057B3576A
:10D77000A457AA57B057C357C657D457D257D357F1
:10D780000A58D657E3570B5819581D587258215844
:10D7900062584B587058C06B52583D58795885584C
:10D7A000B9589F58AB58BA58DE58BB58B858AE58FD
:10D7B000C558D358D158D758D958D858E558DC58F7
:10D7C000E458DF58EF58FA58F958FB58FC58FD5800
:10D7D00002590A5910591B59A66825592C592D5917
:10D7E000325938593E59D27A555950594E595A5989
:10D7F00058596259605967596C5969597859815912
:10D800009D595E4FAB4FA359B259C659E859DC59DF
:10D810008D59D959DA59255A1F5A115A1C5A095A81
:10D820001A5A405A6C5A495A355A365A625A6A5AE2
:10D830009A5ABC5ABE5ACB5AC25ABD5AE35AD75A00
:10D84000E65AE95AD65AFA5AFB5A0C5B0B5B165B3E
:10D85000325BD05A2A5B365B3E5B435B455B405B89
:10D86000515B555B5A5B5B5B655B695B705B735BD4
:10D87000755B785B88657A5B805B835BA65BB85B76
:10D88000C35BC75BC95BD45BD05BE45BE65BE25B1D
:10D89000DE5BE55BEB5BF05BF65BF35B055C075C1B
:10D8A000085C0D5C135C205C225C285C385C395C95
:10D8B000415C465C4E5C535C505C4F5C715B6C5CE5
:10D8C0006E5C624E765C795C8C5C915C945C9B597E
:10D8D000AB5CBB5CB65CBC5CB75CC55CBE5CC75C8F
:10D8E000D95CE95CFD5CFA5CED5C8C5DEA5C0B5D2F
:10D8F000155D175D5C5D1F5D1B5D115D145D225D37
:10D900001A5D195D185D4C5D525D4E5D4B5D6C5D41
:10D91000735D765D875D845D825DA25D9D5DAC5DBE
:10D92000AE5DBD5D905DB75DBC5DC95DCD5DD35D38
:10D93000D25DD65DDB5DEB5DF25DF55D0B5E1A5E83
:10D94000195E115E1B5E365E375E445E435E405E6E
:10D950004E5E575E545E5F5E625E645E475E755EFD
:10D96000765E7A5EBC9E7F5EA05EC15EC25EC85E71
:10D97000D05ECF5ED65EE35EDD5EDA5EDB5EE25EEB
:10D98000E15EE85EE95EEC5EF15EF35EF05EF45E41
:10D99000F85EFE5E035F095F5D5F5C5F0B5F115FBA
:10D9A000165F295F2D5F385F415F485F4C5F4E5FB8
:10D9B0002F5F515F565F575F595F615F6D5F735FA8
:10D9C000775F835F825F7F5F8A5F885F915F875F3A
:10D9D0009E5F995F985FA05FA85FAD5FBC5FD65FF9
:10D9E000FB5FE45FF85FF15FDD5FB360FF5F2160C5
:10D9F00060601960106029600E6031601B60156006
:10DA00002B6026600F603A605A6041606A60776000
:10DA10005F604A6046604D6063604360646042607E
:10DA20006C606B60596081608D60E76083609A60B4
:10DA300084609B60966097609260A7608B60E160F5
:10DA4000B860E060D360B460F05FBD60C660B56090
:10DA5000D8604D6115610661F660F7600061F460A1
:10DA6000FA6003612161FB60F1600D610E61476145
:10DA70003E61286127614A613F613C612C613461EC
:10DA80003D614261446173617761586159615A61D6
:10DA90006B6174616F61656171615F615D6153614B
:10DAA0007561996196618761AC6194619A618A61DF
:10DAB0009161AB61AE61CC61CA61C961F761C86156
:10DAC000C361C661BA61CB61797FCD61E661E36113
:10DAD000F661FA61F461FF61FD61FC61FE61006263
:10DAE000086209620D620C6214621B621E6221628E
:10DAF0002A622E6230623262336241624E625E623C
:10DB000063625B62606268627C62826289627E627A
:10DB1000926293629662D46283629462D762D162A7
:10DB2000BB62CF62FF62C662D464C862DC62CC6250
:10DB3000CA62C262C7629B62C9620C63EE62F16232
:10DB4000276302630863EF62F56250633E634D63CF
:10DB50001C644F6396638E638063AB637663A363D9
:10DB60008F6389639F63B5636B636963BE63E963B6
:10DB7000C063C663E363C963D263F663C4631664B8
:10DB8000346406641364266436641D65176428646F
:10DB90000F6467646F6476644E642A659564936469
:10DBA000A564A9648864BC64DA64D264C564C7648B
:10DBB000BB64D864C264F164E7640982E064E16430
:10DBC000AC62E364EF642C65F664F464F264FA64B6
:10DBD0000065FD6418651C650565246523652B6576
:10DBE000346535653765366538654B754865566506
:10DBF00055654D6558655E655D65726578658265DC
:10DC000083658A8B9B659F65AB65B765C365C66594
:10DC1000C165C465CC65D265DB65D965E065E16544
:10DC2000F16572670A660366FB657367356636667B
:10DC300034661C664F664466496641665E665D668C
:10DC40006466676668665F66626670668366886635
:10DC50008E668966846698669D66C166B966C96681
:10DC6000BE66BC66C466B866D666DA66E0663F66BF
:10DC7000E666E966F066F566F7660F6716671E6783
:10DC80002667276738972E673F673667416738678B
:10DC9000376746675E676067596763676467896768
:10DCA0007067A9677C676A678C678B67A667A167DF
:10DCB0008567B767EF67B467EC67B367E967B8670D
:10DCC000E467DE67DD67E267EE67B967CE67C66760
:10DCD000E7679C6A1E684668296840684D68326834
:10DCE0004E68B3682B685968636877687F689F6877
:10DCF0008F68AD6894689D689B688368AE6AB968F0
:10DD00007468B568A068BA680F698D687E68016933
:10DD1000CA680869D86822692669E1680C69CD6813
:10DD2000D468E768D568366912690469D768E3681A
:10DD30002569F968E068EF6828692A691A69236922
:10DD40002169C668796977695C6978696B69546922
:10DD50007E696E69396974693D69596930696169BB
:10DD60005E695D6981696A69B269AE69D069BF69D6
:10DD7000C169D369BE69CE69E85BCA69DD69BB69FF
:10DD8000C369A7692E6A9169A0699C699569B4699C
:10DD9000DE69E869026A1B6AFF690A6BF969F26960
:10DDA000E769056AB1691E6AED69146AEB690A6A76
:10DDB000126AC16A236A136A446A0C6A726A366A12
:10DDC000786A476A626A596A666A486A386A226A81
:10DDD000906A8D6AA06A846AA26AA36A976A1786A3
:10DDE000BB6AC36AC26AB86AB36AAC6ADE6AD16ADD
:10DDF000DF6AAA6ADA6AEA6AFB6A056B1686FA6A59
:10DE0000126B166B319B1F6B386B376BDC76396B83
:10DE1000EE98476B436B496B506B596B546B5B6B64
:10DE20005F6B616B786B796B7F6B806B846B836BE3
:10DE30008D6B986B956B9E6BA46BAA6BAB6BAF6B8A
:10DE4000B26BB16BB36BB76BBC6BC66BCB6BD36B8D
:10DE5000DF6BEC6BEB6BF36BEF6BBE9E086C136CC4
:10DE6000146C1B6C246C236C5E6C556C626C6A6C5D
:10DE7000826C8D6C9A6C816C9B6C7E6C686C736C24
:10DE8000926C906CC46CF16CD36CBD6CD76CC56C2F
:10DE9000DD6CAE6CB16CBE6CBA6CDB6CEF6CD96CCB
:10DEA000EA6C1F6D4D88366D2B6D3D6D386D196DAB
:10DEB000356D336D126D0C6D636D936D646D5A6DC0
:10DEC000796D596D8E6D956DE46F856DF96D156E7B
:10DED0000A6EB56DC76DE66DB86DC66DEC6DDE6D25
:10DEE000CC6DE86DD26DC56DFA6DD96DE46DD56DF3
:10DEF000EA6DEE6D2D6E6E6E2E6E196E726E5F6E29
:10DF00003E6E236E6B6E2B6E766E4D6E1F6E436E85
:10DF10003A6E4E6E246EFF6E1D6E386E826EAA6E65
:10DF2000986EC96EB76ED36EBD6EAF6EC46EB26EB4
:10DF3000D46ED56E8F6EA56EC26E9F6E416F116FDF
:10DF40004C70EC6EF86EFE6E3F6FF26E316FEF6EDE
:10DF5000326FCC6E3E6F136FF76E866F7A6F786F8D
:10DF6000816F806F6F6F5B6FF36F6D6F826F7C6F10
:10DF7000586F8E6F916FC26F666FB36FA36FA16F93
:10DF8000A46FB96FC66FAA6FDF6FD56FEC6FD46FD8
:10DF9000D86FF16FEE6FDB6F09700B70FA6F117055
:10DFA00001700F70FE6F1B701A70746F1D70187007
:10DFB0001F7030703E703270517063709970927043
:10DFC000AF70F170AC70B870B370AE70DF70CB70C2
:10DFD000DD70D9700971FD701C7119716571557111
:10DFE0008871667162714C7156716C718F71FB71C1
:10DFF00084719571A871AC71D771B971BE71D2710C
:10E00000C971D471CE71E071EC71E771F571FC7179
:10E01000F971FF710D7210721B7228722D722C72C1
:10E02000307232723B723C723F72407246724B7277
:10E03000587274727E728272817287729272967254
:10E04000A272A772B972B272C372C672C472CE7271
:10E05000D272E272E072E172F972F7720F501773C6
:10E060000A731C7316731D7334732F73297325730E
:10E070003E734E734F73D89E57736A736873707391
:10E08000787375737B737A73C873B373CE73BB7312
:10E09000C073E573EE73DE73A27405746F74257438
:10E0A000F87332743A7455743F745F7459744174E0
:10E0B0005C746974707463746A7476747E748B743F
:10E0C0009E74A774CA74CF74D474F173E074E3744B
:10E0D000E774E974EE74F274F074F174F874F77420
:10E0E0000475037505750C750E750D75157513752D
:10E0F0001E7526752C753C7544754D754A754975A8
:10E100005B7546755A756975647567756B756D7560
:10E11000787576758675877574758A758975827553
:10E1200094759A759D75A575A375C275B375C375FC
:10E13000B575BD75B875BC75B175CD75CA75D27537
:10E14000D975E375DE75FE75FF75FC750176F075A2
:10E15000FA75F275F3750B760D7609761F762776CC
:10E160002076217622762476347630763B76477692
:10E17000487646765C765876617662766876697619
:10E180006A7667766C7670767276767678767C7656
:10E190008076837688768B768E7696769376997669
:10E1A0009A76B076B476B876B976BA76C276CD7607
:10E1B000D676D276DE76E176E576E776EA762F8653
:10E1C000FB76087707770477297724771E772577FA
:10E1D00026771B773777387747775A7768776B7763
:10E1E0005B7765777F777E7779778E778B77917797
:10E1F000A0779E77B077B677B977BF77BC77BD77D2
:10E20000BB77C777CD77D777DA77DC77E377EE77A9
:10E21000FC770C781278267920782A7945788E78E0
:10E22000747886787C789A788C78A378B578AA7890
:10E23000AF78D178C678CB78D478BE78BC78C578FA
:10E24000CA78EC78E778DA78FD78F478077912798B
:10E25000117919792C792B794079607957795F791F
:10E260005A79557953797A797F798A799D79A7791D
:10E270004B9FAA79AE79B379B979BA79C979D57949
:10E28000E779EC79E179E379087A0D7A187A197AE5
:10E29000207A1F7A8079317A3B7A3E7A377A437ACC
:10E2A000577A497A617A627A697A9D9F707A797A27
:10E2B0007D7A887A977A957A987A967AA97AC87ABE
:10E2C000B07AB67AC57AC47ABF7A8390C77ACA7AA6
:10E2D000CD7ACF7AD57AD37AD97ADA7ADD7AE17AB9
:10E2E000E27AE67AED7AF07A027B0F7B0A7B067B94
:10E2F000337B187B197B1E7B357B287B367B507BE1
:10E300007A7B047B4D7B0B7B4C7B457B757B657BF4
:10E31000747B677B707B717B6C7B6E7B9D7B987B5A
:10E320009F7B8D7B9C7B9A7B8B7B927B8F7B5D7BAA
:10E33000997BCB7BC17BCC7BCF7BB47BC67BDD7BEE
:10E34000E97B117C147CE67BE57B607C007C077CB0
:10E35000137CF37BF77B177C0D7CF67B237C277C7F
:10E360002A7C1F7C377C2B7C3D7C4C7C437C547C02
:10E370004F7C407C507C587C5F7C647C567C657C08
:10E380006C7C757C837C907CA47CAD7CA27CAB7C1B
:10E39000A17CA87CB37CB27CB17CAE7CB97CBD7C1A
:10E3A000C07CC57CC27CD87CD27CDC7CE27C3B9B84
:10E3B000EF7CF27CF47CF67CFA7C067D027D1C7D91
:10E3C000157D0A7D457D4B7D2E7D327D3F7D357DE2
:10E3D000467D737D567D4E7D727D687D6E7D4F7D61
:10E3E000637D937D897D5B7D8F7D7D7D9B7DBA7D0A
:10E3F000AE7DA37DB57DC77DBD7DAB7D3D7EA27D20
:10E40000AF7DDC7DB87D9F7DB07DD87DDD7DE47DF9
:10E41000DE7DFB7DF27DE17D057E0A7E237E217E11
:10E42000127E317E1F7E097E0B7E227E467E667EB8
:10E430003B7E357E397E437E377E327E3A7E677EF6
:10E440005D7E567E5E7E597E5A7E797E6A7E697ECC
:10E450007C7E7B7E837ED57D7D7EAE8F7F7E887E3B
:10E46000897E8C7E927E907E937E947E967E8E7E3A
:10E470009B7E9C7E387F3A7F457F4C7F4D7F4E7FD1
:10E48000507F517F557F547F587F5F7F607F687FCB
:10E49000697F677F787F827F867F837F887F877FA2
:10E4A0008C7F947F9E7F9D7F9A7FA37FAF7FB27F7B
:10E4B000B97FAE7FB67FB87F718BC57FC67FCA7FBD
:10E4C000D57FD47FE17FE67FE97FF37FF97FDC981A
:10E4D000068004800B801280188019801C802180A7
:10E4E00028803F803B804A804680528058805A80F6
:10E4F0005F806280688073807280708076807980AF
:10E500007D807F808480868085809B8093809A80B8
:10E51000AD809051AC80DB80E580D980DD80C48007
:10E52000DA80D6800981EF80F1801B8129812381E7
:10E530002F814B818B9646813E8153815181FC8096
:10E5400071816E81658166817481838188818A8110
:10E5500080818281A0819581A481A3815F81938143
:10E56000A981B081B581BE81B881BD81C081C281E0
:10E57000BA81C981CD81D181D981D881C881DA811F
:10E58000DF81E081E781FA81FB81FE8101820282E5
:10E59000058207820A820D821082168229822B82CE
:10E5A000388233824082598258825D825A825F82E9
:10E5B0006482628268826A826B822E827182778232
:10E5C00078827E828D829282AB829F82BB82AC8275
:10E5D000E182E382DF82D282F482F382FA82938341
:10E5E0000383FB82F982DE820683DC820983D9827F
:10E5F0003583348316833283318340833983508358
:10E6000045832F832B831783188385839A83AA835B
:10E610009F83A283968323838E8387838A837C83CD
:10E62000B58373837583A0838983A883F48313845C
:10E63000EB83CE83FD830384D8830B84C183F7836C
:10E640000784E083F2830D8422842084BD83388490
:10E650000685FB836D842A843C845A858484778470
:10E660006B84AD846E848284698446842C846F8438
:10E6700079843584CA846284B984BF849F84D984B0
:10E68000CD84BB84DA84D084C184C684D684A1843A
:10E690002185FF84F484178518852C851F851585B1
:10E6A0001485FC84408563855885488541850286AC
:10E6B0004B8555858085A485888591858A85A88523
:10E6C0006D8594859B85EA8587859C8577857E8584
:10E6D0009085C985BA85CF85B985D085D585DD85F5
:10E6E000E585DC85F9850A8613860B86FE85FA8525
:10E6F000068622861A8630863F864D86554E54867B
:10E700005F86678671869386A386A986AA868B868E
:10E710008C86B686AF86C486C686B086C9862388B0
:10E72000AB86D486DE86E986EC86DF86DB86EF86DE
:10E7300012870687088700870387FB86118709876A
:10E740000D87F9860A8734873F8737873B87258778
:10E7500029871A8760875F8778874C874E877487F9
:10E76000578768876E875987538763876A870588C5
:10E77000A2879F878287AF87CB87BD87C087D087D7
:10E78000D696AB87C487B387C787C687BB87EF8713
:10E79000F287E0870F880D88FE87F687F7870E8857
:10E7A000D287118816881588228821883188368872
:10E7B000398827883B8844884288528859885E88EF
:10E7C00062886B8881887E889E8875887D88B588F8
:10E7D0007288828897889288AE889988A2888D8866
:10E7E000A488B088BF88B188C388C488D488D888F2
:10E7F000D988DD88F9880289FC88F488E888F2885D
:10E8000004890C890A89138943891E8925892A89E3
:10E810002B89418944893B89368938894C891D89EE
:10E8200060895E89668964896D896A896F8974895E
:10E8300077897E89838988898A8993899889A1893A
:10E84000A989A689AC89AF89B289BA89BD89BF89EE
:10E85000C089DA89DC89DD89E789F489F889038A46
:10E86000168A108A0C8A1B8A1D8A258A368A418A52
:10E870005B8A528A468A488A7C8A6D8A6C8A628A56
:10E88000858A828A848AA88AA18A918AA58AA68A88
:10E890009A8AA38AC48ACD8AC28ADA8AEB8AF38AE0
:10E8A000E78AE48AF18A148BE08AE28AF78ADE8AB0
:10E8B000DB8A0C8B078B1A8BE18A168B108B178BDC
:10E8C000208B338BAB97268B2B8B3E8B288B418BEE
:10E8D0004C8B4F8B4E8B498B568B5B8B5A8B6B8B38
:10E8E0005F8B6C8B6F8B748B7D8B808B8C8B8E8B0B
:10E8F000928B938B968B998B9A8B3A8C418C3F8C15
:10E90000488C4C8C4E8C508C558C628C6C8C788CDA
:10E910007A8C828C898C858C8A8C8D8C8E8C948C54
:10E920007C8C988C1D62AD8CAA8CBD8CB28CB38C07
:10E93000AE8CB68CC88CC18CE48CE38CDA8CFD8CEC
:10E94000FA8CFB8C048D058D0A8D078D0F8D0D8D36
:10E95000108D4E9F138DCD8C148D168D678D6D8D02
:10E96000718D738D818D998DC28DBE8DBA8DCF8D38
:10E97000DA8DD68DCC8DDB8DCB8DEA8DEB8DDF8D59
:10E98000E38DFC8D088E098EFF8D1D8E1E8E108EE0
:10E990001F8E428E358E308E348E4A8E478E498E33
:10E9A0004C8E508E488E598E648E608E2A8E638E69
:10E9B000558E768E728E7C8E818E878E858E848E1D
:10E9C0008B8E8A8E938E918E948E998EAA8EA18E26
:10E9D000AC8EB08EC68EB18EBE8EC58EC88ECB8EDE
:10E9E000DB8EE38EFC8EFB8EEB8EFE8E0A8F058F08
:10E9F000158F128F198F138F1C8F1F8F1B8F0C8FEA
:10EA0000268F338F3B8F398F458F428F3E8F4C8FB0
:10EA1000498F468F4E8F578F5C8F628F638F648FC5
:10EA20009C8F9F8FA38FAD8FAF8FB78FDA8FE58FBE
:10EA3000E28FEA8FEF8F8790F48F0590F98FFA8F2E
:10EA40001190159021900D901E9016900B9027908C
:10EA5000369035903990F88F4F9050905190529059
:10EA60000E9049903E90569058905E9068906F90AE
:10EA70007690A896729082907D90819080908A90F6
:10EA800089908F90A890AF90B190B590E290E4906B
:10EA90004862DB90029112911991329130914A9122
:10EAA00056915891639165916991739172918B918F
:10EAB00089918291A291AB91AF91AA91B591B491B4
:10EAC000BA91C091C191C991CB91D091D691DF916A
:10EAD000E191DB91FC91F591F6911E92FF911492D8
:10EAE0002C92159211925E9257924592499264929D
:10EAF000489295923F924B9250929C92969293920A
:10EB00009B925A92CF92B992B792E9920F93FA924E
:10EB100044932E93199322931A9323933A93359304
:10EB20003B935C9360937C936E935693B093AC93BA
:10EB3000AD939493B993D693D793E893E593D893F1
:10EB4000C393DD93D093C893E4931A9414941394CD
:10EB500003940794109436942B94359421943A940A
:10EB60004194529444945B94609462945E946A9449
:10EB700029927094759477947D945A947C947E94A1
:10EB800081947F94829587958A959495969598958A
:10EB90009995A095A895A795AD95BC95BB95B99568
:10EBA000BE95CA95F66FC395CD95CC95D595D49560
:10EBB000D695DC95E195E595E295219628962E96D9
:10EBC0002F9642964C964F964B9677965C965E960D
:10EBD0005D965F96669672966C968D9698969596CB
:10EBE0009796AA96A796B196B296B096B496B69610
:10EBF000B896B996CE96CB96C996CD964D89DC96A9
:10EC00000D97D596F99604970697089713970E9740
:10EC100011970F971697199724972A973097399736
:10EC20003D973E97449746974897429749975C97F8
:10EC30006097649766976897D2526B9771977997A8
:10EC400085977C9781977A9786978B978F979097E0
:10EC50009C97A897A697A397B397B497C397C6977F
:10EC6000C897CB97DC97ED974F9FF297DF7AF6978F
:10EC7000F5970F980C9838982498219837983D98D4
:10EC800046984F984B986B986F98709871987498B5
:10EC90007398AA98AF98B198B698C498C398C69834
:10ECA000E998EB980399099912991499189921995F
:10ECB0001D991E99249920992C992E993D993E9938
:10ECC00042994999459950994B99519952994C9922
:10ECD000559997999899A599AD99AE99BC99DF994D
:10ECE000DB99DD99D899D199ED99EE99F199F2993D
:10ECF000FB99F899019A0F9A059AE299199A2B9A19
:10ED0000379A459A429A409A439A3E9A559A4D9A12
:10ED10005B9A579A5F9A629A659A649A699A6B9A13
:10ED20006A9AAD9AB09ABC9AC09ACF9AD19AD39A5D
:10ED3000D49ADE9ADF9AE29AE39AE69AEF9AEB9AED
:10ED4000EE9AF49AF19AF79AFB9A069B189B1A9BF3
:10ED50001F9B229B239B259B279B289B299B2A9BB0
:10ED60002E9B2F9B329B449B439B4F9B4D9B4E9BCB
:10ED7000519B589B749B939B839B919B969B979BCA
:10ED80009F9BA09BA89BB49BC09BCA9BB99BC69B07
:10ED9000CF9BD19BD29BE39BE29BE49BD49BE19BCB
:10EDA0003A9CF29BF19BF09B159C149C099C139C34
:10EDB0000C9C069C089C129C0A9C049C2E9C1B9CF0
:10EDC000259C249C219C309C479C329C469C3E9CCC
:10EDD0005A9C609C679C769C789CE79CEC9CF09C81
:10EDE000099D089DEB9C039D069D2A9D269DAF9D38
:10EDF000239D1F9D449D159D129D419D3F9D3E9DC0
:10EE0000469D489D5D9D5E9D649D519D509D599D73
:10EE1000729D899D879DAB9D6F9D7A9D9A9DA49DB6
:10EE2000A99DB29DC49DC19DBB9DB89DBA9DC69D27
:10EE3000CF9DC29DD99DD39DF89DE69DED9DEF9DF3
:10EE4000FD9D1A9E1B9E1E9E759E799E7D9E819E97
:10EE5000889E8B9E8C9E929E959E919E9D9EA59E29
:10EE6000A99EB89EAA9EAD9E6197CC9ECE9ECF9E37
:10EE7000D09ED49EDC9EDE9EDD9EE09EE59EE89EBA
:10EE8000EF9EF49EF69EF79EF99EFB9EFC9EFD9ED5
:10EE9000079F089FB776159F219F2C9F3E9F4A9FF3
:10EEA000529F549F639F5F9F609F619F669F679F74
:10EEB0006C9F6A9F779F729F769F959F9C9FA09F54
:10EEC0002F58C76959906474DC5199719C4E16553E
:10EED000035A3F96C0541B612863F65922907584EB
:10EEE0001C83507AAA60E163256EED656684A68274
:10EEF000F59B93682757A16571629B5BD0597B8610
:10EF0000F498627DBE7D8E9B16629F7CB788895B7C
:10EF1000B55E096397664868C7958D974F67E54E5C
:10EF20000A4F4D4F9D4F4950F2563759D459015A07
:10EF3000095CDF600F61706113660569BA704F7517
:10EF40007075FB79AD7DEF7DC3800E846388028B85
:10EF500055907A903B53954EA54EDF57B280C190A5
:10EF6000EF78004EF158A26E3890327A28838B8267
:10EF70002F9C41517053BD54E154E056FB59155F2D
:10EF8000F298EB6DE4802D8562967096A096FB97C3
:10EF90000B54F353875BCF70BD7FC28FE8966F53DE
:10EFA0005C9DBA7A114E9378FC81266E18560455F2
:10EFB0001D6B1A853B9CE559A953666DDC748F95D2
:10EFC0004256914E4B90F2964F830C99E153B655B1
:10EFD000305B715F2066F3660468386CF36C296DF2
:10EFE0005B74C8764E7A3498F1825B88608AED92C1
:10EFF000B26DAB75CA76C599A660018B8A8DB29544
:10F000008E69AD538651125730584459B45BF65E41
:10F010002860A963F463BF6C146F8E70147159710A
:10F02000D5713F73017E7682D182978560905B9225
:10F030001B9D6958BC655A6C2575F9512E59655947
:10F04000805FDC5FBC62FA652A6A276BB46B8B73E6
:10F05000C17F56892C9D0E9DC49EA15C966C7B83BE
:10F0600004514B5CB661C68176686172594EFA4FA5
:10F0700078536960296E4F7AF3970B4E1653EE4E14
:10F08000554F3D4FA14F734FA052EF5309560F59A3
:10F09000C15AB65BE15BD17987669C67B6674C6BFA
:10F0A000B36C6B70C2738D79BE793C7A877BB18209
:10F0B000DB8204837783EF83D3836687B28A295602
:10F0C000A88CE68F4E901E978A86C44FE85C11622A
:10F0D00059723B75E581BD82FE86C08CC596139939
:10F0E000D599CB4E1A4FE389DE564A58CA58FB5E73
:10F0F000EB5F2A6094606260D0611262D062396511
:10F10000419B6666B068776D70704C758676757DCC
:10F11000A582F9878B958E969D8CF151BE5216591A
:10F12000B354B35B165D68618269AF6D8D78CB8433
:10F130005788728AA793B89A6C6DA899D986A357F5
:10F14000FF67CE860E92835287560454D35EE162E7
:10F15000B9643C683868BB6B7273BA786B7A9A8909
:10F16000D2896B8D038FED90A39594966997665B1A
:10F17000B35C7D694D984E989B63207B2B6A7F6AB8
:10F18000B6680D9C5F6F72529D557060EC623B6D6E
:10F19000076ED16E5B841089448F144E399CF653F0
:10F1A0001B693A6A84972A685C51C37AB284DC91FD
:10F1B0008C935B56289D226805833184A57C085278
:10F1C000C582E6747E4E834FA051D25B0A52D8525C
:10F1D000E752FB5D9A552A58E6598C5B985BDB5BDE
:10F1E000725E795EA3601F616361BE61DB6362650D
:10F1F000D1675368FA683E6B536B576C226F976FF9
:10F20000456FB0741875E3760B77FF7AA17B217C8C
:10F21000E97D367FF07F9D8066829E83B389CC8AAC
:10F22000AB8C8490519493959195A2956596D397C4
:10F2300028991882384E2B54B85CCC5DA9734C7653
:10F240003C77A95CEB7F0B8DC19611985498589828
:10F25000014F0E4F71539C556856FA574759095B39
:10F26000C45B905C0C5E7E5ECC5FEE633A67D765F4
:10F27000E2651F67CB68C4685F6A305EC56B176C58
:10F280007D6C7F754879635B007A007DBD5F8F89F7
:10F29000188AB48C778DCC8E1D8FE2980E9A3C9B89
:10F2A000804E7D50005193599C5B2F628062EC64CC
:10F2B0003A6BA07291754779A97FFB87BC8A708BE6
:10F2C000AC63CA83A09709540354AB555468586A79
:10F2D000708A27787567CD9E7453A25B1A81508619
:10F2E0000690184E454EC74E114FCA533854AE5B68
:10F2F000135F256051653D67426C726CE36C7870FA
:10F300000374767AAE7A087B1A7DFE7C667DE765AB
:10F310005B72BB53455CE85DD262E0621963206EAC
:10F320005A86318ADD8DF892016FA6795A9BA84ED4
:10F33000AB4EAC4E9B4FA04FD1504751F67A715116
:10F34000F651545321537F53EB53AC558358E15C32
:10F35000375F4A5F2F6050606D601F6359654B6A6D
:10F36000C16CC272ED72EF77F880058108824E851C
:10F37000F790E193FF9757995A9AF04EDD512D5C23
:10F3800081666D69405CF266756989735068817C3D
:10F39000C550E4524757FE5D2693A465236B3D6B31
:10F3A00034748179BD794B7BCA7DB982CC837F88E7
:10F3B0005F89398BD18FD1911F5480925D4E365029
:10F3C000E5533A53D7729673E977E682AF8EC699C2
:10F3D000C899D29977511A615E86B0557A7A76507B
:10F3E000D35B47908596324EDB6AE791515C485C6F
:10F3F00098639F7A936C7497618FAA7A8A718896C2
:10F40000827C1768707E51686C93F2521B54AB85F6
:10F41000138AA47FCD8EE190665388884179C24FCC
:10F42000BE501152445153552D57EA738B575159C1
:10F43000625F845F756076616761A961B2633A64F7
:10F440006C656F664268136E66753D7AFB7C4C7D19
:10F45000997D4B7E6B7F0E834A83CD86088A638AB3
:10F46000668BFD8E1A988F9DB882CE8FE89B87524F
:10F470001F628364C06F999641689150206B7A6CCB
:10F48000546F747A507D4088238A0867F64E39504D
:10F49000265065507C5138526352A7550F57055876
:10F4A000CC5AFA5EB261F861F36272631C69296A30
:10F4B0007D72AC722E7314786F78797D0C77A98089
:10F4C0008B89198BE28CD28E639075937A965598BE
:10F4D000139A789E43519F53B3537B5E265F1B6EF6
:10F4E000906E8473FE73437D3782008AFA8A509649
:10F4F0004E4E0B50E4537C54FA56D159645BF15D87
:10F50000AB5E275F38624565AF67566ED072CA7CC6
:10F51000B488A180E180F0834E86878AE88D379297
:10F52000C7966798139F944E924E0D4F4853495477
:10F530003E542F5A8C5FA15F9F60A7688E6A5A74F1
:10F5400081789E8AA48A778B90915E4EC99BA44E47
:10F550007C4FAF4F1950165049516C519F52B952C0
:10F56000FE529A53E35311540E5489555157A257E2
:10F570007D59545B5D5B8F5BE55DE75DF75D785EB4
:10F58000835E9A5EB75E185F52604C619762D86284
:10F59000A7633B6502664366F4666D6721689768FA
:10F5A000CB695F6C2A6D696D2F6E9D6E32758776A3
:10F5B0006C783F7AE07C057D187D5E7DB17D15809D
:10F5C0000380AF80B18054818F812A8252834C881E
:10F5D00061881B8BA28CFC8CCA90759171923F78CC
:10F5E000FC92A4954D9605989999D89A3B9D5B52AB
:10F5F000AB52F7530854D558F762E06F6A8C5F8FAF
:10F60000B99E4B513B524A54FD56407A7791609DCA
:10F61000D29E4473096F70811175FD5FDA60A89AFC
:10F62000DB72BC8F646B0398CA4EF0566457BE58A9
:10F630005A5A6860C7610F6606663968B168F76D27
:10F64000D5753A7D6E82429B9B4E504FC9530655ED
:10F650006F5DE65DEE5DFB67996C73740278508AAE
:10F660009693DF885057A75E2B63B550AC508D51F1
:10F670000067C9545E58BB59B05B695F4D62A163B6
:10F680003D68736B086E7D70C7918072157826781F
:10F690006D798E65307DDC83C188098F9B966452BD
:10F6A000285750676A7FA18CB45142572A963A581E
:10F6B0008A69B480B2540E5DFC579578FA9D5C4F10
:10F6C0004A528B543E6428661467F567847A567BE9
:10F6D000227D2F935C68AD9B397B19538A51375239
:10F6E000DF5BF662AE64E6642D67BA6BA985D196DE
:10F6F0009076D69B4C630693AB9BBF765266094EC1
:10F700009850C253715CE860926463655F68E6710B
:10F71000CA732375977B827E9586838BDB8C789169
:10F720001099AC65AB668B6BD54ED44E3A4F7F4F7C
:10F730003A52F853F253E355DB56EB58CB59C959BB
:10F74000FF59505B4D5C025E2B5ED75F1D60076307
:10F750002F655C5BAF65BD65E8659D67626B7B6B24
:10F760000F6C45734979C179F87C197D2B7DA28096
:10F770000281F38196895E8A698A668A8C8AEE8A1A
:10F78000C78CDC8CCC96FC986F6B8B4E3C4F8D4FAE
:10F790005051575BFA5B486101634266216BCB6E47
:10F7A000BB6C3E72BD74D475C1783A790C803380DD
:10F7B000EA8194849E8F506C7F9E0F5F588B2B9DA7
:10F7C000FA7AF88E8D5BEB96034EF153F757315969
:10F7D000C95AA45B89607F6E066FBE75EA8C9F5B19
:10F7E0000085E07B7250F4679D82615C4A851E7ED5
:10F7F0000E829951045C6863668D9C656E713E79DA
:10F80000177D05801D8BCA8E6E90C786AA901F50EB
:10F81000FA523A5C53677C7035724C91C8912B93C5
:10F82000E582C25B315FF9603B4ED653885B4B6229
:10F8300031678A6BE972E0732E7A6B81A38D5291E6
:10F8400096991251D7536A54FF5B8863396AAC7D2D
:10F850000097DA56CE536854975B315CDE5DEE4F0D
:10F860000161FE62326DC079CB79427D4D7ED27FDF
:10F87000ED811F82908446887289908B748E2F8FC1
:10F8800031904B916C91C6969C91C04E4F4F455113
:10F890004153935F0E62D467416C0B6E6373267E97
:10F8A000CD918392D4531959BF5BD16D5D792E7E72
:10F8B0009B7C7E589F71FA515388F08FCA4FFB5C36
:10F8C0002566AC77E37A1C82FF99C651AA5FEC6586
:10F8D0006F69896BF36D966E646FFE76147DE15DE2
:10F8E000759087910698E6511D5240629166D966DF
:10F8F0001A6EB65ED27D727FF866AF85F785F88A9C
:10F90000A952D95373598F5E905F5560E492649603
:10F91000B7501F51DD5220534753EC53E85446551E
:10F92000315517566859BE593C5AB55B065C0F5C99
:10F93000115C1A5C845E8A5EE05E705F7F62846246
:10F94000DB628C63776307660C662D6676667E677E
:10F95000A2681F6A356ABC6C886D096E586E3C716E
:10F9600026716771C77501775D7801796579F079DE
:10F97000E07A117BA77C397D9680D6838B8449857C
:10F980005D88F3881F8A3C8A548A738A618CDE8C76
:10F99000A49166927E9318949C9698970A4E084E6E
:10F9A0001E4E574E97517052CE573458CC58225B4A
:10F9B000385EC560FE6461675667446DB6727375E4
:10F9C000637AB884728BB89120933156F457FE98BD
:10F9D000ED620D69966BED71547E77807282E689D7
:10F9E000DF985587B18F3B5C384FE14FB54F0755D6
:10F9F000205ADD5BE95BC35F4E612F63B0654B66E8
:10FA0000EE689B69786DF16D3375B9751F775E7916
:10FA1000E679337DE381AF82AA85AA893A8AAB8EE3
:10FA20009B8F3290DD910797BA4EC14E03527558A5
:10FA3000EC580B5C1A753D5C4E810A8AC58F639643
:10FA40006D97257BCF8A08986291F356A85317903B
:10FA500039548257255EA863346C8A7061778B7C39
:10FA6000E07F708842905491109318938F965E7443
:10FA7000C49A075D695D7065A267A88DDB966E63A9
:10FA800049671969C5831798C096FE88846F7A64A0
:10FA9000F85B164E2C705D752F66C4513652E252DB
:10FAA000D359815F276010623F6574651F66746675
:10FAB000F2681668636B056E72721F75DB76BE7C2A
:10FAC0005680F058FD887F89A08A938ACB8A1D9042
:10FAD00092915297599789650E7A0681BB962D5E51
:10FAE000DC601A62A56514669067F3774D7A4D7CE9
:10FAF0003E7E0A81AC8C648DE18D5F8EA9780752C1
:10FB0000D962A563426498622D8A837AC07BAC8AED
:10FB1000EA96767D0C824987D94E4851435360530B
:10FB2000A35B025C165CDD5D26624762B06413680D
:10FB30003468C96C456D176DD3675C6F4E717D710C
:10FB4000CB657F7AAD7BDA7D4A7EA87F7A811B8286
:10FB50003982A6856E8ACE8CF58D78907790AD929D
:10FB600091928395AE9B4D528455386F3671685192
:10FB70008579557EB381CE7C4C565158A85CAA63DA
:10FB8000FE66FD665A69D9728F758E750E79567943
:10FB9000DF79977C207D447D0786348A3B9661908F
:10FBA000209FE7507552CC53E2530950AA55EE58A6
:10FBB0004F593D728B5B645C1D53E360F3605C6383
:10FBC00083633F63BB63CD64E965F966E35DCD693B
:10FBD000FD69156FE571894EE975F876937ADF7CDA
:10FBE000CF7D9C7D6180498358836C84BC84FB8578
:10FBF000C588708D01906D9097931C97129ACF5085
:10FC000097588E61D3813585088D2090C34F7450ED
:10FC1000475273536F6049635F672C6EB38D1F90BB
:10FC2000D74F5E5CCA8CCF659A7D525396887651C9
:10FC3000C363585B6B5B0A5C0D6451675C90D64E86
:10FC40001A592A59706C518A3E551558A559F060B9
:10FC50005362C167358255694096C499289A534FBB
:10FC60000658FE5B1080B15C2F5E855F20604B61A3
:10FC70003462FF66F06CDE6ECE807F81D4828B882A
:10FC8000B88C00902E908A96DB9EDB9BE34EF0535F
:10FC900027592C7B8D914C98F99DDD6E277053531D
:10FCA0004455855B58629E62D362A26CEF6F2274EA
:10FCB000178A3894C16FFE8A3883E751F886EA5371
:10FCC000E953464F5490B08F6A593181FD5DEA7A0D
:10FCD000BF8FDA68378CF872489C3D6AB08A394E1B
:10FCE000585306566657C562A263E6654E6BE16DD2
:10FCF0005B6EAD70ED77EF7AAA7BBB7D3D80C680F1
:10FD0000CB86958A5B93E356C7583E5FAD65966692
:10FD1000806AB56B3775C78A2450E57730571B5F0B
:10FD200065607A66606CF4751A7A6E7FF481188764
:10FD30004590B399C97B5C75F97A517BC484109066
:10FD4000E979927A3683E15A40772D4EF24E995BEB
:10FD5000E05FBD623C66F167E86C6B8677883B8A42
:10FD60004E91F392D099176A26702A73E7825784CE
:10FD7000AF8C014E4651CB518B55F55B165E335E11
:10FD8000815E145F355F6B5FB45FF2611163A266E1
:10FD90001D676E6F52723A753A7774803981788137
:10FDA0007687BF8ADC8A858DF38D9A927795029843
:10FDB000E59CC5525763F4761567886CCD73C38C88
:10FDC000AE937396256D9C580E69CC69FD8F9A93FE
:10FDD000DB751A905A580268B463FB69434F2C6F65
:10FDE000D867BB8F2685B47D54933F69706F6A577F
:10FDF000F7582C5B2C7D2A720A54E391B49DAD4ECA
:10FE00004E4F5C50755043529E8C485424589A5B18
:10FE10001D5E955EAD5EF75E1F5F8C60B5623A63F6
:10FE2000D063AF68406C87788E790B7AE07D47822B
:10FE3000028AE68A448E1390B8902D91D8910E9F35
:10FE4000E56C5864E2647565F46E84761B7B69909A
:10FE5000D193BA6EF254B95FA4644D8FED8F449282
:10FE600078516B582959555C975EFB6D8F7E1C75D8
:10FE7000BC8CE28E5B98B9701D4FBF6BB16F307553
:10FE8000FB964E51105435585758AC59605C925FF0
:10FE900097655C67216E7B76DF83ED8C1490FD9017
:10FEA0004D9325783A78AA52A65E1F57745912606E
:10FEB00012505A51AC51CD51005210555458585807
:10FEC0005759955BF65C8B5DBC6095622D647167DC
:10FED0004368BC68DF68D776D86D6F6E9B6D6F70B6
:10FEE000C871535FD8757779497B547B527BD67C38
:10FEF000717D305263846985E4850E8A048B468C5B
:10FF00000F8E03900F90199476962D98309AD8956D
:10FF1000CD50D5520C5402580E5CA7619E641E6DE4
:10FF2000B377E57AF480048453908592E05C079D72
:10FF30003F53975FB35F9C6D79726377BF79E47BC2
:10FF4000D26BEC72AD8A0368616AF851817A3469C8
:10FF50004A5CF69CEB82C55B49911E7078566F5CDB
:10FF6000C76066658C6C5A8C419013985154C76673
:10FF70000D924859A39085514D4EEA5199850E8BAB
:10FF800058707A634B936269B499047E77755753BE
:10FF90006069DF8EE3965D6C8C4E3C5C105FE98F90
:10FFA0000253D18C89807986FF5EE565734E655179
:10FFB00082593F5CEE97FB4E8A59CD5F8D8AE16F87
:10FFC000B0796279E75B71842B73B171745EF55F10
:10FFD0007B639A64C371987C434EFC5E4B4EDC5746
:10FFE000A256A960C36F0D7DFD803381BF81B28FA2
:10FFF0009789A486F45D8A62AD6487897767E26C2D
:020000041001E9
:100000003E6D36743478465A757FAD82AC99F34FA5
:10001000C35EDD62926357656F67C3764C72CC80B6
:10002000BA80298F4D910D50F957925A856873699E
:100030006471FD72B78CF258E08C6A9619907F87D4
:10004000E479E77729842F4F65525A53CD62CF6701
:10005000CA6C7D76947B957C36828485EB8FDD66D9
:10006000206F06721B7EAB83C199A69EFD51B17BAA
:100070007278B87B8780487BE86A615E8C805175B6
:1000800060756B5162928C6E7A769791EA9A104FF6
:10009000707F9C624F7BA595E99C7A565958E486FF
:1000A000BC96344F24524A53CD53DB53065E2C6426
:1000B00091657F673E6C4E6C4872AF72ED735475FC
:1000C000417E2C82E985A98CC47BC6916971129806
:1000D000EF983D6369666A75E476D0784385EE866D
:1000E0002A53515326548359875E7C5FB26049621C
:1000F0007962AB629065D46BCC6CB275AE76917858
:10010000D879CB7D777FA580AB88B98ABB8C7F906F
:100110005E97DB980B6A387C99503E5CAE5F8767D0
:10012000D86B357409778E7F3B9FCA67177A39532E
:100130008B75ED9A665F9D81F18398803C5FC55F0A
:100140006275467B3C906768EB599B5A107D7E76C2
:100150002C8BF54F6A5F196A376C026FE27468790D
:100160006888558A798CDF5ECF63C575D279D7826E
:100170002893F2929C84ED862D9CC1546C5F8C6513
:100180005C6D1570A78CD38C3B984F65F6740D4E43
:10019000D84EE0572B59665ACC5BA851035E9C5E43
:1001A000166076627765A7656E666E6D3672267B21
:1001B00050819A8199825C8BA08CE68C748D1C9600
:1001C0004496AE4FAB64666B1E8261846A85E8908C
:1001D000015C5369A8987A8457850F4F6F52A95FC5
:1001E000455E0D678F79798107898689F56D175F7F
:1001F0005562B86CCF4E6972929B06523B5474564E
:10020000B358A4616E621A716E59897CDE7C1B7DC5
:10021000F09687655E80194E754F75514058635E44
:10022000735E0A5FC467264E3D8589955B96737C35
:100230000198FB50C1585676A7782552A5771185AD
:10024000867B4F5009594772C77BE87DBA8FD48FA0
:100250004D90BF4FC952295A015FAD97DD4F1782AC
:10026000EA9203575563696B2B75DC88148F427AC9
:10027000DF52935855610A62AE66CD6B3F7CE983CD
:100280002350F84F05534654315849599D5BF05C53
:10029000EF5C295D965EB16267633E65B9650B6789
:1002A000D56CE16CF97032782B7EDE80B3820C84E1
:1002B000EC84028712892A8A4A8CA690D292FD98F1
:1002C000F39C6C9D4F4EA14E8D5056524A57A859E3
:1002D0003D5ED85FD95F3F62B4661B67D067D26866
:1002E0009251217DAA80A881008B8C8CBF8C7E923C
:1002F000329620542C981753D5505C53A858B264AA
:10030000346767726677467AE691C352A16C866B52
:1003100000584C5E54592C67FB7FE151C6766964E6
:10032000E878549BBB9ECB57B95927669A67CE6B2A
:10033000E954D969555E9C819567AA9BFE67529CDA
:100340005D68A64EE34FC853B9622B67AB6CC48F90
:10035000AD4F6D7EBF9E074E6261806E2B6F138521
:1003600073542A67459BF35D957BAC5CC65B1C8729
:100370004A6ED184147A088199598D7C116C20774A
:10038000D952225921715F72DB772797619D0B69E2
:100390007F5A185AA5510D547D540E66DF76F78F9B
:1003A0009892F49CEA595D72C56E4D51C968BF7D43
:1003B000EC7D6297BA9E7864216A028384595F5B00
:1003C000DB6B1B73F276B27D1780998432512867FC
:1003D000D99EEE766267FF520599245C3B627E7C73
:1003E000B08C4F55B6600B7D809501535F4EB65172
:1003F0001C593A723680CE91255FE2778453795F3B
:10040000047DAC85338A8D8E5697F367AE85539401
:1004100009610861B96C5276ED8A388F2F55514FBA
:100420002A51C752CB53A55B7D5EA0608261D66323
:100430000967DA67676E8C6D36733773317550797B
:10044000D588988A4A909190F590C4968D871559D1
:10045000884E594F0E4E898A3F8F1098AD507C5E62
:100460009659B95BB85EDA63FA63C164DC664A69BF
:10047000D8690B6DB66E94712875AF7A8A7F00804B
:100480004984C9848189218B0A8E65907D960A9959
:100490007E619162326B836C746DCC7FFC7FC06D2A
:1004A000857FBA87F8886567B1833C98F7961B6D9E
:1004B000617D3D846A91714E7553505D046BEB6FA5
:1004C000CD852D86A78929520F54655C4E67A86893
:1004D00006748374E275CF88E188CC91E2967896B1
:1004E0008B5F8773CB7A4E84A06365758952416DAB
:1004F0009C6E097459756B78927C8696DC7A8D9F18
:10050000B64F6E61C5655C86864EAE4EDA50214EA2
:10051000CC51EE5B99658168BC6D1F734276AD77F7
:100520001C7AE77C6F82D28A7C90CF91759618985E
:100530009B52D17D2B5098539767CB6DD0713374FC
:10054000E8812A8FA396579C9F9E60744158996DAD
:100550002F7D5E98E44E364F8B4FB751B152BA5D46
:100560001C60B2733C79D3823492B796F6960A97A0
:10057000979E629FA666746B1752A352C870C2887A
:10058000C95E4B609061236F49713E7CF47D6F8042
:10059000EE8423902C9342546F9BD36A8970C28C53
:1005A000EF8D3297B452415ACA5E045F17677C6977
:1005B00094696A6D0F6F6272FC72ED7B01807E80C0
:1005C0004B87CE906D51939E84798B803293D68ADF
:1005D0002D508C54718A6A6BC48C0781D160A067DE
:1005E000F29D994E984E109C6B8AC1856885006972
:1005F0007E6E977855810000002502250C25102578
:10060000182514251C252C25242534253C250125B9
:1006100003250F2513251B251725232533252B25DA
:100620003B254B2520252F25282537253F251D2512
:100630003025252538254225100411041204130401
:1006400014041504010416041704180419041A04E8
:100650001B041C041D041E041F0420042104220486
:1006600023042404250426042704280429042A0436
:100670002B042C042D042E042F0400000000000085
:10068000000000000000000000000000000000006A
:100690000000000000000000300431043204330484
:1006A00034043504510436043704380439043A0458
:1006B0003B043C043D043E043F0440044104420426
:1006C00043044404450446044704480449044A04D6
:1006D0004B044C044D044E044F040000910392035C
:1006E00093039403950396039703980399039A033E
:1006F0009B039C039D039E039F03A003A103A303ED
:10070000A403A503A603A703A803A90300000000F0
:10071000000000000000000000000000B103B20370
:10072000B303B403B503B603B703B803B903BA03FD
:10073000BB03BC03BD03BE03BF03C003C103C303AC
:10074000C403C503C603C703C803C90300000000F0
:100750000000000000000000000000010101010194
:100760000101010101000000000000000101010180
:100770000101010101010101010101010101010169
:100780000101010101010000000000000001010160
:100790000101010101010101010101010101010149
:1007A0000101010101010100C625A125A025B325F4
:1007B000B225BD25BC253B201230922190219121EC
:1007C0009321133000000000000000000000000032
:1007D0000000000000000000000008220B2286221A
:1007E0008722822283222A22292200000000000080
:1007F0000000000000000000000027222822AC00BA
:10080000D221D4210022032229220000000000006E
:100810000000000000000000000000000000202296
:10082000A522122302220722612252226A226B226F
:100830001A223D221D2235222B222C2200000000EC
:10084000000000000000000000002B2130206F2677
:100850006D266A2620202120B6002C2200000000F0
:100860000000EF250030013002300CFF0EFFFB309E
:100870001AFF1BFF1FFF01FF9B309C30B40040FF9D
:10088000A8003EFF3E203FFFFD30FE309D309E30F1
:100890000330DD4E053006300730FC3014201020C8
:1008A0000FFF3CFF1C3016205CFF2620252018205F
:1008B00019201C201D2008FF09FF143015303BFFB4
:1008C0003DFF5BFF5DFF083009300A300B300C3014
:1008D0000D300E300F30103011300BFF1222B100EE
:1008E000D700F7001DFF60221CFF1EFF6622672253
:1008F0001E22342242264026B0003220332003211B
:10090000A50004FFA200A30005FF03FF06FF0AFFE6
:1009100020FFA70006260526CB25CF25CE25C725F7
:1009200000000000000000000000000000000000C7
:1009300000000000000000000000000000000000B7
:1009400000000000000000000000000000000000A7
:1009500010111213141516171819000000000000CA
:10096000001A1B1C1D1E1F000000000000000000DC
:100970000000000000000000000000000000000077
:10098000001A1B1C1D1E1F000000000000000000BC
:100990000000000000000000000000000000000057
:1009A0000000000000000000000000000000000047
:1009B0000000000000000000000000000000000037
:1009C0000000000000000000000000000000000027
:1009D0000000000000000000000000000000000017
:1009E0000000000000000000000000000000000007
:1009F00000000000000000000000000000000000F7
:100A000000000000000000000000000000000000E6
:100A100000000000000000000000000000000000D6
:100A200005000000190000007D000000000000002B
:100A30000080E03779C34143176E05B5B5B89346DA
:100A4000F5F93FE9034F384D321D30F94877825AA6
:100A50003CBF737FDD4F1575000000000000F03FC4
:100A60000000000000002440000000000000594089
:100A70000000000000408F40000000000088C340DC
:100A800000000000006AF8400000000080842E4151
:100A900000000000D01263410000000084D797419D
:100AA0000000000065CDCD41000000205FA00242A3
:100AB000000000E876483742000000A2941A6D4218
:100AC000000040E59C30A2420000901EC4BCD6420B
:100AD00000003426F56B0C430080E03779C34143B6
:100AE00000A0D8855734764300C84E676DC1AB432C
:100AF000003D9160E458E143408CB5781DAF15444A
:100B000050EFE2D6E41A4B4492D54D06CFF0804424
:100B1000F64AE1C7022DB544B49DD9794378EA4439
:100B2000000000001F001C20000000001421000035
:100B30000200162400000000142500000200152801
:100B400000000000112900000000142A000000002D
:100B5000182B00000000142C00000000102D0000D5
:100B60000000142E000001000C3000000900143AAF
:100B700000000100183C00000200143F00000100CA
:100B8000034100001900155B00000000145C000028
:100B90000000115D00000000175E000000000F5F04
:100BA0000000000017600000000003610000190051
:100BB000157B00000000187C00000000117D000083
:100BC0000000187E00000000007F000020001CA034
:100BD0000000000014A10000000016A200000300A5
:100BE00019A60000000014A70000000017A80000CC
:100BF000000019A90000000006AA0000000013ABC5
:100C00000000000018AC0000000001AD0000000072
:100C100019AE0000000017AF0000000019B000007E
:100C2000000018B1000000000EB20000010017B46F
:100C30000000000003B50000000014B60000010031
:100C400017B8000000000EB90000000006BA00004E
:100C5000000012BB000000000EBC0000020014BF28
:100C60000000000003C00000160018D700000000BC
:100C700003D80000060004DF0000000003E00000CD
:100C8000160018F70000000003F800003F000438C9
:100C900001000000033901000F00044901000000B9
:100CA000034A01004200048D01000000038E010090
:100CB0000C00049B01000000039C01000D0004AA2D
:100CC0000100010003AC01000D0004BA01000000A6
:100CD00006BB0100000003BC0100010004BE0100CE
:100CE000000003BF0100000006C00100030003C4B0
:100CF0000100000007C50100000003C6010001005B
:100D000007C80100000003C90100010007CB010072
:100D1000000003CC0100230004F00100000003F1F7
:100D20000100000007F20100000003F301002D00A4
:100D3000042102000000032202001100043402001A
:100D40000500033A02001A00045502000000035691
:100D500002000100045802000000035902000000D4
:100D6000045A02000000035B02000100045D02005F
:100D7000020003600200010004620200000003633D
:100D8000020000000464020000000365020001008C
:100D9000046702000000036802000400046D020002
:100DA0000100036F020000000470020000000371E4
:100DB000020001000473020001000375020000003C
:100DC000047602000600037D02000000047E02009B
:100DD0000100038002000000048102000000038281
:100DE00002000100048402000200038702000500E3
:100DF000048D02000400039202000000049302002C
:100E00000000069402000000049502000700039D04
:100E100002000100049F0200100005B00200110052
:100E200017C20200030005C602000B0017D2020021
:100E30000D0005E00200040017E50200060005ECC5
:100E40000200000017ED0200000005EE02000000A5
:100E500017EF020010000B0003006F000370030087
:100E600003000574030000001775030000000376FB
:100E700003000100057A03000000037B0300020069
:100E8000147E03000000037F0300000017840300AA
:100E9000010003860300000014870300000003889C
:100EA00003000200038C03000000038E0300010016
:100EB00004900300000003910300100003A303004B
:100EC0000C0004B00300000003B10300200008D2AE
:100ED0000300020003D50300200018F60300000001
:100EE00003F70300040004FC0300000003FD0300FB
:100EF00084001982040000000B83040004000A88A7
:100F000004000100038A0400A50003310500250048
:100F1000055905000000145A05000500046005008D
:100F20000000036105002500048705000100148905
:100F300005000000108A05000000198D0500010061
:100F4000168F050000000B9105002C0010BE050057
:100F500000000BBF0500000014C0050000000BC11D
:100F60000500010014C3050000000BC405000100CA
:100F700014C6050000000BC70500000006D00500E0
:100F80001A0006EF0500030014F30500010001003C
:100F900006000500180606000200140906000100FC
:100FA000160B06000000140C06000100190E0600C6
:100FB00001000B1006000A00141B06000000011CB3
:100FC00006000000141D06000200062006001F0097
:100FD0000540060000000641060009000B4B060014
:100FE00014000C6006000900146A06000300066E77
:100FF000060001000B70060000000671060062008A
:1010000014D40600000006D5060000000BD606002A
:10101000060001DD0600000019DE060000000BDFFF
:101020000600050005E5060001000BE706000100CB
:1010300019E9060000000BEA0600030006EE0600B0
:1010400001000CF00600090006FA0600020019FD76
:101050000600010006FF06000000140007000D0056
:10106000010F070000000610070000000B11070029
:101070000000061207001D000B3007001A00064D85
:10108000070058000BA607000A0006B10700000081
:101090000CC00700090006CA070020000BEB070080
:1010A000080005F40700010019F60700000014F716
:1010B0000700020005FA070000000BFD0700000012
:1010C00016FE070001000600080015000B160800B8
:1010D0000300051A080000000B1B08000800052487
:1010E000080000000B250800020005280800000089
:1010F0000B2908000400143008000E000640080008
:1011000018000B5908000200145E08000000066079
:1011100008000A0006700800170017880800000081
:101120000689080005000190080001000B980800DE
:10113000070006A00800280005C9080000000BCA27
:101140000800170001E2080000000BE308001F0080
:101150000903090000000604090035000B3A0900E4
:101160000000093B090000000B3C09000000063D9F
:1011700009000000093E090002000B4109000700B8
:101180000949090003000B4D09000000094E090040
:1011900001000650090000000B5109000600065826
:1011A000090009000B620900010014640900010034
:1011B0000C6609000900147009000000057109009F
:1011C0000000067209000E000B8109000000098270
:1011D00009000100068509000700068F09000100CB
:1011E00006930900150006AA0900060006B20900C8
:1011F000000006B6090003000BBC0900000006BD94
:101200000900000009BE090002000BC1090003002B
:1012100009C70900010009CB090001000BCD090035
:10122000000006CE0900000009D70900000006DC16
:101230000900010006DF090002000BE209000100BD
:101240000CE60900090006F00900010016F2090089
:1012500001000EF40900050019FA0900000016FB50
:101260000900000006FC0900000014FD0900000050
:101270000BFE090000000B010A00010009030A002F
:10128000000006050A000500060F0A00010006130B
:101290000A001500062A0A00060006320A000100AC
:1012A00006350A00010006380A0001000B3C0A005E
:1012B0000000093E0A0002000B410A0001000B4732
:1012C0000A0001000B4B0A0002000B510A0000004B
:1012D00006590A000300065E0A0000000C660A00B8
:1012E00009000B700A00010006720A0002000B756B
:1012F0000A00000014760A0000000B810A000100B9
:1013000009830A00000006850A000800068F0A000B
:10131000020006930A00150006AA0A00060006B29B
:101320000A00010006B50A0004000BBC0A00000018
:1013300006BD0A00000009BE0A0002000BC10A0037
:1013400004000BC70A00010009C90A00000009CB0C
:101350000A0001000BCD0A00000006D00A000000C0
:1013600006E00A0001000BE20A0001000CE60A0098
:10137000090014F00A00000016F10A00000006F946
:101380000A0000000BFA0A0005000B010B00000028
:1013900009020B00010006050B000700060F0B00F9
:1013A000010006130B001500062A0B00060006328A
:1013B0000B00010006350B0004000B3C0B00000085
:1013C000063D0B000000093E0B0000000B3F0B0028
:1013D000000009400B0000000B410B00030009470F
:1013E0000B000100094B0B0001000B4D0B0000002E
:1013F0000B550B00010009570B000000065C0B00A9
:101400000100065F0B0002000B620B0001000C667E
:101410000B00090019700B00000006710B000000A2
:101420000E720B0005000B820B00000006830B0000
:10143000000006850B000500068E0B0002000692D8
:101440000B00030006990B000100069C0B00000036
:10145000069E0B00010006A30B00010006A80B006E
:10146000020006AE0B000B0009BE0B0001000BC012
:101470000B00000009C10B00010009C60B000200AF
:1014800009CA0B0002000BCD0B00000006D00B00B8
:10149000000009D70B0000000CE60B0009000EF05D
:1014A0000B00020019F30B00050016F90B000000F9
:1014B00019FA0B0000000B000C00000009010C00E1
:1014C00002000B040C00000006050C000700060ECD
:1014D0000C00020006120C001600062A0C000F0079
:1014E0000B3C0C000000063D0C0000000B3E0C0005
:1014F000020009410C0003000B460C0002000B4ADD
:101500000C0003000B550C00010006580C000200F3
:10151000065D0C00000006600C0001000B620C0070
:1015200001000C660C00090014770C0000000E7816
:101530000C000600197F0C00000006800C00000063
:101540000B810C00000009820C00010014840C00C7
:10155000000006850C000700068E0C0002000692B3
:101560000C00160006AA0C00090006B50C000400C9
:101570000BBC0C00000006BD0C00000009BE0C00F6
:1015800000000BBF0C00000009C00C0004000BC6DB
:101590000C00000009C70C00010009CA0C00010082
:1015A0000BCC0C00010009D50C00010006DD0C007D
:1015B000010006E00C0001000BE20C0001000CE64B
:1015C0000C00090006F10C00010009F30C000000FA
:1015D0000B000D00010009020D00010006040D00C2
:1015E0000800060E0D00020006120D0028000B3B3D
:1015F0000D000100063D0D000000093E0D00020037
:101600000B410D00030009460D000200094A0D00C0
:1016100002000B4D0D000000064E0D000000194F9A
:101620000D00000006540D00020009570D000000D7
:101630000E580D000600065F0D0002000B620D0043
:1016400001000C660D0009000E700D0008001979EC
:101650000D000000067A0D0005000B810D00000052
:1016600009820D00010006850D001100069A0D008B
:10167000170006B30D00080006BD0D00000006C0EF
:101680000D0006000BCA0D00000009CF0D0002007E
:101690000BD20D0002000BD60D00000009D80D0082
:1016A00007000CE60D00090009F20D00010014F41A
:1016B0000D00000006010E002F000B310E0000008F
:1016C00006320E0001000B340E000600163F0E001D
:1016D000000006400E00050005460E0000000B4706
:1016E0000E000700144F0E0000000C500E00090001
:1016F000145A0E00010006810E00010006840E003F
:10170000000006860E000400068C0E00170006A5D9
:101710000E00000006A70E0009000BB10E0000002D
:1017200006B20E0001000BB40E00080006BD0E004C
:10173000000006C00E00040005C60E0000000BC825
:101740000E0006000CD00E00090006DC0E0003009F
:1017500006000F00000019010F00020014040F0022
:101760000E0019130F00000014140F0000001915CB
:101770000F0002000B180F000100191A0F000500DE
:101780000C200F0009000E2A0F00090019340F0069
:1017900000000B350F00000019360F0000000B375A
:1017A0000F00000019380F0000000B390F00000077
:1017B000153A0F000000113B0F000000153C0F0010
:1017C0000000113D0F000000093E0F00010006401F
:1017D0000F00070006490F0023000B710F000D00DA
:1017E000097F0F0000000B800F00040014850F001C
:1017F00000000B860F00010006880F0004000B8D0F
:101800000F000A000B990F00230019BE0F000700FC
:101810000BC60F00000019C70F00050019CE0F00FE
:10182000010014D00F00040019D50F00030014D9D3
:101830000F000100060010002A00092B1000010013
:101840000B2D100003000931100000000B321000B6
:1018500005000938100000000B3910000100093B99
:10186000100001000B3D10000100063F10000000B9
:101870000C4010000900144A10000500065010002A
:1018800005000956100001000B5810000100065A0F
:10189000100003000B5E1000020006611000000043
:1018A00009621000020006651000010009671000BF
:1018B0000600066E100002000B7110000300067592
:1018C00010000C000B8210000000098310000100C2
:1018D0000B85100001000987100005000B8D10001A
:1018E0000000068E10000000098F100000000C9010
:1018F00010000900099A100002000B9D1000000062
:10190000199E1000010003A01000250003C710005D
:10191000000003CD1000000003D010002A0014FBCB
:101920001000000005FC1000000003FD1000020084
:10193000060011004801064A12000300065012007A
:101940000600065812000000065A12000300066046
:1019500012002800068A12000300069012002000E0
:1019600006B21200030006B81200060006C01200FC
:10197000000006C21200030006C812000E0006D8BE
:10198000120038000612130003000618130042006C
:101990000B5D130002001460130008000E691300B1
:1019A0001300068013000F0019901300090003A014
:1019B0001300550003F81300050010001400000088
:1019C000060114006B02196D16000000146E16005B
:1019D0000000066F160010001C8016000000068133
:1019E00016001900159B16000000119C160000003F
:1019F00006A016004A0014EB160002000DEE1600B9
:101A0000020006F1160007000600170011000B1275
:101A100017000200091517000000061F170012002A
:101A20000B321700010009341700000014351700AD
:101A300001000640170011000B521700010006605C
:101A400017000C00066E170002000B721700010051
:101A50000680170033000BB41700010009B6170009
:101A600000000BB71700060009BE170007000BC6E1
:101A70001700000009C7170001000BC917000A0072
:101A800014D41700020005D71700000014D817005F
:101A9000020016DB1700000006DC170000000BDD5B
:101AA000170000000CE0170009000EF017000900F5
:101AB0001400180005001006180000001407180094
:101AC00003000B0B18000200010E180000000B0FA2
:101AD000180000000C101800090006201800220051
:101AE0000543180000000644180034000680180062
:101AF00004000B85180001000687180021000BA9BF
:101B00001800000006AA1800000006B018004500E2
:101B1000060019001E000B201900020009231900FD
:101B200003000B27190001000929190002000930E0
:101B3000190001000B3219000000093319000500DB
:101B40000B39190002001940190000001444190053
:101B500001000C4619000900065019001D0006700E
:101B600019000400068019002B0006B019001900A6
:101B70000CD0190009000EDA1900000019DE190056
:101B8000210006001A0016000B171A00010009199F
:101B90001A0001000B1B1A000000141E1A0001009D
:101BA00006201A00340009551A0000000B561A00CE
:101BB000000009571A0000000B581A0006000B60BD
:101BC0001A00000009611A0000000B621A000000F0
:101BD00009631A0001000B651A000700096D1A005D
:101BE00005000B731A0009000B7F1A0000000C801F
:101BF0001A0009000C901A00090014A01A0006002F
